:1080000000000120755D0200ED310200ED3102003B
:10801000ED310200ED310200ED3102000000000000
:10802000000000000000000000000000ED31020030
:10803000ED31020000000000ED310200FDAD010055
:10804000ED310200ED310200ED310200ED310200B0
:10805000ED310200ED310200ED310200ED310200A0
:10806000ED310200ED310200ED310200ED31020090
:10807000ED310200ED310200ED310200ED31020080
:10808000ED310200ED310200ED310200ED31020070
:10809000ED310200ED310200ED310200ED31020060
:1080A000ED310200ED310200ED310200ED31020050
:1080B000ED310200ED310200ED310200ED31020040
:1080C000ED310200ED310200ED310200ED31020030
:1080D000ED310200ED310200ED310200ED31020020
:1080E000ED310200ED310200ED310200ED31020010
:1080F000ED3102003DC80100ED310200ED3102001A
:10810000ED310200D1C60100ED310200ED31020077
:10811000ED31020085BE0100ED310200ED310200BB
:10812000ED310200ED310200ED310200ED310200CF
:10813000ED310200ED310200ED31020079DE010087
:10814000B9D30100ED310200ED310200ED31020042
:10815000ED310200ED310200ED310200ED3102009F
:10816000ED31020075440200ED310200ED310200F4
:10817000ED310200ED310200ED310200ED3102007F
:10818000ED310200ED310200ED310200ED3102006F
:10819000ED310200ED310200ED310200ED3102005F
:1081A0004DD30100ED310200ED310200ED3102004E
:0C81B000ED310200ED310200ED31020063
:10840000FFFFFFFFFFFFFFFFFFFFFFFF7EF9FFFF03
:1084200010B5054C237833B9044B13B10448AFF3AE
:1084300000800123237010BD0010FF1F000000000A
:108440006090020008B5034B1BB103490348AFF32A
:10845000008008BD000000000410FF1F60900200B3
:1084600038B5064C2368C31AB3F5FA7F054604D322
:10847000034B9B699B699847256038BD1C10FF1F03
:108480003C7A020010B514F0C3FF064B00221A70AC
:10849000054B1B689847054B9B69BDE810405B691D
:1084A000184700BF300AFF1FB000FF1F3C7A0200D0
:1084B000431E2DE9F0471546072B00F24B82DFE8FB
:1084C00013F008000E000E0050006A00BA00F80019
:1084D000B101FFF7D7FF47F6A8532B603FE0A24B4F
:1084E000A24C022816BFA14699461C46A04BDF6845
:1084F000A9F10409043C4FF0FF364FF000084FF09B
:10850000010A3B68D9F804001B6998473B6860681A
:10851000DB6898473B6854F8040F5B6998473B68F1
:1085200059F8040F5B6A984718B90AFA08F326EA63
:1085300003063B6820689B6998473B68D9F80000B0
:108540005B6A984718B10AFA08F326EA030608F1AD
:108550000108B8F1110FD4D1C6F310062E60002027
:1085600020E0296003291CD8DFE801F0020A0E127E
:108570007F4BDB691B681A88322353431B14ACE71B
:108580007B4BDB695B68F6E7794BDB699B68F2E75D
:10859000784B1B69A1E7012929601CD004D302296B
:1085A0002FD00220BDE8F087714BDC68D4E90030A1
:1085B000DB6864309847D4E90030DB688430984742
:1085C000D4E900305B6964309847D4E900305B69D6
:1085D00084309847C3E7664BDC68D4E90030DB6839
:1085E000C4309847D4E90030DB68A4309847D4E918
:1085F00000305B69C4309847D4E900305B69A4302F
:10860000E7E75B4BDC68D4E90030DB6800F5A2707B
:108610009847D4E90030DB6800F5B2709847D4E998
:1086200000305B6900F5A2709847D4E900305B69BF
:1086300000F5B270CDE70129296025D019D30229B0
:10864000AFD14B4BDC68D4E90030DB6800F5A27099
:108650009847D4E90030DB6800F5B2709847D4E958
:1086600000305B6900F5A2709847D4E900309B693F
:10867000DEE73F4BDC68D4E90030DB6884309847A4
:10868000D4E900301B699EE7394BDC68D4E900303F
:10869000DB68C4309847D4E90030DB68A4309847E1
:1086A000D4E900305B69C4309847D4E900309B6955
:1086B000A5E7296000295FD001297FF472AF2C4B18
:1086C000DC68D4E90030DB6800F2C4609847D4E984
:1086D00000309B6900F2C4609847D4E90030DB6841
:1086E00000F2E4609847D4E900309B6900F2E4604E
:1086F0009847D4E90030DB6800F204709847D4E969
:1087000000309B6900F204709847D4E90030DB68C0
:1087100000F224709847D4E900309B6900F224707D
:108720009847D4E90030DB6800F244709847D4E9F8
:1087300000309B6900F244709847D4E90030DB6850
:1087400000F264709847D4E900309B6900F26470CD
:108750009847D4E90030DB6800F284709847D4E988
:1087600000309B695BE000BFF45AFF1FC059FF1F38
:108770003C7A0200300AFF1F774BDD68D5E90030F4
:10878000DB6800F2C4609847D5E900305B6900F20D
:10879000C4609847D5E90030DB6800F2E460984790
:1087A000D5E900305B6900F2E4609847D5E9003014
:1087B000DB6800F204709847D5E900305B6900F28D
:1087C00004709847D5E90030DB6800F224709847C0
:1087D000D5E900305B6900F224709847D5E9003094
:1087E000DB6800F244709847D5E900305B6900F21D
:1087F00044709847D5E90030DB6800F26470984710
:10880000D5E900305B6900F264709847D5E9003023
:10881000DB6800F284709847D5E900305B6900F2AC
:108820008470D6E6296000294AD001297FF4B9AEC8
:10883000494BDC68D4E90030DB6800F2845098478B
:10884000D4E900309B6900F284509847D4E90030A5
:10885000DB6800F2A4509847D4E900309B6900F22D
:10886000A4509847D4E90030DB6800F2C450984720
:10887000D4E900309B6900F2C4509847D4E9003035
:10888000DB6800F2E4509847D4E900309B6900F2BD
:10889000E4509847D4E90030DB6800F20460984760
:1088A000D4E900309B6900F204609847D4E90030B5
:1088B000DB6800F224609847D4E900309B6946E009
:1088C000254BDD68D5E90030DB6800F2845098471D
:1088D000D5E900305B6900F284509847D5E9003053
:1088E000DB6800F2A4509847D5E900305B6900F2DC
:1088F000A4509847D5E90030DB6800F2C45098478F
:10890000D5E900305B6900F2C4509847D5E90030E2
:10891000DB6800F2E4509847D5E900305B6900F26B
:10892000E4509847D5E90030DB6800F204609847CE
:10893000D5E900305B6900F204609847D5E9003062
:10894000DB6800F224609847D5E900305B6900F2EB
:1089500024603EE6042025E63C7A02003A4B3B4A7E
:10896000DB685B6803F59271116003F144015160AB
:1089700003F18401916003F1C401D16003F58271B8
:10898000116103F5B271516103F5D271916103F583
:10899000F271D16103F50971116203F51971516228
:1089A00003F52971916203F53971D16203F54971BB
:1089B000116303F55971516303F56971916303F50F
:1089C0007971D16303F224411164214A191D1160A8
:1089D00003F12401516003F16401916003F1A401EA
:1089E000D16003F1E401116103F5A271516103F556
:1089F000C271916103F5E271D16103F501711162F8
:108A000003F51171516203F52171916203F5317122
:108A1000D16203F54171116303F55171516303F59F
:108A20006171916303F5717103F204431364094B9F
:108A3000D16301221A70084B084A1A65084A9A65E0
:108A4000084A5A65704700BF3C7A0200C059FF1FB0
:108A5000F45AFF1F300AFF1F045AFF1FB1840000A1
:108A60008584000061840000704702207047022066
:108A700070477047704702207047022070470220FD
:108A80007047012070477047022070477047436964
:108A9000134A144910B5C3F80422C3F80822124B34
:108AA0008365124B8361C0E909131149C361C0E9B1
:108AB0000B13104B4364104B8364104B4363C0E9AA
:108AC0000F330F4B036600230E4C83660E4B0F4A89
:108AD00042658463C0E91314C265C0E91B3310BD4D
:108AE000838A00006B8A0000698A00006F8A000098
:108AF000778A0000738A0000758A00007B8A000074
:108B0000878A00007F8A0000898A00008D8A000021
:108B1000704700BF0A480B4B0022012110B44FF0F0
:108B2000FF3480F884205A7083F81012C0E91F4186
:108B3000C0F8883082671A70743010BCFFF7A7BF86
:108B4000045AFF1F2C10FF1F084A094800234FF04A
:108B5000FF314FF0010C1370537082F810324261F4
:108B6000C0E9021C03744360FFF791BF4C12FF1F62
:108B7000045AFF1F10B50023064C18461A5D590011
:108B800002F0030201338A40072B40EA0200F5D1CC
:108B900010BD00BF6C14FF1F044900235A5C02F093
:108BA0000302C2540133072BF8D170476C14FF1F26
:108BB000074B1A7802705A7842709A788270DA7885
:108BC000C2701A7902715A7942719B798371704728
:108BD0006C14FF1FF8B5094B094F0A4EDD680024DD
:108BE000E15D726C2B6852F82400DB6901F003012F
:108BF00001349847072CF3D1F8BD00BF3C7A02003E
:108C00006C14FF1F0800FF1F054A002300F003013A
:108C100099540133072B4FEA9000F7D1DAE700BFF0
:108C20006C14FF1F014B586AEEE700BF0800FF1FDE
:108C300004490023C25C02F003025A540133072B9B
:108C4000F8D1C7E76C14FF1F074B02781A704278FF
:108C50005A7082789A70C278DA7002791A71427901
:108C60005A7182799A71B5E76C14FF1F014B00228B
:108C70009A677047045AFF1F10B50348144615F051
:108C80008AFF206010BD00BFA014FF1F10B50F4C5D
:108C90000146204615F0EEFF002015F029FA6F215D
:108CA000204615F078FFC0F30061002015F0F2F9BE
:108CB000012015F01DFA7F21204615F06CFFBDE85C
:108CC0001040C0F30061012015F0E4B9A014FF1FAB
:108CD000014815F052BF00BFA014FF1F012808B5BE
:108CE00003D815F043F9002008BD0820FCE701284F
:108CF00008B503D815F014F9002008BD0820FCE7DA
:108D00000021F4E74942F2E7F1E7014815F099BF85
:108D1000A014FF1F38B5002015F07AFA08B1002022
:108D200038BD012015F074FA05460028F7D10C4C27
:108D3000204615F071FF15F0EBFA2B46D4F88C2283
:108D4000D4F88412284615F07BF901202B46D4F87C
:108D50009022D4F8881215F073F90120E0E700BFE3
:108D6000A014FF1F022804BF0C4B93F8E80038B989
:108D70000B4BDB681B685B690A4AD2F89402184700
:108D8000012809D1054B93F8E830012B04D1044B9D
:108D9000DB681B689B69EFE7704700BF045AFF1F41
:108DA0003C7A0200A014FF1F70B50020FFF7DAFF25
:108DB0000C4B0D4CDD68D4F894022B689B689847E7
:108DC0002B68D4F8A4029B6898472B68D4F8A802B3
:108DD0009B68984715F00EFB044BBDE870405B683C
:108DE000184700BF3C7A0200A014FF1FDC09FF1FD8
:108DF0000346052B10B5084614460BD006D8022BA7
:108E000006D315F061FA2060002010BD182BF8D0B1
:108E10000420FAE715F066FAF5E7012838B50446AC
:108E20000D4605D820B915F0F3F92860204638BD65
:108E30000820FCE7022810B5144611D0032817D0EB
:108E4000012819D10D4B0E4ADB68D2F8A4021B6829
:108E50005B6A9847003018BF01202060002010BDD9
:108E6000064B074ADB68D2F8A8021B685B6AF0E78A
:108E7000084615F0BDF8F0E70420F0E73C7A020060
:108E8000A014FF1F012838B504460D4608D815F078
:108E90009FF92B68C11829602046BDE838401DE7BE
:108EA000082038BDA32A2DE9F04105460C461E4690
:108EB00000F090814BD8072A00F0EC8024D8032AD8
:108EC00000F0BD800BD8012A00F0AA8040F29A8001
:108ED000002840F0AF80084615F0AAF996E0052A70
:108EE00000F0C08040F2B180202101FA04F444F087
:108EF0001004E4B22146B648002D40F0BD8015F0C4
:108F00004AFEC0F3042081E0322A00F0F2800FD83C
:108F10001C2A00F0D5801D2A00F0E780082A59D1CC
:108F2000002857D1084615F063F8C0F300106DE033
:108F30008C2A00F0ED80A22A00F03581332A49D135
:108F4000002840F0E080084615F0BEF95EE0AB2A4C
:108F500000F0F88132D8A72A4FEA011400F0B68158
:108F60001AD8A52A00F05F8140F2498144F06C04D0
:108F7000E4B22146964815F00EFE214600F48040EA
:108F8000002D40F09681002800F08D81904815F06A
:108F900002FEC0F3021039E0A92A00F0B68140F2C7
:108FA000A18144F06D04E4B221468948002D40F0CF
:108FB000C08115F0F0FDC0F3032027E0B32A00F0D4
:108FC000138209D8AD2A00F0DE81C0F0D081AE2A2C
:108FD00000F0EE81042520E0B52A00F02782C0F0E1
:108FE0001882B82A00F02C82CE2AF3D10028F1D1C1
:108FF000090141F06F01C9B2754815F0CCFDC0F30D
:10900000090003E020B9084615F0F2F8306004E0EA
:109010001968204614F0AAFF00252846BDE8F08113
:1090200018B9084615F0D4F8F0E71968204615F08D
:109030007DF8F1E71968204614F072FFECE700288C
:10904000C8D1084615F0E4F8E0E718B9084615F06D
:109050000FF9DBE719680029B8BF4942204615F02F
:1090600081F8D9E718B9084615F0F2F8CEE7196883
:10907000204615F0F0F9CFE715F08DFD33681B029F
:1090800003F4F85320F4F8521A432146504815F0DF
:1090900074FDC1E7202101FA04F444F01004E4B2A5
:1090A00021464B4825B915F076FD00F01F00ADE7CD
:1090B00015F071FD336820F01F0203F01F03E3E792
:1090C0000C0144F06C04E4B22146414825B915F086
:1090D00062FDC0F3804099E715F05DFD33689B04A5
:1090E00003F4802320F48022CEE700287FF472AFBF
:1090F000A8E718B9084615F0D9F887E71978204687
:1091000015F04CF888E71968204615F057F883E702
:1091100050B9090141F06C0101F0FC012C4815F037
:109120003AFDC0F3036071E71B68102B35D00DDCEE
:10913000022B2ED004DC012B16D04FF0FF3314E0AD
:10914000042B28D0082BF8D105230EE0402B26D085
:1091500003DC202BF1D1032307E0802B21D0B3F5D2
:10916000807FEAD1002300E00823336033680133B5
:109170003FF452AF240144F06C04E4B22146144899
:1091800015F009FD33681B0603F0706320F0706270
:109190007AE70723E9E70623E7E70423E5E7022365
:1091A000E3E70123E1E70C0144F06C04E4B221465B
:1091B000074825B915F0EFFCC0F3C13026E715F0DC
:1091C000EAFC3368DB0303F4C03320F4C0325BE70E
:1091D000A014FF1F0C0144F06C04E4B22146A34824
:1091E00025B915F0D8FCC0F380300FE715F0D3FC9B
:1091F00033689B0303F4804320F4804244E744F047
:109200006C04E4B22146994825B915F0C4FCC0F3BA
:109210000030FBE615F0BFFC33681B0303F48053FA
:1092200020F4805230E744F06C04E4B221468F48C9
:1092300015F0B1FC2146804600F480478B4885B983
:1092400027B115F0A8FCC0F3C310DFE615F0A3FCAE
:1092500018F4006FC0F3021018BF40F0080030602F
:10926000DAE647B115F097FC3368DB0103F4F063ED
:1092700020F4F06208E715F08EFC3268120120F04D
:10928000700002F0700202432146784815F075FC28
:109290002146764815F07FFC33681B0203F4006317
:1092A00020F40062F0E6714815F075FCC0F3C310BD
:1092B000D5E748B16D4815F06EFC33681B0103F02B
:1092C000700320F07002DFE66848CBE744F06C04DE
:1092D000E4B221466548002D4DD115F05CFC00F04C
:1092E0000F0093E644F06D04E4B221465F4825B9CF
:1092F00015F051FCC0F3C03088E615F04CFC336823
:10930000DB039BB220F40042BEE644F06D04E4B2FD
:109310002146564825B915F03EFCC0F3413075E6AC
:1093200015F039FC33685B0303F4C04320F4C042FA
:10933000AAE615F030FC33681B0203F4706320F4D6
:109340007062A1E60C0144F06D04E4B22146474886
:1093500025B915F020FCC0F3411057E615F01BFCB1
:1093600033685B0103F0600320F060028CE60C01BF
:1093700044F06D04ACE715F00EFC336820F00F02EA
:1093800003F00F0380E60C0144F06D04E4B22146C3
:10939000364825B915F0FFFBC0F3006036E615F03E
:1093A000FAFB33681B0603F0807320F080726BE6D3
:1093B0000C0144F06D04E4B221462C485DB915F06F
:1093C000EAFB001400F07F0310F0400018BF6FF0BC
:1093D0007F0018431AE615F0DEFB33681B0403F424
:1093E000FE0320F4FE024FE60C0144F06C04E4B2EC
:1093F00021461E4825B915F0CEFBC0F3404005E6D6
:1094000015F0C9FB33685B0403F4003320F4003229
:109410003AE600287FF4DEAD090141F06F01C9B2E0
:10942000124815F0B8FBC0F30440EFE518B9084640
:1094300014F02EFFEAE51968204614F0A1FEEBE5D2
:109440000C0144F06C04E4B22146084825B915F03B
:10945000A2FBC0F34030D9E515F09DFB33685B03F8
:1094600003F4005320F400520EE600BFA014FF1FC7
:1094700007B50129019207D8024601AB0120FFF789
:1094800011FD03B05DF804FB0820FAE7012913463B
:1094900002D80246002005E508207047022806D3BE
:1094A000052801D9182802D1002010607047042037
:1094B0007047034BD3F8B0320846DB6811461847B3
:1094C000A014FF1F2DE9F0415B4C5C4D5C4FD4F8BC
:1094D00088205C4B0121284615F082FBFE687368EA
:1094E00003F16402C5F8942203F1E402C5F8A8224E
:1094F00003F58272C5F8A42203F5A272C5F88C2286
:1095000003F5B27203F59270C5F8882203F5C272B2
:1095100003F50173C5F8AC323368C5F89022DB68F7
:10952000C5F8840298473368D5F88C02DB68984701
:109530003368D5F88802DB6898473368D5F890021D
:10954000DB6898473368D5F89402DB68984733683E
:10955000D5F8AC02DB6898473B6903F11402C5F803
:10956000B022D5F8AC229A6114F0D2FE0023D5F8CF
:109570008C22D5F88412184614F062FDD5F88812B2
:10958000D5F890220023012014F05AFDD4F8883039
:109590002D4AC3F804222D4AC3F8082200250122CF
:1095A0001A705D702A4BC4F894302A4BC4F890307E
:1095B000294BC4F88C30294BC4F89830284BC4F898
:1095C000AC30284BC4F8A830274BC4F89C30274B4C
:1095D000C4F8A030264BC4F8BC30264BC4F8B830D1
:1095E000254BC4F8C830254BC4F8C430244BC4F80C
:1095F000C030244BC4F8D430234BC4F8D0303222CE
:109600004FF48F73C4E91F32204BC4F8CC30204B89
:10961000C4F8E03002201F4B84F88400C4F8E43022
:109620001D4CFFF79FFB23689847A36829462846EF
:10963000BDE8F041184700BF045AFF1FA014FF1FE8
:109640003C7A020014600200158D00000B8D0000B2
:10965000EF8C0000098D0000058D0000018D0000D9
:109660008D94000071940000DD8C0000858E000058
:10967000D18C0000798C00008D8C0000358E0000AC
:109680001B8E0000658D00006D8C0000A98D000010
:109690009D940000F18D0000DC09FF1F014B104676
:1096A000DB6B18470800FF1F034B10B51B6C1446FB
:1096B0009847206010BD00BF0800FF1F062873B543
:1096C00004460E467BD8404D68462B6B013C9847BC
:1096D0002B46042C04D8DFE804F00866696C6F00A0
:1096E0009DF80030336000200BE09DF80120E97800
:1096F000914208D19DF80200297B884203D10020C5
:10970000306002B070BD1979914206D19DF8020017
:10971000597B884201D10123E4E75979914206D16E
:109720009DF80200997B884201D10223DAE79979FA
:10973000914206D19DF80200D97B884201D10323D2
:10974000D0E7D979914206D19DF80200197C884270
:1097500001D10423C6E7597A914206D19DF802004F
:10976000997C884201D10523BCE7997A914206D1C0
:109770009DF80200D97C884201D10623B2E7197A0C
:10978000914206D19DF80200597C884201D10723FD
:10979000A8E7D97A914214D19DF802201B7D9A4204
:1097A0000FD108239EE79DF803309BE79DF8043016
:1097B00098E79DF8053095E79DF8063092E704207C
:1097C0009FE710209DE700BF0800FF1F07B5034B70
:1097D00068461B6B984703B05DF804FB0800FF1F49
:1097E00070B50020FFF7F2FF1E4B1F4CDD68206BA9
:1097F0002B689B6898472B68E06A9B6898472B68A2
:10980000E0689B6898472B68A0689B6898472B681E
:1098100060689B6898472B6820689B6898472B680E
:10982000A0699B6898472B68E0699B6898472B68FC
:10983000A06A9B6898472B6860699B6898472B686B
:10984000206A9B6898472B68606A9B6898472B68DA
:1098500020699B68984714F0CDFD044BBDE870402B
:109860005B6818473C7A02006017FF1FDC09FF1F86
:10987000002014F03DBC10B5044618B914F076FB76
:10988000204610BD0820FCE710B5044618B914F0B6
:1098900047FB204610BD0820FCE70021F4E74942C1
:1098A000F2E7F1E7062873B505460C465DD80229B4
:1098B00003D901285BD10F2959DC2E4E6846336B42
:1098C00098473346052D06D8DFE805F0030B4346DD
:1098D000494C8DF800406846DB6A9847002002B08A
:1098E00070BD082CF7D8DFE804F0050C11161B201A
:1098F000252A2F00F2788DF80120327B8DF8022086
:10990000E9E732798DF80120727BF7E772798DF8FB
:109910000120B27BF2E7B2798DF80120F27BEDE70E
:10992000F2798DF80120327CE8E7727A8DF8012017
:10993000B27CE3E7B27A8DF80120F27CDEE7327A7E
:109940008DF80120727CD9E7F27A8DF80120327D02
:10995000D4E78DF80340BEE78DF80440BBE78DF8EF
:109960000540B8E78DF80640B5E70420B7E71020BA
:10997000B5E700BF0800FF1F38B5154618B101282C
:1099800007D0042004E0084614F032FB28600020D1
:1099900038BD094B094DDC68094B606800F59270D1
:1099A000D8616B6C58612368DB6898476A6C2368E0
:1099B00050699B699847EAE73C7A02000800FF1F5C
:1099C0006017FF1F38B50D46044648B914F000FC77
:1099D0002B68C1182960204614F0C8FA204638BD0B
:1099E0000820FCE770B5054616460C4600295DD1F7
:1099F0000B2810D806283CD202282ED004D808B351
:109A0000012825D0042421E004282ED029D9084695
:109A100014F01EFC1FE013280CD80E283CD20C2892
:109A20002FD00D28EED1224B224ADB68106B1B6829
:109A30005B6A2CE0322835D03328E3D1084614F095
:109A400043FC08E014F0D4FB2C463060204670BD87
:109A5000084614F0BDFB3060F8E7084614F0E8FB58
:109A6000F9E7084614F0D4FBF5E7084614F000FCCB
:109A7000F1E70828C6D1084614F0BAFAC0F300107E
:109A8000E9E70B4B0B4ADB68D06A1B685B6A9847B7
:109A9000003018BF0120DEE70E381146C0B2FFF7D4
:109AA0000DFED3E7084614F001FCD4E70824CDE707
:109AB0003C7A02006017FF1F30B585B00546019261
:109AC0000C4600296ED10B2812D8062846D202284F
:109AD00037D004D848B301282CD004242EE0042821
:109AE00034D00528F9D11146204614F0B4FC25E005
:109AF00013280FD80E2845D20C2836D00D28ECD1CB
:109B000042F210739A42E8D8274B91B29B682046E4
:109B1000984713E0332837D08C283AD03228DCD14C
:109B2000D1B2204614F03AFB08E0114614F01EFAB8
:109B30002C4603E01146204614F0F8FA204605B002
:109B400030BD1146204614F0EBF9F7E782EAE271E6
:109B5000A1EBE271204614F005FBEFE70638114651
:109B6000C0B2FFF79FFE0446E8E7104B1049DB68E0
:109B7000C86A1B68154612B15B699847DEE79B69A6
:109B80009847D5E70E38EAE71146204614F016FB51
:109B9000D4E701A90120FFF791FD064B04469B6B1A
:109BA00002A8EAE70824C9E7DC09FF1F3C7A0200A3
:109BB0006017FF1F0800FF1F6C4B2DE9F041DE68A6
:109BC0006B4C70686B4F00F5E273236300F5D27342
:109BD000E36200F52173E36000F52973A36000F5EB
:109BE0001973636000F50173236000F55973A36175
:109BF00000F55173E36100F16403A36200F5A27301
:109C0000636100F56973236200F571736362336801
:109C100000F59270DB682061984733686069DB6803
:109C200098473368206BDB6898473368E06ADB68E5
:109C300098473368206A1B6998473368606A1B69D4
:109C400098477B6CE2681A60A2685A6062689A6002
:109C50002268DA60A2691A61E2695A61A26A9A61AD
:109C600000257A6C33685059DB6898477A6C336802
:109C700050599B69043598471C2DF2D13E4DD5F8BB
:109C800088304FF0000883F8008014F041FBD4E9DD
:109C900004124346404614F0D3F944F6206140468E
:109CA00014F060FA46F2A811404614F0D4FB334B8E
:109CB000C5F89430324BC5F89030324BC5F88C3033
:109CC000314BC5F89830314BC5F8AC30304BC5F846
:109CD000A830304BC5F89C302F4BC5F8A0302F4B27
:109CE000C5F8BC302E4BC5F8B8302E4BC5F8C43083
:109CF0002D4BC5F8C8302D4BC5F8D430012385F85D
:109D0000843002202A4BC5F8CC30FFF75FFD404677
:109D100014F07EFA10B1274B9B789BB1BB6A984731
:109D200014F0F6FA0023D4E90412184614F088F966
:109D300044F62061002014F015FA46F2A811002024
:109D400014F089FB3368206BDB689847206B1A4C52
:109D50000423437533681B6898472368984700219C
:109D6000A3680846BDE8F041184700BF3C7A0200EE
:109D70006017FF1F0800FF1F045AFF1F899800008B
:109D8000A39800009F9800009B980000E5990000B0
:109D9000B99A000077980000C59900009D960000D0
:109DA000A99600007999000071980000CD970000F5
:109DB000E1970000300AFF1FDC09FF1F1B4B70B545
:109DC000DD681B4C2B68A0685B6998472B6820688E
:109DD0009B6898472B6860689B6898472B68206A47
:109DE0009B6898472B68606A9B6898472B68E06877
:109DF0009B6898472B6820699B6898472B68606927
:109E00009B6898472B68A0699B6898472B68E06916
:109E10009B6898472B68A0689B68984714F0EAFAFB
:109E2000044BBDE870405B68184700BF3C7A0200F5
:109E3000A017FF1FDC09FF1F10B5144605284CD8DA
:109E4000DFE800F0032220313C41146844F620632F
:109E50009C4244D8234B244ADB68106A1B6842F2B8
:109E600010718C42DB6994BF00210121984742F2B6
:109E70001173B4FBF3F103FB11411C4B89B29B68D6
:109E800000209847002010BD164B2468DA68D2E9FC
:109E9000003000F5F2701CB1DB6900219847F1E752
:109EA0009B689847EEE70F4B1168DB680E4A1B680A
:109EB0001069DB69003118BF0121EFE7084614F093
:109EC00097F82060DEE7074B074ADB6858681B6895
:109ED00000F592701061DB68E3E70420D3E71020FF
:109EE000D1E700BF3C7A0200A017FF1FDC09FF1F6B
:109EF00010B50348144614F03AFF206010BD00BFAF
:109F0000385BFF1F10B5094C0146204614F09EFF38
:109F1000002014F0EDF86F21204614F028FFBDE872
:109F20001040C0F30061002014F0B4B8385BFF1F8C
:109F3000014814F00EBF00BF385BFF1F10B5044688
:109F400018B914F013F8204610BD0820FCE710B52E
:109F5000044618B913F0E4FF204610BD0820FCE7C2
:109F60000021F4E74942F2E7F1E7014814F055BF58
:109F7000385BFF1F022804BF0B4B93F8E80030B991
:109F80000A4BDB681B685B69094A9068184701281F
:109F900009D1054B93F8E830012B04D1034BDB6862
:109FA0001B689B69F0E77047045AFF1F3C7A020068
:109FB000A017FF1F0346052B10B5084614460BD00B
:109FC00006D8022B06D314F07FF92060002010BDC4
:109FD000182BF8D00420FAE714F084F9F5E738B527
:109FE0000D46044620B914F013F92860204638BD08
:109FF0000820FCE7012903D1024A702114F0A9BE10
:10A00000704700BFC8040500A52970B50446154671
:10A0100000F0538200F28C80172900F077812DD850
:10A02000042900F036810CD8012900F01481C0F019
:10A030000781022900F01881032900F01F81042400
:10A04000F9E1072900F049810ED8052900F02D819A
:10A050000629F4D11021C048002C40F0308114F0C2
:10A0600086FEC0F30420EEE0082900F046811529A1
:10A07000E5D10028E3D0126811212AE1322900F04D
:10A08000A1812FD81B2900F079810ED8182900F062
:10A090005C811A29D3D16C21AF48002C40F0638138
:10A0A00014F065FEC0F38040CDE01C2900F07781FC
:10A0B0001D29C4D10028C2D1204614F005F912216F
:10A0C0000646A54814F053FEC0F313027A20D317B6
:10A0D000A6FB00011BF096FC00F11303262B98BF92
:10A0E0000020B0E0A22900F0BD8112D8332900F091
:10A0F00072818C29A3D1002840F077816C21964889
:10A1000014F035FE4FF48073C0F3036043FA00F09F
:10A1100099E0A32900F0B781A42990D16C218E4841
:10A12000002C40F0C18114F022FEC0F300308AE020
:10A13000B42900F0BF823FD8AA2900F0658214D864
:10A14000A72900F03682C0F00982A82900F04182D8
:10A15000A9297FF474AF6D217F48002C40F04B8219
:10A1600014F005FEC0F341306DE0AD2900F07082BF
:10A1700012D8AB2900F05982AC297FF460AF6D2171
:10A180007548002C00F0188214F0F1FD2B6820F0C7
:10A190000F0203F00F032BE2AE2900F06A82B3290D
:10A1A0007FF44DAF6C216C48002C40F07A8214F0A3
:10A1B000DEFDC0F3404046E0BB2900F0CF821BD853
:10A1C000B82900F099820BD8B52900F07D82B62914
:10A1D0007FF435AF614E002840F08082142198E072
:10A1E000B92900F09A82BA297FF429AF5B4E002882
:10A1F00040F0A68213218CE0C02900F0EE820FD837
:10A20000BC2900F0CB82BF297FF419AF002840F0B1
:10A21000D4827021504814F0AAFDC0F3014012E02E
:10A22000CC2900F0EA82CE297FF409AF00287FF420
:10A2300006AF6F21484814F09AFDC0F3090002E010
:10A2400018B913F0D5FF2860F5E01168002013F06D
:10A250008DFE0024EFE010B913F0BAFFF3E71168A8
:10A26000002013F063FFF4E718B9002013F0E0FFBB
:10A27000E9E71168002013F053FEEAE700287FF4B5
:10A28000DEAE14F013F800287FF416AF13F0C0FF11
:10A29000D9E710B913F0ECFFD5E711680029B8BF72
:10A2A0004942002013F05EFFD3E718B9002013F0F5
:10A2B000CFFFC8E71168002014F0CDF8C9E714F00B
:10A2C00056FD2B681B0203F4F85320F4F8521A438E
:10A2D0001021214814F03DFDBBE710211E4824B990
:10A2E00014F045FD00F01F00ADE714F040FD2B68B1
:10A2F00020F01F0203F01F03E9E700287FF49FAE60
:10A30000002013F075FEC0F300109CE7134E70B9E7
:10A310001521114814F02BFD002800F00F824FF09A
:10A32000807393FBF0F0B042A8BF3046E2E01368C0
:10A330004BB14FF0807292FBF3F2B242A8BF3246AB
:10A340002A601521C5E73246FAE748B933210248A9
:10A3500014F00DFD77E700BF385BFF1FFFFF0F0014
:10A3600012683321B5E714F002FD2B689B0403F457
:10A37000802320F480221A436C21AAE76C21B34881
:10A3800024B914F0F4FCC0F3C0405CE714F0EFFC17
:10A390002B68DB0403F4002320F40022EBE7002108
:10A3A000AA4824B914F0E3FCC0F340004BE714F0D2
:10A3B000DEFC2B685B0003F0020320F002021A436C
:10A3C000002186E710B913F071FF3CE711780020F7
:10A3D00013F0E4FE3DE718B9002013F075FF32E7F3
:10A3E0001168002013F0EAFE33E71368102B28D021
:10A3F0000DDC022B21D004DC012B16D04FF0FF33F3
:10A4000014E0042B1BD0082BF8D105230EE0402BC1
:10A4100019D003DC202BF1D1032307E0802B14D0CB
:10A42000B3F5807FEAD1002300E008232B602B687E
:10A4300001330CD11024204670BD0723F6E7062314
:10A44000F4E70423F2E70223F0E70123EEE76C21AF
:10A450007E4814F08CFC2B681B0603F0706320F020
:10A46000706288E76C21794824B914F080FCC0F34D
:10A47000C130E8E614F07BFC2B68DB0303F4C03347
:10A4800020F4C03277E76C21704824B914F06FFCD7
:10A49000C0F38030D7E614F06AFC2B689B0303F40A
:10A4A000804320F4804266E714F061FC2B681B03B4
:10A4B00003F4805320F480525DE76C216348DCB9DB
:10A4C00014F055FC10F480464FF06C015F4804D046
:10A4D00014F04DFCC0F3C310B5E614F048FC6C2139
:10A4E00004465A4814F043FCC0F30210230548BF49
:10A4F00040F008002860ACE614F039FC10F4804409
:10A500004FF06C01514808D014F031FC2B68DB018E
:10A5100003F4F06320F4F0622DE714F028FC6C21C2
:10A520004A4814F024FC2A68120220F4006002F465
:10A53000006202436C21454814F00BFC6C21434837
:10A5400014F015FC2B681B0103F0700320F070025F
:10A550001A436C213D4814F0FCFB6CE76C213B482E
:10A56000B4B914F004FC10F4804F4FF06C0137487C
:10A5700004D014F0FCFBC0F3021064E614F0F7FB07
:10A580006C210446314814F0F2FBC0F3C310ADE770
:10A5900014F0EDFB10F4804F4FF06C012B48B3D05A
:10A5A00014F0E5FB2B681B0103F0700320F0700230
:10A5B000E1E66C21254824B914F0D9FB00F00F0026
:10A5C00041E614F0D4FB2B6820F00F0203F00F03D8
:10A5D000D1E66D211D4824B914F0C9FBC0F3C03089
:10A5E00031E614F0C4FB2B68DB039BB220F400427D
:10A5F0001A436D216DE614F0BAFB2B685B0303F47C
:10A60000C04320F4C042F3E76D21104824B914F090
:10A61000AEFBC0F3032016E614F0A9FB2B681B0267
:10A6200003F4706320F47062E2E76D21074824B9F7
:10A6300014F09DFBC0F3411005E614F098FB2B6865
:10A640005B0103F0600320F06002D1E7385BFF1F7D
:10A650006D21724824B914F08AFBC0F30060F2E562
:10A6600014F085FB2B681B0603F0807320F08072CA
:10A67000BEE76D2169485CB914F079FB001400F065
:10A680007F0310F0400018BF6FF07F001843DAE539
:10A6900014F06DFB2B681B0403F4FE0320F4FE0290
:10A6A000A6E714F064FB2B685B0403F4003320F48A
:10A6B000003260E600287FF4C2AC6F21574814F0E6
:10A6C00056FBC0F30440BEE518B9002013F0E0FDCE
:10A6D000B9E51168002013F053FDBAE513684BB1DA
:10A6E0004FF0807292FBF3F2B242A8BF32462A606A
:10A6F0001421EEE53246FAE76C21484824B914F0FB
:10A7000036FBC0F340309EE514F031FB2B685B0351
:10A7100003F4005320F400522DE66C213F4824B985
:10A7200014F025FBC0F303508DE514F020FB2B68DB
:10A730001B0503F4700320F470021CE63046D9E6D2
:10A7400013684BB14FF0807292FBF3F2B242A8BF94
:10A7500032462A601321BCE53246FAE770212F48C1
:10A7600024B914F004FBC0F307206CE514F0FFFAE1
:10A770002A68120220F47F4092B2024370212748D7
:10A7800014F0E7FA0021254814F0F1FA2B68002BA9
:10A7900020F00402CCBF0423002310E670211F48E0
:10A7A0001CB914F0E4FAC0B24DE514F0E0FA2A78CE
:10A7B00020F0FF00024370218BE51368032B3FF666
:10A7C00039AE7021154814F0D2FA2B681B0403F43B
:10A7D000403320F440321A43EDE770210F48002C3B
:10A7E0003FF45EAC14F0C3FA2B68002B20F48022F7
:10A7F00014BF4FF480230023EDE77021074824B9EC
:10A8000014F0B5FAC0F301501DE514F0B0FA2B684E
:10A810001B0503F4401320F44012DCE7385BFF1FF4
:10A820000B4619B901461846FFF7EEBB08207047E2
:10A8300008B5002013F0ECFC10B1084B987860B11B
:10A84000074814F0D5FA13F063FD064900231846B3
:10A85000D1E9001213F0F4FB012008BD300AFF1FFC
:10A86000385BFF1FA017FF1F38B50D46044648B9D7
:10A8700013F0AEFC2B68C1182960204613F076FB5C
:10A88000204638BD0820FCE707B5019239B90146DA
:10A8900001AA0120FFF7B8FB03B05DF804FB082014
:10A8A000FAE7022806D3052801D9182802D100208A
:10A8B0001060704704207047044B9B6E0846114699
:10A8C00003B11847024B1B68DB68FAE7045AFF1F05
:10A8D000BC5DFF1F2DE9F041694D6A4CD5F8882019
:10A8E000694B6A4F2046012114F066FA68492046F8
:10A8F00014F0A8FAFE68674C736803F16402A26062
:10A9000003F59272226003F5A272626003F5D272BF
:10A91000226203F5E272626203F55172E26003F5AE
:10A92000597203F56970226103F5617203F5717361
:10A93000E361336862611B69A06198473368E0692D
:10A940001B699847336860691B69984733682068BA
:10A95000DB68984733686068DB6898473368A068AD
:10A96000DB68984733682069DB6898473368E0689C
:10A97000DB6898473368606ADB6898473368206A09
:10A98000DB6898473368606A9B6998473368206A38
:10A990009B699847336860699B6998473368E068AA
:10A9A0009B6998473A693C4B02F11401196073683E
:10A9B00003F50173936113F0ABFC0023D4E900129B
:10A9C000184613F03DFBD5F88830344AC3F804220A
:10A9D000334AC3F80822002701221A705F70314BF6
:10A9E000C5F89430304BC5F89030304BC5F88C30FA
:10A9F0002F4BC5F898302F4BC5F8AC302E4BC5F80F
:10AA0000A8302E4BC5F89C302D4BC5F8A0302D4BEF
:10AA1000C5F8BC302C4BC5F8B8302C4BC5F8C83045
:10AA20002B4BC5F8C4302B4BC5F8C0302A4BC5F8AA
:10AA3000D43085F884204FF4F0733222C5E91F32F8
:10AA4000264BC5F8CC30264BC5F8E0300220254B0C
:10AA5000C5F8E430FFF78EFA3368606ADB68984720
:10AA6000606A214C0423437533681B689847236848
:10AA70009847A36839463846BDE8F041184700BFFB
:10AA8000045AFF1F385BFF1F146202003C7A020069
:10AA9000F59F0000A017FF1FBC5DFF1F31A800003D
:10AAA0006B9F00004F9F0000699F0000659F0000A2
:10AAB000619F000021A8000089A800003D9F0000C0
:10AAC00069A80000319F0000F19E0000059F000072
:10AAD000399E0000DF9F0000759F0000BD9D0000B3
:10AAE000A3A80000B59F0000DC09FF1F38B5184B74
:10AAF000184CDD6820682B685B6998472B68606894
:10AB00009B6898472B68A0689B6898472B68E0680B
:10AB10009B6898472B6820699B6898472B686069F9
:10AB20009B6898472B68A0699B6898472B68E069E9
:10AB30009B6898472B68206A9B68984713F05AFCDB
:10AB4000054B5B689847002384F8243038BD00BF6C
:10AB50003C7A0200D417FF1FDC09FF1F10B5034821
:10AB6000144614F0F0F9206010BD00BFC45DFF1F53
:10AB7000014814F0DAB900BFC45DFF1F10B50446E8
:10AB800018B913F0F3F9204610BD0820FCE710B502
:10AB9000044618B913F0C4F9204610BD0820FCE79C
:10ABA0000021F4E74942F2E7F1E7014814F047BA1F
:10ABB000C45DFF1F022804BF0B4B93F8E80030B9B7
:10ABC0000A4BDB681B685B69094A10681847012853
:10ABD00009D1054B93F8E830012B04D1034BDB6816
:10ABE0001B689B69F0E77047045AFF1F3C7A02001C
:10ABF000D417FF1F10B51446062844D8DFE800F02C
:10AC00000416142530353F00136844F62062934241
:10AC10003BD842F21172B3FBF2F102FB11311C4B33
:10AC200089B29B6800209847002010BD194B24680A
:10AC3000DA68D2E9003000F5F2701CB1DB6900215E
:10AC40009847F1E79B689847EEE7124B1168DB687D
:10AC5000114A1B685069DB69003118BF0121EFE719
:10AC6000084613F0C5F92060DEE70A4B0A4ADB68A4
:10AC700058681B6800F592705061DB68E3E70220BA
:10AC8000FFF798FFD0E70420CFE71020CDE700BF03
:10AC9000DC09FF1F3C7A0200D417FF1F0346052B77
:10ACA00010B5084614460BD006D8022B06D313F075
:10ACB0000BFB2060002010BD182BF8D00420FAE711
:10ACC00013F010FBF5E738B50D46044620B913F034
:10ACD0009FFA2860204638BD0820FCE738B5194C9B
:10ACE000054694F8240001281CD002281FD02946CC
:10ACF000154814F0BDF9002013F0FAF9002013F004
:10AD000077F910F008041BD1820619D56F210E487F
:10AD100014F019F9C30113D520460221BDE83840CB
:10AD200013F03CB9A562022384F82430DFE7A36A5C
:10AD3000EB1AB3F5FA6FDAD9FFF73CFF0323F3E719
:10AD400038BD00BFD417FF1FC45DFF1FA52970B514
:10AD50000446154600F0538200F28C80172900F05B
:10AD600077812DD8042900F036810CD8012900F014
:10AD70001481C0F00781022900F01881032900F036
:10AD80001F810424F9E1072900F049810ED8052923
:10AD900000F02D810629F4D11021C048002C40F08C
:10ADA000308114F0D0F8C0F30420EEE0082900F060
:10ADB00046811529E5D10028E3D0126811212AE146
:10ADC000322900F0A1812FD81B2900F079810ED8FB
:10ADD000182900F05C811A29D3D16C21AF48002CCE
:10ADE00040F0638114F0AFF8C0F38040CDE01C293F
:10ADF00000F077811D29C4D10028C2D1204613F06C
:10AE000063FA12210646A54814F09DF8C0F3130218
:10AE10007A20D317A6FB00011AF0F4FD00F113030A
:10AE2000262B98BF0020B0E0A22900F0BD8112D8E7
:10AE3000332900F072818C29A3D1002840F077815A
:10AE40006C21964814F07FF84FF48073C0F30360D0
:10AE500043FA00F099E0A32900F0B781A42990D12A
:10AE60006C218E48002C40F0C18114F06CF8C0F3C6
:10AE700000308AE0B42900F0BF823FD8AA2900F050
:10AE8000658214D8A72900F03682C0F00982A8296B
:10AE900000F04182A9297FF474AF6D217F48002C16
:10AEA00040F04B8214F04FF8C0F341306DE0AD2913
:10AEB00000F0708212D8AB2900F05982AC297FF4DF
:10AEC00060AF6D217548002C00F0188214F03BF83B
:10AED0002B6820F00F0203F00F032BE2AE2900F0E5
:10AEE0006A82B3297FF44DAF6C216C48002C40F08E
:10AEF0007A8214F028F8C0F3404046E0BB2900F005
:10AF0000CF821BD8B82900F099820BD8B52900F060
:10AF10007D82B6297FF435AF614E002840F08082F3
:10AF2000142198E0B92900F09A82BA297FF429AF58
:10AF30005B4E002840F0A68213218CE0C02900F06F
:10AF4000EE820FD8BC2900F0CB82BF297FF419AF65
:10AF5000002840F0D4827021504813F0F4FFC0F371
:10AF6000014012E0CC2900F0EA82CE297FF409AF3B
:10AF700000287FF406AF6F21484813F0E4FFC0F3C8
:10AF8000090002E018B913F033F92860F5E0116800
:10AF9000002012F0EBFF0024EFE010B913F018F9D5
:10AFA000F3E71168002013F0C1F8F4E718B90020A6
:10AFB00013F03EF9E9E71168002012F0B1FFEAE76B
:10AFC00000287FF4DEAE13F071F900287FF416AF8D
:10AFD00013F01EF9D9E710B913F04AF9D5E7116853
:10AFE0000029B8BF4942002013F0BCF8D3E718B9D4
:10AFF000002013F02DF9C8E71168002013F02BFA98
:10B00000C9E713F0A0FF2B681B0203F4F85320F4E8
:10B01000F8521A431021214813F087FFBBE7102193
:10B020001E4824B913F08FFF00F01F00ADE713F0A6
:10B030008AFF2B6820F01F0203F01F03E9E70028B6
:10B040007FF49FAE002012F0D3FFC0F300109CE706
:10B05000134E70B91521114813F075FF002800F048
:10B060000F824FF0807393FBF0F0B042A8BF3046E0
:10B07000E2E013684BB14FF0807292FBF3F2B24200
:10B08000A8BF32462A601521C5E73246FAE748B91B
:10B090003321024813F057FF77E700BFC45DFF1F5D
:10B0A000FFFF0F0012683321B5E713F04CFF2B6848
:10B0B0009B0403F4802320F480221A436C21AAE726
:10B0C0006C21B34824B913F03EFFC0F3C0405CE7E5
:10B0D00013F039FF2B68DB0403F4002320F4002273
:10B0E000EBE70021AA4824B913F02DFFC0F340007C
:10B0F0004BE713F028FF2B685B0003F0020320F0FE
:10B1000002021A43002186E710B913F0CFF83CE79A
:10B110001178002013F042F83DE718B9002013F031
:10B12000D3F832E71168002013F048F833E71368CA
:10B13000102B28D00DDC022B21D004DC012B16D0E3
:10B140004FF0FF3314E0042B1BD0082BF8D105235C
:10B150000EE0402B19D003DC202BF1D1032307E0B4
:10B16000802B14D0B3F5807FEAD1002300E00823C0
:10B170002B602B6801330CD11024204670BD0723AF
:10B18000F6E70623F4E70423F2E70223F0E70123BE
:10B19000EEE76C217E4813F0D6FE2B681B0603F009
:10B1A000706320F0706288E76C21794824B913F04D
:10B1B000CAFEC0F3C130E8E613F0C5FE2B68DB031E
:10B1C00003F4C03320F4C03277E76C21704824B90F
:10B1D00013F0B9FEC0F38030D7E613F0B4FE2B684D
:10B1E0009B0303F4804320F4804266E713F0ABFE38
:10B1F0002B681B0303F4805320F480525DE76C211D
:10B200006348DCB913F09FFE10F480464FF06C01E8
:10B210005F4804D013F097FEC0F3C310B5E613F0F7
:10B2200092FE6C2104465A4813F08DFEC0F30210C2
:10B23000230548BF40F008002860ACE613F083FE09
:10B2400010F480444FF06C01514808D013F07BFE9D
:10B250002B68DB0103F4F06320F4F0622DE713F0B8
:10B2600072FE6C214A4813F06EFE2A68120220F426
:10B27000006002F4006202436C21454813F055FE61
:10B280006C21434813F05FFE2B681B0103F0700331
:10B2900020F070021A436C213D4813F046FE6CE723
:10B2A0006C213B48B4B913F04EFE10F4804F4FF0C0
:10B2B0006C01374804D013F046FEC0F3021064E678
:10B2C00013F041FE6C210446314813F03CFEC0F3FC
:10B2D000C310ADE713F037FE10F4804F4FF06C0150
:10B2E0002B48B3D013F02FFE2B681B0103F0700323
:10B2F00020F07002E1E66C21254824B913F023FE0A
:10B3000000F00F0041E613F01EFE2B6820F00F0244
:10B3100003F00F03D1E66D211D4824B913F013FE8D
:10B32000C0F3C03031E613F00EFE2B68DB039BB296
:10B3300020F400421A436D216DE613F004FE2B68E1
:10B340005B0303F4C04320F4C042F3E76D211048CF
:10B3500024B913F0F8FDC0F3032016E613F0F3FD53
:10B360002B681B0203F4706320F47062E2E76D2126
:10B37000074824B913F0E7FDC0F3411005E613F0C8
:10B38000E2FD2B685B0103F0600320F06002D1E76F
:10B39000C45DFF1F6D21724824B913F0D4FDC0F3C2
:10B3A0000060F2E513F0CFFD2B681B0603F08073FD
:10B3B00020F08072BEE76D2169485CB913F0C3FDCF
:10B3C000001400F07F0310F0400018BF6FF07F0002
:10B3D0001843DAE513F0B7FD2B681B0403F4FE03F2
:10B3E00020F4FE02A6E713F0AEFD2B685B0403F425
:10B3F000003320F4003260E600287FF4C2AC6F21F5
:10B40000574813F0A0FDC0F30440BEE518B9002072
:10B4100012F03EFFB9E51168002012F0B1FEBAE566
:10B4200013684BB14FF0807292FBF3F2B242A8BFA7
:10B4300032462A601421EEE53246FAE76C2148488C
:10B4400024B913F080FDC0F340309EE513F07BFD7E
:10B450002B685B0303F4005320F400522DE66C21AB
:10B460003F4824B913F06FFDC0F303508DE513F08E
:10B470006AFD2B681B0503F4700320F470021CE6C0
:10B480003046D9E613684BB14FF0807292FBF3F26D
:10B49000B242A8BF32462A601321BCE53246FAE721
:10B4A00070212F4824B913F04EFDC0F307206CE53E
:10B4B00013F049FD2A68120220F47F4092B2024341
:10B4C0007021274813F031FD0021254813F03BFD82
:10B4D0002B68002B20F00402CCBF0423002310E6CD
:10B4E00070211F481CB913F02EFDC0B24DE513F0BA
:10B4F0002AFD2A7820F0FF00024370218BE51368B3
:10B50000032B3FF639AE7021154813F01CFD2B6854
:10B510001B0403F4403320F440321A43EDE770215A
:10B520000F48002C3FF45EAC13F00DFD2B68002B90
:10B5300020F4802214BF4FF480230023EDE7702114
:10B54000074824B913F0FFFCC0F301501DE513F0C8
:10B55000FAFC2B681B0503F4401320F44012DCE7CF
:10B56000C45DFF1F0B4619B901461846FFF7EEBB35
:10B570000820704708B5002012F04AFE10B1084BB1
:10B58000987860B1074813F045FD12F0C1FE0649F6
:10B5900000231846D1E9011212F052FD012008BD26
:10B5A000300AFF1FC45DFF1FD417FF1F012910B50C
:10B5B00004460DD1074A702113F0B7FC2046064A15
:10B5C0000A2113F0B2FC2046BDE8104013F0FCBC89
:10B5D00010BD00BF1E000CC40004080038B50D46A5
:10B5E000044648B912F0F4FD2B68C11829602046C2
:10B5F00012F0BCFC204638BD0820FCE707B50192DC
:10B6000039B9014601AA0120FFF7A0FB03B05DF89C
:10B6100004FB0820FAE7022806D3052801D91828D8
:10B6200002D100201060704704207047044B9B6ECD
:10B630000846114603B11847024B1B68DB68FAE75E
:10B64000045AFF1FC05DFF1F2DE9F0415A4C5B4DAE
:10B65000D4F888205A4B5B4F2846012113F098FC00
:10B660005949284613F000FDFE68584D736803F1F0
:10B6700064022A6003F592726A6003F5A272AA60FE
:10B6800003F5E272EA6003F551722A6103F559721B
:10B6900003F561706A6103F5697203F571732B62DA
:10B6A0003368EA611B69A861984733682868DB68DA
:10B6B000984733686868DB6898473368A868DB6830
:10B6C00098473368E868DB68984733686869DB68DF
:10B6D000984733682869DB6898473368E8685B698E
:10B6E00098473368A8699B699847336828699B69BC
:10B6F00098473A69364B02F114011960736803F5F3
:10B700000173936112F004FE0023D5E9011218467B
:10B7100012F096FCD4F888302E4AC3F804222E4A40
:10B72000C3F80822002601225E701A702B4BC4F861
:10B7300094302B4BC4F890302A4BC4F88C302A4BF1
:10B74000C4F89830294BC4F8AC30294BC4F8A83061
:10B75000284BC4F89C30284BC4F8A030274BC4F8C1
:10B76000BC30274BC4F8B830264BC4F8C830264B41
:10B77000C4F8C430254BC4F8C030254BC4F8D430CD
:10B7800032214FF4F073C4E91F31224BC4F8CC309E
:10B79000214BC4F8E030214BC4F8E43084F8842015
:10B7A0001F4C85F8242023689847A368314630460B
:10B7B000BDE8F041184700BF045AFF1FC45DFF1FDA
:10B7C000146402003C7A0200ADB50000D417FF1FDC
:10B7D000C05DFF1F75B50000ABAB00008FAB000074
:10B7E000A9AB0000A5AB0000A1AB000065B500004F
:10B7F000FDB500007DAB0000DDB5000071AB0000C1
:10B800005DAB0000DDAC0000F5AB0000C7AC000094
:10B81000B5AB0000EDAA000017B600009DAC00001B
:10B82000DC09FF1F014B00229A677047045AFF1F73
:10B83000F8B50A4E30460C4650F8047B154613F016
:10B84000E8FC2B4622460146384610F0CAFF7368D2
:10B8500004F07F0403EB84046560F8BD0C18FF1F3F
:10B8600008B50146034813F05FFC0020BDE808401E
:10B8700012F03EBC1018FF1F38B51546044628B913
:10B88000084612F0B5FB2860204638BD0420FCE7CE
:10B8900010B5044618B912F069FB204610BD082007
:10B8A000FCE710B5044618B912F03AFB204610BD6B
:10B8B0000820FCE70021F4E74942F2E7F1E70148FC
:10B8C00013F09DBC1018FF1F10B5084C12F020FD9E
:10B8D0000023D4F8A022D4F89C12184612F0B0FB32
:10B8E000201DBDE8104013F072BC00BF0C18FF1FF4
:10B8F000022804BF0C4B93F8E80038B90B4BDB6807
:10B900001B685B690A4AD2F898021847012809D1D6
:10B91000054B93F8E830012B04D1044BDB681B681E
:10B920009B69EFE7704700BF045AFF1F3C7A020093
:10B930000C18FF1F38B50020FFF7DAFF144B154C29
:10B94000DD68D4F898022B689B6898472B68D4F878
:10B950009C029B6898472B68D4F8A0029B68984784
:10B960002B68D4F8A4029B6898472B68D4F8A802E7
:10B970009B6898472B68D4F8AC029B6898472B6863
:10B98000D4F8B0029B689847BDE8384012F032BD49
:10B990003C7A02000C18FF1F70B50E4801F07F03BF
:10B9A0001446C2180D4692F81422D2070BD550F84F
:10B9B000046B13F02EFC23462A4601463046BDE8B0
:10B9C000704010F0C7BE416801EB83014B682360F3
:10B9D00070BD00BF0C18FF1F38B50D46044648B9AE
:10B9E00012F0F6FB2B68C1182960204612F0BEFA4F
:10B9F000204638BD0820FCE710B5144629BB0628B0
:10BA000025D8DFE800F0040A0E12161A1E000020E6
:10BA100012F0EEFB2060002010BD002012F0D8FBD9
:10BA2000F8E7002012F004FCF4E7002012F0F0FB2D
:10BA3000F0E7002012F01CFCECE7002012F008FCFC
:10BA4000E8E7044813F0E5FBE4E70820E4E7042016
:10BA5000E2E700BF1018FF1F08B549BB062829D828
:10BA6000DFE800F0040A0F28141C21001146002012
:10BA700012F07CFA002008BD1146002012F056FB9F
:10BA8000F8E71146002012F04BFAF3E782EAE27180
:10BA9000A1EBE271002012F065FBEBE711460020FC
:10BAA00012F0D9FCE6E7D1B2034813F0B5FBE1E7A9
:10BAB0000820E0E70420DEE71018FF1FF8B5012298
:10BAC000544E554C1146072012F0BEFDF5686B68C8
:10BAD00003F59272C4F89C2203F5A272C4F8A02266
:10BAE00003F1C402C4F8A42203F1E40203F16400E8
:10BAF000C4F8A82203F18402A433C4F8B0322B683E
:10BB0000C4F8AC22DB68C4F8980298472B68D4F8D4
:10BB10009C02DB6898472B68D4F8A002DB68984742
:10BB20002B68D4F8A402DB6898472B68D4F8A802E5
:10BB3000DB6898472B68D4F8AC021B6998472B68E0
:10BB4000D4F8B0021B6998472746F36A47F8043BCC
:10BB500000251D705B689847304B3149D3F8882029
:10BB6000C2F804122F49C2F8081201262E49167095
:10BB70005570C3F894102D49C3F890102C49C3F8A0
:10BB80008C102C49C3F898102B49C3F8AC102B49E2
:10BB9000C3F8A8102A49C3F89C102A49C3F8A0107A
:10BBA0002949C3F8BC102949C3F8B8102849C3F87B
:10BBB000C4102849C3F8D4102749C3F8D010322044
:10BBC0004FF4C371C3E91F102449C3F8CC102449B2
:10BBD00083F884603846C3F8C8102946214B13F017
:10BBE00083FA12F095FB2B46D4F8A022D4F89C12CD
:10BBF000284612F025FA28464FF4484112F0B2FACE
:10BC000028464FF4484112F026FC3046BDE8F84083
:10BC10006EE600BF3C7A02000C18FF1F045AFF1F9B
:10BC2000C9B80000BFB80000A3B80000BDB800004C
:10BC3000B9B80000B5B80000F9B9000059BA000061
:10BC400091B80000D9B9000031B8000099B90000DE
:10BC500079B80000F1B8000025B8000035B900003F
:10BC600061B8000014660200014B00229A67704719
:10BC7000045AFF1FF8B50A4E30460C4650F8047BB4
:10BC8000154613F060FB2B4622460146384610F05D
:10BC9000A8FD736804F07F0403EB84046560F8BDBD
:10BCA000CC1AFF1F08B50146034813F0D7FA00204D
:10BCB000BDE8084012F01CBAD01AFF1F10B50B46A1
:10BCC000144606286AD8DFE800F004090F131B2881
:10BCD0004A00084612F08CF9206003E021783048D1
:10BCE00013F034FB002010BD2D4813F02CFBF3E7BC
:10BCF00023685A1E534253412A4A82F89832F1E788
:10BD000023684FF4FA5159436423B1FBF3F1264BF6
:10BD100089B29B6802209847E4E72168214A013BE9
:10BD200001F00301D2F89C02042B06D8DFE803F0EF
:10BD3000030B0E111400D2F8A0021C4BDB681B6829
:10BD4000DB699847CEE7D2F8AC02F6E7D2F8B0024A
:10BD5000F3E7D2F8BC02F0E7D2F8C002EDE71149F0
:10BD6000013BD1F89C02042B06D8DFE803F0030B5B
:10BD70000E111400D1F8A0020C4BDB681B681B6A83
:10BD80009847A9E7D1F8AC02F6E7D1F8B002F3E79B
:10BD9000D1F8BC02F0E7D1F8C002EDE70420A2E739
:10BDA000D01AFF1FCC1AFF1FDC09FF1F3C7A0200CC
:10BDB00010B5044618B912F0D9F8204610BD082075
:10BDC000FCE710B5044618B912F0AAF8204610BDD9
:10BDD0000820FCE70021F4E74942F2E7F1E70148D7
:10BDE00013F0A7BAD01AFF1F10B5084C12F090FA42
:10BDF0000023D4F8A822D4F8A412184612F020F98F
:10BE0000201DBDE8104013F07CBA00BFCC1AFF1F04
:10BE1000022804BF0C4B93F8E80038B90B4BDB68E1
:10BE20001B685B690A4AD2F89C021847012809D1AD
:10BE3000054B93F8E830012B04D1044BDB681B68F9
:10BE40009B69EFE7704700BF045AFF1F3C7A02006E
:10BE5000CC1AFF1F70B50020FFF7DAFF1D4B1E4CF8
:10BE6000DD68D4F89C022B689B6898472B68D4F84F
:10BE7000A0029B6898472B68D4F8A4029B68984757
:10BE80002B68D4F8A8029B6898472B68D4F8AC02BA
:10BE90009B6898472B68D4F8B0029B6898472B683A
:10BEA000D4F8B4029B6898472B68D4F8B8029B6812
:10BEB00098472B68D4F8C0029B6898472B68D4F841
:10BEC000BC029B68984712F095FA044BBDE870409D
:10BED0005B6818473C7A0200CC1AFF1FDC09FF1F81
:10BEE0002DE9F74F3A4C94F898320D469046002BC6
:10BEF00055D0002953D1D2F80090DFF8DCA04FF0E4
:10BF0000030BEBB2B9F1000F06D1D4F8C432C8F874
:10BF1000003003B0BDE8F08F052BF6D8DFE803F062
:10BF2000032B2E313437D4F89C62DAF80C300193AD
:10BF30001A6809F00307D26830469047022F019B28
:10BF400028D0032F13D0012F1B6826D15B69304600
:10BF500098476A0002F4FF72D4F8C4320BFA02F177
:10BF6000974023EA01030F401F43C4F8C4724FEA0D
:10BF700099090135C5E7D4F8A062D6E7D4F8AC62D8
:10BF8000D3E7D4F8B062D0E7D4F8BC62CDE7D4F8F8
:10BF9000C062CAE71B689B68D9E79B69D7E705F0D1
:10BFA0007F02A31893F81432DB070CD509482468E4
:10BFB00013F0C9F9434601462A46204603B0BDE8BE
:10BFC000F04F10F0C7BB636803EB82035B689EE72A
:10BFD000CC1AFF1FD01AFF1F3C7A020038B50D465D
:10BFE000044648B912F0F4F82B68C11829602046BD
:10BFF00011F0BCFF204638BD0820FCE710B5144600
:10C0000029BB062825D8DFE800F0040A0E12161A0C
:10C010001E00002012F0ECF82060002010BD00206F
:10C0200012F0D6F8F8E7002012F002F9F4E7002049
:10C0300012F0EEF8F0E7002012F01AF9ECE7002019
:10C0400012F006F9E8E7044813F07DF9E4E7082068
:10C05000E4E70420E2E700BFD01AFF1F08B549BBA0
:10C06000062829D8DFE800F0040A0F28141C210054
:10C070001146002011F07AFF002008BD1146002073
:10C0800012F054F8F8E71146002011F049FFF3E7E9
:10C0900082EAE271A1EBE271002012F063F8EBE7B3
:10C0A0001146002012F0D7F9E6E7D1B2034813F0A9
:10C0B0004DF9E1E70820E0E70420DEE7D01AFF1F92
:10C0C0002DE9F04101226B4E6B4C1146072012F016
:10C0D000BBFAF5686B6803F5B272C4F8A02203F5E9
:10C0E0009272C4F8A42203F5A272C4F8A82203F144
:10C0F000C402C4F8AC2203F1E402C4F8B02203F194
:10C10000840203F16400C4F8B42203F1A40203F52D
:10C11000C273C4F8BC322B68C4F8B822DB68C4F818
:10C120009C02C4F8C00298472B68D4F8A002DB68D0
:10C1300098472B68D4F8A402DB6898472B68D4F89A
:10C14000A802DB6898472B68D4F8AC02DB689847F4
:10C150002B68D4F8B002DB6898472B68D4F8B40297
:10C160001B6998472B68D4F8B8021B6998472B685D
:10C17000D4F8AC029B6998472B68D4F8B0029B694D
:10C180009847A046F36A48F8043B01271F705B6894
:10C1900098473A4B3A49D3F88820C2F804123949F3
:10C1A000C2F808120026384917705670C3F8941068
:10C1B0003649C3F890103649C3F88C103549C3F896
:10C1C00098103549C3F8AC103449C3F8A810344965
:10C1D000C3F89C103349C3F8A0103349C3F8BC100E
:10C1E0003249C3F8B8103249C3F8C4103149C3F812
:10C1F000D4103149C3F8D01032204FF4C371C3E9D1
:10C200001F102E49C3F8CC102D4983F88470404686
:10C21000C3F8C81031462B4B13F002F812F078F82F
:10C22000D4F8A822D4F8A4123346304611F008FFFF
:10C2300030464FF4484111F095FF4FF448413046E5
:10C2400012F009F92B68D4F8BC02DB689847D4F8DF
:10C25000BC021D4C042343752B681B689847236858
:10C260009847A3683146022098473846BDE8F04118
:10C27000CEE500BF3C7A0200CC1AFF1F045AFF1F14
:10C28000E9BD0000DFBD0000C3BD0000DDBD000052
:10C29000D9BD0000D5BD0000FDBF00005DC000009D
:10C2A000B1BD0000DDBF000075BC0000E1BE0000B4
:10C2B000BDBC000011BE000069BC000055BE0000FE
:10C2C000A5BC000014680200DC09FF1F014B00221E
:10C2D0009A677047045AFF1F074870B550F8044B1F
:10C2E0000D46164613F091F833462A46014620467D
:10C2F000BDE8704010F075BAA01DFF1F074870B56B
:10C3000050F8044B0D46164613F07FF833462A4684
:10C3100001462046BDE8704010F01CBAA01DFF1F6A
:10C3200008B5064A0146D2F894320020043213F0D0
:10C330004BF80020BDE8084011F0DABEA01DFF1F39
:10C3400038B51546044628B9084611F051FE286054
:10C35000204638BD0420FCE710B5044618B911F09A
:10C3600005FE204610BD0820FCE710B5044618B9AC
:10C3700011F0D6FD204610BD0820FCE70021F4E7AF
:10C380004942F2E7F1E7024BD3F8940213F034B8D4
:10C39000A01DFF1F10B5084C11F0BAFF0023D4F800
:10C3A000A022D4F89C12184611F04AFED4F8940248
:10C3B000BDE8104013F017B8A01DFF1F022804BFEE
:10C3C0000C4B93F8E80038B90B4BDB681B685B69D2
:10C3D0000A4AD2F898021847012809D1054B93F868
:10C3E000E830012B04D1044BDB681B689B69EFE745
:10C3F000704700BF045AFF1F3C7A0200A01DFF1FB8
:10C4000038B50020FFF7DAFF164B174CDD68D4F87B
:10C4100098022B689B6898472B68D4F89C029B680D
:10C4200098472B68D4F8A0029B6898472B68D4F8EB
:10C43000A4029B6898472B68D4F8A8029B68984789
:10C440002B68D4F8AC029B6898472B68D4F8B002EC
:10C450009B68984723689B689847BDE8384011F06F
:10C46000C9BF00BF3C7A0200A01DFF1F38B50D46B2
:10C47000044648B911F0ACFE2B68C118296020466B
:10C4800011F074FD204638BD0820FCE710B51446B5
:10C4900029BB062825D8DFE800F0040A0E12161A78
:10C4A0001E00002011F0A4FE2060002010BD00201E
:10C4B00011F08EFEF8E7002011F0BAFEF4E700203C
:10C4C00011F0A6FEF0E7002011F0D2FEECE700200C
:10C4D00011F0BEFEE8E7044812F097FFE4E70820F9
:10C4E000E4E70420E2E700BFA41DFF1F08B549BB35
:10C4F000062829D8DFE800F0040A0F28141C2100C0
:10C500001146002011F032FD002008BD1146002028
:10C5100011F00CFEF8E71146002011F001FDF3E7E1
:10C5200082EAE271A1EBE271002011F01BFEEBE761
:10C530001146002011F08FFFE6E7D1B2034812F058
:10C5400067FFE1E70820E0E70420DEE7A41DFF1F06
:10C5500070B50122524C534E1146072012F074F868
:10C56000201D12F0F7FEF5686B6803F59272C4F8AF
:10C570009C2203F5A272C4F8A02203F1C402C4F8FD
:10C58000A42203F1E40203F16400C4F8A82203F139
:10C590008402A433C4F8B0322B68C4F8AC22DB6840
:10C5A000C4F8980298472B68D4F89C02DB68984737
:10C5B0002B68D4F8A002DB6898472B68D4F8A40253
:10C5C000DB6898472B68D4F8A802DB6898472B688B
:10C5D000D4F8AC021B6998472B68D4F8B0021B69E9
:10C5E0009847F36A23605B6898472F4B2F49D3F82D
:10C5F0008820C4F8942200250126C2F804122C4990
:10C6000016705570C2F808122A4AC3F894202A4AB4
:10C61000C3F89020294AC3F88C20294AC3F89820EF
:10C62000284AC3F8AC20284AC3F8A820274AC3F8F0
:10C630009C20274AC3F8A020264AC3F8BC20264ADB
:10C64000C3F8B820254AC3F8C420254AC3F8D4202B
:10C65000244AC3F8D02032214FF4C372C3E91F210A
:10C66000214AC3F8CC20214A83F88460C3F8C8204B
:10C6700011F04EFE2B46D4F8A022D4F89C12284686
:10C6800011F0DEFC28464FF4484111F06BFD2846BE
:10C690004FF4484111F0DFFE3046BDE870408DE6B2
:10C6A000A01DFF1F3C7A0200045AFF1F95C3000023
:10C6B00087C300006BC3000085C3000081C3000076
:10C6C0007DC300008DC40000EDC4000059C300000C
:10C6D0006DC40000D9C20000FDC2000041C30000CB
:10C6E000BDC30000CDC2000001C4000021C3000092
:10C6F000012810B514460CD003D3022810D0042012
:10C7000006E01368094AB3FA83F35B0993730020C8
:10C7100010BD1368064AB3FA83F35B091360F6E7AA
:10C72000084611F065FC2060F1E700BF6020FF1FA4
:10C730006C00FF1F10B50348144612F0B5FE2060D0
:10C7400010BD00BF6020FF1F014812F09BBE00BF5C
:10C750006020FF1FF8B5374C374D064600212046B4
:10C7600012F0A2FE2A79C0F3C017BA4217D00621F0
:10C770002046002F4CD012F097FE00F01F00E0730F
:10C780000621204612F090FE237903F01F0320F0CB
:10C790001F021A430621204612F074FE2F71274A09
:10C7A000217B936F00293ED043F00103617B002978
:10C7B0003CD043F002030020936711F029FD636928
:10C7C00094F84C200028B8BF4042984234BF00275C
:10C7D0000127BA4213D098424FF0050115482CBFEB
:10C7E000657C257C12F060FE05F00F0520F00F023D
:10C7F0002A4305210F4812F045FE84F84C7031465B
:10C800000C4812F09BFE0020BDE8F84011F070BC0F
:10C8100012F04AFE00F01F0020710621204612F09F
:10C8200043FEE37BB1E723F00103BFE723F00203FC
:10C83000C1E700BF6020FF1F6C00FF1F045AFF1FED
:10C8400010B5044618B911F091FB204610BD082020
:10C85000FCE7014812F0E3BE6020FF1F022804BF7E
:10C860000B4B93F8E80030B90A4BDB681B685B6937
:10C87000094AD06D1847012809D1054B93F8E830D3
:10C88000012B04D1034BDB681B689B69F0E7704701
:10C89000045AFF1F3C7A02006020FF1F38B50020B9
:10C8A000FFF7DCFF0F4B104CDD68E06D2B685B6918
:10C8B00098472B68206D9B6898472B68A06D9B68F4
:10C8C00098472B68E06D9B6898472B68206E9B68A3
:10C8D00098472B68606D9B689847BDE8384011F019
:10C8E00089BD00BF3C7A02006020FF1F0346052B74
:10C8F00010B5084614460BD006D8022B06D311F00B
:10C90000E3FC2060002010BD182BF8D00420FAE7CB
:10C9100011F0E8FCF5E738B50D46044620B911F0F2
:10C9200077FC2860204638BD0820FCE710B5044697
:10C9300028B9044B988111F0F3FA204610BD082065
:10C94000FCE700BF6020FF1F0021EFE74942EDE751
:10C95000ECE7A729F8B504460E46154600F01D82FF
:10C9600067D81D2900F0038121D8042900F0068131
:10C970000CD8012900F0E880C0F0DA80022900F02C
:10C98000EC80032900F0F3800424D5E0062900F0B0
:10C990000A81C0F0FF80072900F01E810829F3D129
:10C9A0000028F1D111F024FBC0F30010C3E0A1294D
:10C9B00000F08F811BD8332900F0298108D8322953
:10C9C000E2D1002840F01E81002011F06FFCB2E09F
:10C9D0008C2900F02581A029D6D1002840F06E8155
:10C9E0000821B44812F060FDC0F34020A3E0A42960
:10C9F00000F0A2810ED8A22900F07E81A329C3D124
:10CA0000002840F08E810C21AA4812F04DFDC0F3A1
:10CA1000803090E0A52900F0A281A629B4D1002899
:10CA200040F0B0810C21A34812F03EFDC0F302108B
:10CA300081E0B22900F04D8241D8AC2900F0FC81A0
:10CA400013D8A92900F0CD81C0F0B981AA2900F03E
:10CA5000D981AB2998D105219648002C40F0E3817B
:10CA600012F022FDC0F3411065E0AF2900F005820D
:10CA700015D8AD2900F0E781AE2985D106218D4872
:10CA8000002C40F0F18112F00FFD000A00F07F034E
:10CA900010F0400018BF6FF07F0018434BE0B02942
:10CAA00000F0FD81B1297FF46FAF07218148002C90
:10CAB00040F0068212F0F8FCC0F380203BE0B7297A
:10CAC00000F0408210D8B42900F02582C0F0128214
:10CAD000B52900F02A82B6297FF456AF754B00289D
:10CAE00040F02D825B6961E0CE2900F04F8213D8BF
:10CAF000B82900F03782B9297FF446AF07216D4885
:10CB0000002C00F0A38112F0CFFC2B681B0403F46F
:10CB1000803320F48032BFE1D02900F04D82D62945
:10CB20007FF432AF634B002840F04F829B683DE0BA
:10CB300020B911F05DFB28602046F8BD1168002087
:10CB400011F014FA0024F7E710B911F041FBF2E7F5
:10CB50001168002011F0EAFAF4E718B9002011F08A
:10CB600067FBE8E71168002011F0DAF9EAE7002C2A
:10CB70007FF40AAF204611F04BFBDCE710B911F04F
:10CB800077FBD8E711680029B8BF4942002011F0AF
:10CB9000E9FAD7E710B911F05BFBCCE71168002088
:10CBA00011F059FCCEE7434F10B9FB7B2B60C3E774
:10CBB0001368FB73404B1C79002CC3D1384612F02C
:10CBC00073FCFB7B20F01F0203F01F031A43314666
:10CBD000384612F057FCAFE7364E08B93379E5E72F
:10CBE00013683371344B1B79012BABD106213148CB
:10CBF00012F05AFC337920F01F0203F01F031A438E
:10CC0000062148E01178002011F0C8FA9AE710B91F
:10CC100011F05AFB8FE71168002011F0CFFA91E76D
:10CC200040B90821234812F03FFC00F00F00C0F18A
:10CC3000080080E71368102B35D00DDC022B2ED0B6
:10CC400004DC012B16D04FF0FF3314E0042B28D066
:10CC5000082BF8D105230EE0402B26D003DC202B37
:10CC6000F1D1032307E0802B21D0B3F5807FEAD1F7
:10CC7000002300E008232B602B68013300F0A8811B
:10CC800000210C4812F010FC2B6820F00F0203F07A
:10CC90000F031A430021074812F0F4FB52E7072361
:10CCA000E9E70623E7E70423E5E70223E3E70123B7
:10CCB000E1E700BF6020FF1F6C00FF1F0021B248AA
:10CCC00012F0F2FB2B685B0203F4007320F4007295
:10CCD000DFE730B90821AC4812F0E6FBC0F30020D2
:10CCE00029E70021A84812F0DFFB2B681B0203F4A0
:10CCF000807320F48072CCE730B90C21A24812F086
:10CD0000D3FBC0F3C13016E704219F4812F0CCFBDF
:10CD10002B68DB0303F4C03320F4C0321A43042130
:10CD2000B9E70421984812F0BFFB2B689B0303F47A
:10CD3000804320F48042F1E730B90C21924812F090
:10CD4000B3FBC0F3C120F6E604218F4812F0ACFB20
:10CD50002B68DB0203F4C05320F4C052DEE730B985
:10CD60000C21894812F0A0FBC0F3C310E3E60421B4
:10CD7000854812F099FB2B68DB0103F4F06320F483
:10CD8000F062CBE70421804812F08EFB2B681B0178
:10CD900003F0700320F07002C0E730B90C217A482C
:10CDA00012F082FB00F00F00C5E60421764812F075
:10CDB0007BFB2B6820F00F0203F00F03AEE7052189
:10CDC000714824B912F070FBC0F3C030B3E612F022
:10CDD0006BFB2B68DB039BB220F400421A43052156
:10CDE00059E70521684824B912F05EFBC0F34130D1
:10CDF000A1E612F059FB2B685B0303F4C04320F457
:10CE0000C042EBE70521604824B912F04DFBC0F3A6
:10CE1000032090E612F048FB2B681B0203F47063BA
:10CE200020F47062DAE712F03FFB2B685B0103F03D
:10CE3000600320F06002D1E7534B08B95B7CB5E694
:10CE400012685A747EE606214F4824B912F02CFB72
:10CE5000C0F300406FE612F027FB2B681B0403F4BD
:10CE6000803320F48032CAE612F01EFB2B681B02CE
:10CE700003F4FE4320F4FE42C1E60721424824B9F0
:10CE800012F012FBC0F3813055E612F00DFB2B6857
:10CE90009B039BB220F440421A430721FBE6072183
:10CEA000394824B912F000FBC0F3013043E612F018
:10CEB000FBFA2B681B0303F4405320F44052EBE7CA
:10CEC00012F0F2FA2B689B0203F4806320F4806274
:10CED000E2E707212C4824B912F0E6FAC0F301205A
:10CEE00029E612F0E1FA2B681B0203F4407320F4E8
:10CEF0004072D1E70721244824B912F0D5FAC0F3D3
:10CF0000801018E612F0D0FA2B689B0103F0400362
:10CF100020F04002C0E700287FF436AD02211A4815
:10CF200012F0C2FAC0F3842005E618B9002011F00F
:10CF3000AFF900E61168002011F022F902E612684C
:10CF40005A61FFE50721104824B912F0ADFAC0F389
:10CF5000C010F0E512F0A8FA2B68DB01DBB220F07C
:10CF6000800299E70421084824B912F09DFAC0F321
:10CF70004030E0E512F098FA2B685B0303F40053AD
:10CF800020F40052CAE600BF6020FF1F00287FF493
:10CF9000FBAC104B1B6843B102210F4812F084FA1E
:10CFA000800A00F478702860CCE501210A4812F06C
:10CFB0007BFAC0F38920F6E700287FF4E5AC032173
:10CFC000054812F071FAC0B2B5E512689A60B9E589
:10CFD0001024B1E56C00FF1F6020FF1F0B4611B944
:10CFE00001461846B5E40820704770B5002011F0DE
:10CFF0000FF9064698B90B4D284612F0F4FA0A4B81
:10D00000022001241C60FFF729FC11F081F9304651
:10D010002B6ED5E9151211F013F8204670BD0020D3
:10D02000FCE700BF6020FF1F6C00FF1F38B50D46F6
:10D03000044648B911F0CCF82B68C1182960204685
:10D0400010F094FF204638BD0820FCE707B5019298
:10D0500039B9014601AA0120FFF77BFC03B05DF856
:10D0600004FB0820FAE7022806D3052801D918286E
:10D0700002D100201060704704207047044B9B6E63
:10D080000846114603B11847024B9B6EDB68FAE76E
:10D09000045AFF1F6020FF1F2DE9F041484B494C07
:10D0A000494DDFF87881D4F88820012700211F60DE
:10D0B0002846464B12F01CFAD8F80C60736803F14E
:10D0C0006402EA6503F1840203F592702A6603F5AF
:10D0D000A27203F501732B653368AA65DB68686586
:10D0E00098473368A86DDB6898473368E86DDB685C
:10D0F00098473368286E1B6998473368286DDB684A
:10D100009847D8F8103003F11402AA662A6D9A6184
:10D1100005232B714FF47A73AB6011F0F9F82B6E85
:10D12000D5E91512002010F08BFFD4F88830284A7A
:10D13000C3F80822274AC3F8042200225A701A7042
:10D14000254BC4F89430254BC4F89030244BC4F8D8
:10D150008C30244BC4F89830234BC4F8AC30234BAC
:10D16000C4F8A830224BC4F89C30224BC4F8A0303D
:10D17000214BC4F8BC30214BC4F8B830204BC4F864
:10D18000C830204BC4F8C4301F4BC4F8C0301F4B0C
:10D19000C4F8D43032224FF41673C4E91F321C4B4A
:10D1A000C4F8CC301B4BC4F8E0301B4B84F88470BF
:10D1B000C4F8E4300220BDE8F041FFF74FBB00BFE8
:10D1C0006C00FF1F045AFF1F6020FF1F146A02003B
:10D1D00053C80000EBCF00002DC9000051C900006A
:10D1E0004DC9000049C90000DDCF00004DD000004E
:10D1F00041C800002DD0000049C7000035C700001D
:10D2000055C70000F1C6000017C900005DC8000046
:10D210009DC8000067D00000EDC800003C7A020005
:10D22000012810B514460CD003D3022810D00420D6
:10D2300006E01368094AB3FA83F35B09937200208E
:10D2400010BD1368064AB3FA83F35B091360F6E76F
:10D25000084610F0CDFE2060F1E700BFD820FF1F88
:10D260007400FF1F10B5044618B910F07FFE204669
:10D2700010BD0820FCE7024B986C12F084BA00BF86
:10D28000D820FF1F022804BF0B4B93F8E80030B9E9
:10D290000A4BDB681B685B69094A906D18470128D7
:10D2A00009D1054B93F8E830012B04D1034BDB681F
:10D2B0001B689B69F0E77047045AFF1F3C7A020025
:10D2C000D820FF1F38B50020FFF7DCFF0F4B104CB4
:10D2D000DD68A06D2B685B6998472B68E06C9B68E4
:10D2E00098472B68606D9B6898472B68A06D9B687A
:10D2F00098472B68E06D9B6898472B68206D9B686A
:10D300009847BDE8384011F075B800BF3C7A02007C
:10D31000D820FF1F38B50D46044620B910F078FF1D
:10D320002860204638BD0820FCE710B5044628B91F
:10D33000034B188110F0F4FD204610BD0820FCE7D7
:10D34000D820FF1F0021F0E74942EEE7EDE770B576
:10D35000002010F05DFF0646A0B90B4DA96C2846D1
:10D3600012F0F4F9094B022001241C60FFF78AFF38
:10D3700010F0CEFF3046EB6DD5E9141210F060FED0
:10D38000204670BD0020FCE7D820FF1F7400FF1F5F
:10D3900038B50D46044648B910F01AFF2B68C1187D
:10D3A0002960204610F0E2FD204638BD0820FCE749
:10D3B00038B51F4C636E05469B680021C0F30740DB
:10D3C000984794F86820A36C03EB8203000258602E
:10D3D000636E00219B68C5F30720984794F8683076
:10D3E000A26C02EB8302012153681843636E0002B2
:10D3F00050609B68E8B29847A26C94F8681002EB02
:10D4000081014B6818430011AB0C486010610AD0D1
:10D41000C5F34243072B03D1C5F3011184F868100B
:10D4200043F0080300E0082302EB83035D6038BD8E
:10D43000D820FF1F10B40A4C00F07702A36C42F012
:10D44000080203EB8203C1F313015960A37A23B9E5
:10D4500041EA404010BCFFF7ABBF10BC704700BFB3
:10D46000D820FF1F08461146E4E738B504460F20D0
:10D4700000F013F80323B4FBF3F303EB4303E41AC4
:10D480000546E4B220F0300040EA0410FFF790FFB8
:10D490002846BDE83840FFF78BBF38B5074DAA7A5C
:10D4A00004461AB9030701D4FFF7DFFFAB6C04F0A1
:10D4B0007F0403EB8404606838BD00BFD820FF1FE1
:10D4C000A72970B50446154600F0F58164D81D29DA
:10D4D00000F0F48021D8042900F0F7800CD801294D
:10D4E00000F0D980C0F0CB80022900F0DD80032954
:10D4F00000F0E4800424C6E0062900F0FB80C0F0C0
:10D50000F080072900F010810829F3D10028F1D11B
:10D5100010F06EFDC0F30010B4E0A12900F0778197
:10D520001AD8332900F01B8108D83229E2D100280B
:10D5300040F01081002010F0B9FEA3E08C2900F02B
:10D540001781A029D6D10820002C40F05781FFF781
:10D55000A4FFC0F3402095E0A42900F083810DD8FA
:10D56000A22900F06481A329C4D10C20002C40F032
:10D570007081FFF792FFC0F3803083E0A52900F0AF
:10D580008181A629B6D10C20002C40F08B81FFF7B9
:10D5900084FFC0F3021075E0B22900F02F823ED85C
:10D5A000AC2900F0D78112D8A92900F0A781C0F0DA
:10D5B0009181AA2900F0B381AB299BD1002840F0CA
:10D5C000BF810520FFF769FFC0F341105AE0AF2982
:10D5D00000F0E78114D8AD2900F0C881AE2989D1C7
:10D5E000002840F0D4810620FFF757FF000A00F022
:10D5F0007F0310F0400018BF6FF07F00184341E038
:10D60000B02900F0E081B1297FF474AF002840F028
:10D61000EB810720FFF741FFC0F3802032E0B729FC
:10D6200000F0248210D8B42900F00A82C0F0F781FB
:10D63000B52900F00E82B6297FF45CAFAE4B00280E
:10D6400040F011821B6958E0CE2900F03A820AD8D6
:10D65000B82900F01B82B9297FF44CAF002840F0B4
:10D660002682072084E1D02900F03F82D6297FF46A
:10D6700041AFA14B002840F040825B683DE020B9FB
:10D6800010F0B6FD2860204670BD1168002010F033
:10D690006DFC0024F7E710B910F09AFDF2E711686D
:10D6A000002010F043FDF4E718B9002010F0C0FD91
:10D6B000E8E71168002010F033FCEAE7002C7FF463
:10D6C00019AF204610F0A4FDDCE710B910F0D0FD32
:10D6D000D8E711680029B8BF4942002010F042FD88
:10D6E000D7E710B910F0B4FDCCE71168002010F0B6
:10D6F000B2FECEE7804E10B9F37A2B60C3E7136811
:10D70000F3720020FFF7C9FE10F08004C1D10E2093
:10D71000FFF7C3FEF37A20F01F0103F01F03194344
:10D720000E20FFF787FEAEE7734E08B93378E4E7C3
:10D73000136833700020FFF7B0FE0306A9D50E2052
:10D74000FFF7ABFE337820F01F0103F01F031943EE
:10D750000E2046E01178002010F020FD99E710B966
:10D7600010F0B2FD8EE71168002010F027FD90E761
:10D7700038B90820FFF791FE00F00F00C0F1080053
:10D7800080E71368102B33D00DDC022B2CD004DC87
:10D79000012B16D04FF0FF3314E0042B26D0082BBA
:10D7A000F8D105230EE0402B24D003DC202BF1D14F
:10D7B000032307E0802B1FD0B3F5807FEAD100233D
:10D7C00000E008232B602B68013300F099810820CA
:10D7D000FFF763FE2B6820F00F0103F00F031943DE
:10D7E0000820FFF727FE54E70723EBE70623E9E7C6
:10D7F0000423E7E70223E5E70123E3E7FFF74DFE14
:10D800002B685B0203F4007320F40071E7E7082043
:10D8100024B9FFF742FEC0F3002033E7FFF73DFED7
:10D820002B681B0203F4807320F48071D7E70C206F
:10D8300024B9FFF732FEC0F3C13023E7FFF72DFE16
:10D840002B68DB0303F4C03320F4C03119430C20F0
:10D85000C7E7FFF722FE2B689B0303F4804320F405
:10D860008041F3E70C2024B9FFF717FEC0F3C12075
:10D8700008E7FFF712FE2B68DB0203F4C05320F425
:10D88000C051E3E70C2024B9FFF707FEC0F3C31033
:10D89000F8E6FFF702FE2B68DB0103F4F06320F4E7
:10D8A000F061D3E7FFF7F9FD2B681B0103F070036C
:10D8B00020F07001CAE70C2024B9FFF7EEFD00F05C
:10D8C0000F00DFE6FFF7E9FD2B6820F00F0103F002
:10D8D0000F03BBE728B90520FFF7DFFDC0F3C03019
:10D8E000D0E60D20FFF7D9FD2B68DB039BB220F4B7
:10D8F000004119430D2074E7D820FF1F28B90520E7
:10D90000FFF7CBFDC0F34130BCE60D20FFF7C5FDAE
:10D910002B685B0303F4C04320F4C041E9E728B956
:10D920000520FFF7BAFDC0F30320ABE60D20FFF79B
:10D93000B4FD2B681B0203F4706320F47061D8E718
:10D940000D20FFF7AAFD2B685B0103F0600320F0B8
:10D950006001CEE708B90520AFE70D20FFF79DFD78
:10D960002B6820F00F0103F00F03C2E728B906204F
:10D97000FFF793FDC0F3004084E60E20FFF78DFD16
:10D980002B681B0403F4803320F48031DFE60E2083
:10D99000FFF783FD2B681B0203F4FE4320F4FE41D6
:10D9A000D5E628B90720FFF778FDC0F3813069E696
:10D9B0000F20FFF772FD2B689B039BB220F44041C0
:10D9C00019430F200DE728B90720FFF766FDC0F3C4
:10D9D000013057E60F20FFF760FD2B681B0303F4AF
:10D9E000405320F44051EBE70F20FFF756FD2B6822
:10D9F0009B0203F4806320F48061E1E728B90720EB
:10DA0000FFF74BFDC0F301203CE60F20FFF745FD7B
:10DA10002B681B0203F4407320F44071D0E728B94F
:10DA20000720FFF73AFDC0F380102BE60F20FFF729
:10DA300034FD2B689B0103F0400320F04001BFE759
:10DA400000287FF457AD0220FFF727FDC0F38420A4
:10DA500018E618B9002010F01BFC13E6116800202E
:10DA600010F08EFB15E612681A6112E628B907203D
:10DA7000FFF713FDC0F3C01004E60F20FFF70DFD04
:10DA80002B68DB01DBB220F0800199E728B9042084
:10DA9000FFF703FDC0F34030F4E50C20FFF7FDFC79
:10DAA0002B685B0303F4005320F40051CEE60F20F3
:10DAB000FFF7F3FC2B681B0403F4803320F4803160
:10DAC0007EE700287FF416AD0E4B1B683BB10220A9
:10DAD000FFF7E3FC800A00F478702860D9E50120A4
:10DAE000FFF7DBFCC0F38920F7E700287FF402ADE5
:10DAF0000320FFF7D2FCC0B2C4E512685A60C8E543
:10DB00001024C0E57400FF1F0B4611B901461846EA
:10DB1000D6E40820704707B5019239B9014601AA39
:10DB20000120FFF7CDFC03B05DF804FB0820FAE705
:10DB300010B508461446FFF7B0FC206010BDF8B5DC
:10DB400006460020FFF7A9FC324C94F86930C0F378
:10DB5000C015AB4215D00E20002D4BD0FFF79DFC19
:10DB600000F01F00E0720E20FFF797FC237803F00F
:10DB70001F0320F01F0119430E20FFF75BFC84F800
:10DB80006950254A217A936F00293DD043F0010363
:10DB9000617A00293BD043F002030020936710F024
:10DBA00037FB236994F86A200028B8BF40429842A6
:10DBB00034BF00270127BA4211D098424FF00D0020
:10DBC0002CBF657B257BFFF768FC05F00F0520F077
:10DBD0000F0129430D20FFF72DFC84F86A70A36C18
:10DBE0000C4A3146002011F05CFD0020BDE8F840F1
:10DBF00010F07EBAFFF751FC00F01F0020700E20DD
:10DC0000FFF74BFCE37AB2E723F00103C0E723F010
:10DC10000203C2E7D820FF1F045AFF1F0A4810B4AE
:10DC2000836C01F0770444F0080403EB8403C2F32F
:10DC300013025A60837A23B942EA414010BCFFF7CD
:10DC4000B7BB10BC704700BFD820FF1F38B5084DC8
:10DC5000AA7A0C4622B90B0702D40846FFF705FC46
:10DC6000A96C04F07F0401EB8404606838BD00BF38
:10DC7000D820FF1F38B51F4C636E0D469B680021EE
:10DC8000C5F30740984794F86B20A36C03EB82031D
:10DC900000025860636E00219B68C5F30720984717
:10DCA00094F86B30A26C02EB830201215368184395
:10DCB000636E000250609B68E8B29847A26C94F8CB
:10DCC0006B1002EB81014B6818430011AB0C4860EC
:10DCD00010610AD0C5F34243072B03D1C5F30111EC
:10DCE00084F86B1043F0080300E0082302EB830381
:10DCF0005D6038BDD820FF1FF8B5424C424B434F02
:10DD0000012620461E6011F0ABFCFD686B6803F134
:10DD10006402A26503F1840203F59270E26503F5E3
:10DD2000A27203F50173E3642B686265DB6820650A
:10DD300098472B68606DDB6898472B68A06DDB689F
:10DD400098472B68E06D1B6998472B68E06CDB688F
:10DD500098473B6903F114026266E26C9A610523FD
:10DD600023704FF47A73636010F0D2FAD4E914127E
:10DD7000E36D002010F064F9254B2649D3F8882084
:10DD8000A264C2F808122449C2F80412002151709A
:10DD90001170224AC3F89420214AC3F89020214AE6
:10DDA000C3F88C20204AC3F89820204AC3F8AC203E
:10DDB0001F4AC3F8A8201F4AC3F89C201E4AC3F874
:10DDC000A0201E4AC3F8BC201D4AC3F8B8201D4A33
:10DDD000C3F8C8201C4AC3F8C4201C4AC3F8C0209A
:10DDE0001B4AC3F8D42032214FF41672C3E91F2115
:10DDF00083F88460174AC3F8CC200220BDE8F840BD
:10DE0000FFF740BAD820FF1F7400FF1F3C7A0200C2
:10DE1000045AFF1F77D200004FD300002BD300001D
:10DE20004DD3000049D3000045D3000009DB0000BA
:10DE300017DB000065D2000091D3000065D400001C
:10DE400031DB00003FDB000021D2000015D30000D1
:10DE500085D20000C5D20000014B00225A607047F5
:10DE6000045AFF1F70B5184E184CF56860682B688F
:10DE70009B6998472B68A0699B6898472B686069E5
:10DE80009B6898472B6820699B6898472B68E068D7
:10DE90009B6898472B68A0689B6898472B68206A06
:10DEA0009B6898472B68E0699B6898472B682068B7
:10DEB0009B6898472B6860689B6898473369BDE802
:10DEC00070405B6A184700BF3C7A02005021FF1F78
:10DED000022870B5144649D004D890B1012836D034
:10DEE000042432E003284FD0FF28F9D12B4CD4F87A
:10DEF0008830D3F8043298476369D3F804329847DE
:10DF000003E0126832F0030301D000241DE0244B2B
:10DF1000244DDE6868693368D2070AD51B699847C3
:10DF200024683268A86914F0020408D0136998477D
:10DF3000EBE7DB689847336868699B69EFE7D3686C
:10DF400098473368A8699B699847204670BD144B71
:10DF5000144DDE681468286933680CB11B69E6E764
:10DF6000DB689847336828699B69EDE70C4B0D4DDA
:10DF7000DE6814683368A868002CEFD1DB68984726
:10DF80003368A8689B69DFE70121074811F02EFD7F
:10DF900020600028B9D12024D7E700BF045AFF1F12
:10DFA0003C7A02005021FF1F7421FF1F01460148E7
:10DFB00011F0D2BD7421FF1F10B50348144611F0B3
:10DFC00044FC206010BD00BF7421FF1F014811F008
:10DFD0002EBC00BF7421FF1F08B50448D0F8B8223A
:10DFE000243011F0F3FC002008BD00BF5021FF1FBA
:10DFF00008B50448D0F8B822243011F0CBFC00203A
:10E0000008BD00BF5021FF1F08B50021024811F0D4
:10E01000A3FC002008BD00BF7421FF1F08B54942C2
:10E02000024811F099FC002008BD00BF7421FF1FB9
:10E0300008B5024811F090FC002008BD7421FF1FB4
:10E0400038B50A4B0A4CDD6860682B689B699847B5
:10E0500001200CF0F3FE2B6860685B69984704F1BF
:10E06000240011F04EFC012038BD00BF3C7A0200B4
:10E070005021FF1F38B50A4B0A4CDD6860682B68D9
:10E080009B69984701200CF0D9FE2B6860685B699A
:10E09000984704F1240011F01FFC012038BD00BF97
:10E0A0003C7A02005021FF1F6E2970B504461546C8
:10E0B00000F0BB8170D8122900F06C8138D8052996
:10E0C00000F0298118D8022900F0018107D8002921
:10E0D00000F0E880012900F0F4800424E8E003293E
:10E0E00000F002810429F8D1B64E002840F00181E9
:10E0F000D6F8B8322B60DBE00F2900F030810DD864
:10E10000082900F01B810E29E7D1002840F020816A
:10E110002021AD4811F099FB4000C8E0102900F023
:10E1200024811129D9D1002840F02B812921F4E044
:10E13000182900F05C8117D8152900F0408109D812
:10E14000132900F02D811429C7D1002840F0348113
:10E150002621A9E0162900F041811729BDD1002808
:10E1600040F042812E219FE01B2900F04F8109D809
:10E17000192900F042811A29AFD1002840F04381CB
:10E18000332191E06C2900F047816D29A5D1002849
:10E1900040F04881612187E07E2900F0B0813CD8C1
:10E1A000742900F0798119D8712963D009D86F29B1
:10E1B00000F04B81702990D1002840F05681592100
:10E1C00072E0722900F05481732986D1002840F052
:10E1D00060817C4B5B6AD3F86C318BE7772900F068
:10E1E0007F810FD8752900F0608176297FF475AFA3
:10E1F0007448436AD3F87021002C40F06781C2F361
:10E2000007422BE07C2900F071817D297FF465AF06
:10E21000002840F071815F2146E0892900F0B28139
:10E220001ED8852900F093810AD8812900F07881D1
:10E2300084297FF452AF00287FF44FAF652133E08B
:10E24000862900F0918188297FF447AF5D48436AB1
:10E25000D3F89021002C40F08D81D2B22A6027E0C3
:10E26000D12900F0AE8112D88A2900F09A81C829FC
:10E270007FF433AF05215448002C00F0E98011F001
:10E28000E4FA2A7820F0FF000243052114E0D429A3
:10E2900000F09D81D6297FF420AF002840F09F81B7
:10E2A000152101E030B93721474811F0CEFA286036
:10E2B000204670BD12683721434811F0B8FA002497
:10E2C000F6E708B92121EFE712682121F4E728B920
:10E2D00024213D4811F0B9FA0012E8E7106811F066
:10E2E00029FB24210246E7E700287FF4F6AE22212D
:10E2F000DAE71368C6F8B832202106F1240011F0DD
:10E30000A4FA4207DBD5D6F8B80211F013FB24219A
:10E3100002467018D1E728B928212B4811F095FA48
:10E320008010C4E71268940DA405002C40F05C81B5
:10E3300092002821244811F07AFAB9E700287FF4E6
:10E34000CCAE0F21204811F080FA00F00100AEE7BA
:10E350001368002B0CBF012202222021ACE708B970
:10E360002521A1E712682521A6E708B92A21D4E7CB
:10E370001268940DA405002C40F0368192002A21E9
:10E38000D8E71268940DA405002C40F02D8192006E
:10E390002921CFE708B9272186E7126827218BE7D3
:10E3A00008B92B21B9E71268940DA405002C40F0A0
:10E3B0001B8192002B21BDE7126826217CE728B93A
:10E3C0002C2171E75021FF1F7421FF1F1268940D4B
:10E3D000A405002C40F008812C21ABE708B92D21C1
:10E3E00062E712682D2167E712682E2164E708B9F9
:10E3F0002F2159E712682F215EE708B9302153E732
:10E400001268302158E71268332155E708B93421E2
:10E410004AE7126834214FE708B9602144E71268DF
:10E42000602149E71268612146E71C216F481CB949
:10E4300011F00BFA00143AE711F007FA2A68C0F35A
:10E44000080040EA02421C2136E71C2167481CB93B
:10E4500011F0FBF9C0B22AE711F0F7F92B6800F4CC
:10E460007F02C3F308031A43EDE71268592123E73B
:10E4700005215E4824B911F0E8F9C0F3072016E73A
:10E4800011F0E3F92B681B0220F47F429BB21A4380
:10E49000FBE612685A210FE720B9554B5B6AD3F8A7
:10E4A000703127E612685B2106E7514B5B6AD3F8AF
:10E4B000703110B9C3F30E031CE6126823F4FF4356
:10E4C00023F07F03C2F30E021A43ECE72B681B0410
:10E4D00022F47F0203F47F031A435B212430ECE62D
:10E4E00008B95E21E0E612685E21E5E608B95C2124
:10E4F000DAE612685C21DFE612685F21DCE60521BE
:10E500003A4824B911F0A1F9C0F30740CFE611F061
:10E510009CF92B681B0420F47F0203F47F03B6E709
:10E5200000283FF4CCAE14684CB101212F4811F003
:10E530005DFA286000287FF4C2AE2024B8E60721E7
:10E540002A4811F082F9072120F48002F2E600281F
:10E550007FF4B5AE0721254811F077F9C0F381505B
:10E56000431E58425841A2E608B952219CE612685F
:10E570005221A1E62B6822F0FF0203F00F031A4399
:10E580006321ABE71A48436AD3F8902114B9C2F368
:10E59000032263E62B681B0222F4706203F47063AB
:10E5A000EDE7134B5B6AD3F8902100283FF427AEC8
:10E5B0002B681B0422F47F0203F47F031A436321B8
:10E5C0007AE608B950216FE61268502174E618B94E
:10E5D000074B5B6A9B698DE5126853216CE61368F3
:10E5E000044A15215A4367E6102461E67421FF1F8F
:10E5F0005021FF1F007102000B4611B90146184659
:10E6000052E50820704708B5024811F0A5F900202E
:10E6100008BD00BF7421FF1F07B5019239B901463B
:10E6200001AA0120FFF740FD03B05DF804FB0820BC
:10E63000FAE7034BD3F8BC320846DB6811461847AB
:10E640005021FF1FF8B5494C494D4A4F4A4B6A6962
:10E65000002104F1240011F021F9FE68736803F130
:10E66000E402226203F58272E26103F55172A26153
:10E6700003F55972626103F56172226103F56972F3
:10E6800003F57970E26003F5717203F204432360CD
:10E690003368A260DB68606098473368A069DB6814
:10E6A000984733686069DB68984733682069DB689E
:10E6B00098473368E068DB6898473368A068DB6890
:10E6C0009847336860685B6998473368A0695B69FD
:10E6D0009847336860695B699847336820695B696C
:10E6E00098473368E0685B6998473368A0685B695E
:10E6F00098473368206A1B6998473368E0691B694B
:10E700009847336820681B69984773683A69C4F86A
:10E71000BC2203F5317353606B69002159701749AE
:10E72000C3F80412012216491A70C3F80812154BD7
:10E730002B62154BEB61154BAB61154B6B62154BA7
:10E74000AB63154B6B63154BAB62154BEB62154B13
:10E75000AB64154B6B64154B6B65154B2B65154BFB
:10E76000EB65154B2A74AB65F8BD00BF5021FF1F48
:10E77000045AFF1F3C7A0200346A020075E0000070
:10E7800041E0000007E6000031E000001DE000006D
:10E7900009E00000F9E5000019E60000F1DF0000E3
:10E7A000D9DF0000CDDF0000B9DF0000ADDF0000E1
:10E7B000D1DE000059DE000065DE0000014B0022C2
:10E7C0005A607047045AFF1F022870B5144648D09B
:10E7D00004D8A0B1012835D004200FE003280CD0C4
:10E7E000FF28F9D1264CD4F88830D3F80432984762
:10E7F0006369D3F80432984716E0202070BD126890
:10E8000032F00303FAD11F4B1F4DDE68686933688D
:10E81000D2070BD51B69984724683268A86914F0A1
:10E82000020409D0136998470020E7E7DB6898479E
:10E83000336868699B69EEE7D36898473368A869CD
:10E840009B69F0E70F4B104DDE6814682869336848
:10E850000CB11B69E7E7DB689847336828699B6957
:10E86000E1E7084B084DDE6814683368A868002C9F
:10E87000EFD1DB6898473368A8689B69D3E700BF8E
:10E88000045AFF1F3C7A02002024FF1F70B5184E67
:10E89000184CF56860682B689B6998472B68A069DD
:10E8A0009B6898472B6860699B6898472B6820692C
:10E8B0009B6898472B68E0689B6898472B68A0681E
:10E8C0009B6898472B68206A9B6898472B68E0698B
:10E8D0009B6898472B6820689B6898472B686068FE
:10E8E0009B6898473369BDE870405B6A184700BF72
:10E8F0003C7A02002024FF1F0A460146014811F01D
:10E90000DFB900BF4424FF1F0146014811F08EBA51
:10E910004424FF1F10B50348144611F0A8F92060E5
:10E9200010BD00BF4424FF1F6C2938B50C461546A6
:10E930000BD06D2902D10A4BC3F8B8222A462146D2
:10E940000848BDE8384011F084B9054BD3F8B81237
:10E95000054B01F07F01D3F8BC309847EEE700BFCC
:10E960002024FF1F4424FF1F045AFF1F08B504483A
:10E97000D0F8BC22243011F0E7FA002008BD00BF17
:10E980002024FF1F08B50448D0F8BC22243011F021
:10E99000BFFA002008BD00BF2024FF1F08B50021DA
:10E9A000024811F097FA002008BD00BF4424FF1F61
:10E9B00008B54942024811F08DFA002008BD00BF99
:10E9C0004424FF1F08B5024811F084FA002008BD56
:10E9D0004424FF1F38B50A4B0A4CDD6860682B6879
:10E9E0009B69984701200CF029FA2B6860685B69E5
:10E9F000984704F1240011F000FA012038BD00BF4F
:10EA00003C7A02002024FF1F38B50A4B0A4CDD680F
:10EA100060682B689B69984701200CF00FFA2B68FF
:10EA200060685B69984704F1240011F0D1F9012076
:10EA300038BD00BF3C7A02002024FF1F70B5114C86
:10EA400094F87430012B0D4619D0032B0BBF002214
:10EA500028220C230F2343F0884343F0401343EA5A
:10EA60004232042111F0F5F8D4F88830012D0CBFA2
:10EA7000D3F80432D3F80832BDE8704018470022BA
:10EA80000B23E8E7045AFF1F2DE9F84F424CD4F856
:10EA9000C462D4F8C0524FEA062949EA1569C6B2E1
:10EAA0004FEA052894F8C802D4F8D452002748EA5F
:10EAB0000602D4F8D06249EA070301302F0E2D0276
:10EAC00045EA166504F5307C3602C0B204F5347EA2
:10EAD000C4F8D062C4F8D452CCE9002384F8C80248
:10EAE00066467546002954D0042805D91A466D217A
:10EAF00004F1240011F0ADF8D4F8C02227486C21AD
:10EB000011F0A7F801200CF099F9D4F8C02223489D
:10EB10006C2111F09EF894F8C8324FF0000B042BD2
:10EB2000C5E900BB0CD96F211C4811F0A0F8D5E94C
:10EB30000023814643EA090142EA0B00C5E90001CE
:10EB40006E21164811F093F8D5E9002343EAE079E5
:10EB500094F8C832C3F10803DB0042EA0008A3F1CD
:10EB6000200EC3F1200C09FA03F208FA0EFE42EA65
:10EB70000E0228FA0CFC42EA0C02404698406A60F9
:10EB800000230022C6E900230023C4F8D00284F841
:10EB9000C8323846BDE8F88F2024FF1F4424FF1FE9
:10EBA00008B5024811F096F9002008BD4424FF1F63
:10EBB00038B515460C4600297BD1112869D01FD8DD
:10EBC00004284ED008D8012840D03AD302283FD09C
:10EBD000032844D0042448E00E284ED00AD8052843
:10EBE00045D00828F6D10F21334811F040F800F045
:10EBF000010032E00F284AD01028EBD12A2137E05B
:10EC000017284ED00ED8142847D005D8122842D045
:10EC10001328DFD12B212BE0152840D01628D9D17D
:10EC20002D210FE01A2840D005D818283BD01928EC
:10EC3000D0D1302106E01B2839D0D628CAD11521E1
:10EC400000E037211C4811F012F806E02121F9E715
:10EC50002421194811F00BF80012286005E0222148
:10EC6000F0E7164BD3F8BC321360204638BD28219C
:10EC7000114810F0FCFF8010EFE720210E4810F043
:10EC8000F6FF00F00300831E58425841E5E72521B6
:10EC9000D8E72921ECE72721D4E72621D2E72C2148
:10ECA000D0E72E21CEE72F21CCE73321CAE734214C
:10ECB000C8E70824D9E700BF4424FF1F2024FF1F12
:10ECC00038B514460D46002940F08B80122871D0CB
:10ECD00022D8052860D008D8012840D039D302288E
:10ECE0003FD0042843D0042537E00F285AD007D856
:10ECF0000E28F8D1002A14BF02220122202129E087
:10ED0000102851D01128EED1930D9B05002B6AD10C
:10ED10009200292135483BE017285AD008D81428FA
:10ED200050D049D315284FD01628DCD12D2111E021
:10ED30001A2852D005D818284DD01928D3D13021FF
:10ED400008E01B284BD0D628CDD1294A1521624393
:10ED500000E03721254810F07CFF284638BD2121EE
:10ED6000F8E782EAE272A2EBE4722421F2E7214D95
:10ED7000202105F12400C5F8BC2210F078FF4307DC
:10ED800008D5D5F8BC0211F093F824210246681882
:10ED900010F05FFF0025E0E7950DAD051DBB92006B
:10EDA0002821D7E72521D5E7950DAD05DDB99200DE
:10EDB0002A21CFE72721CDE7950DAD059DB992001A
:10EDC0002B21C7E72621C5E7950DAD055DB92C219F
:10EDD000C0E72E21BEE72F21BCE73321BAE734215B
:10EDE000B8E70825B9E71025B7E700BF4424FF1F9F
:10EDF000007102002024FF1F034BD3F8D8320846CD
:10EE0000DB681146184700BF2024FF1FF8B54D4CA2
:10EE10004D4D4E4B6A694E4F04F124063046002199
:10EE200010F0B9FF4B49304610F0FCFFFE687368E4
:10EE300003F1E402226203F58272E26103F551728A
:10EE4000A26103F55972626103F56172226103F5F3
:10EE5000697203F57970E26003F5717203F204439D
:10EE600023603368A260DB68606098473368A069FC
:10EE7000DB68984733686069DB68984733682069C6
:10EE8000DB6898473368E068DB6898473368A068B8
:10EE9000DB689847336860685B6998473368A069A6
:10EEA0005B699847336860695B6998473368206994
:10EEB0005B6998473368E0685B6998473368A06886
:10EEC0005B6998473368206A1B6998473368E06933
:10EED0001B699847336820681B69984773683A69CB
:10EEE000C4F8D82203F5317353606B69002159705F
:10EEF0001949C3F80412012218491A70C3F80812FC
:10EF0000174B6B66174B2B62174BEB61174BAB61C3
:10EF1000174B6B62174BAB63174B6B63174BAB62B3
:10EF2000174BEB62174BAB64174B6B64174B6B655E
:10EF3000174B2B65174BEB65174BAB65174B2A74BB
:10EF4000AB66F8BD2024FF1F045AFF1F346C02007B
:10EF50003C7A02003DEA000009EA0000D5E9000021
:10EF600089EA0000A1EB0000C5E90000B1E900005A
:10EF70009DE90000B1EB0000C1EC000085E9000054
:10EF80006DE9000029E9000015E9000009E9000029
:10EF9000C9E70000BDE700008DE80000F9E80000C7
:10EFA000014B00225A607047045AFF1F70B5184E7B
:10EFB000184CF56860682B689B6998472B68A069B6
:10EFC0009B6898472B6860699B6898472B68206905
:10EFD0009B6898472B68E0689B6898472B68A068F7
:10EFE0009B6898472B68206A9B6898472B68E06964
:10EFF0009B6898472B6820689B6898472B686068D7
:10F000009B6898473369BDE870405B6A184700BF4A
:10F010003C7A02000827FF1F0A460146014811F00A
:10F0200011B800BF2C27FF1F022870B5144649D025
:10F0300004D890B1012836D0042432E003284FD000
:10F04000FF28F9D12B4CD4F88830D3F804329847F4
:10F050006369D3F80432984703E0126832F003037F
:10F0600001D000241DE0244B244DDE68686933681C
:10F07000D2070AD51B69984724683268A86914F03A
:10F08000020408D013699847EBE7DB6898473368B8
:10F0900068699B69EFE7D36898473368A8699B69FB
:10F0A0009847204670BD144B144DDE6814682869DB
:10F0B00033680CB11B69E6E7DB6898473368286959
:10F0C0009B69EDE70C4B0D4DDE6814683368A8684A
:10F0D000002CEFD1DB6898473368A8689B69DFE7AD
:10F0E0000121074811F0C2F820600028B9D120247E
:10F0F000D7E700BF045AFF1F3C7A02000827FF1F12
:10F100002C27FF1F0146014811F066B92C27FF1F6D
:10F1100010B50348144610F06CFF206010BD00BF0E
:10F120002C27FF1F6C2938B50C4615460BD06D29CE
:10F1300002D10A4BC3F8B8222A4621460848BDE846
:10F14000384010F048BF054BD3F8B812054B01F01A
:10F150007F01D3F8BC309847EEE700BF0827FF1FB8
:10F160002C27FF1F045AFF1F08B50448D0F8BC2203
:10F17000243011F06BF8002008BD00BF0827FF1FE6
:10F1800008B50448D0F8BC22243011F043F8002020
:10F1900008BD00BF0827FF1F08B50021024811F075
:10F1A0001BF8002008BD00BF2C27FF1F08B54942EF
:10F1B000024811F011F8002008BD00BF2C27FF1FE6
:10F1C00008B5024811F008F8002008BD2C27FF1FE1
:10F1D00038B50A4B0A4CDD6860682B689B69984714
:10F1E00001200BF02BFE2B6860685B69984704F1E7
:10F1F000240010F0C6FF012038BD00BF3C7A020099
:10F200000827FF1F38B50A4B0A4CDD6860682B6879
:10F210009B69984701200BF011FE2B6860685B69C1
:10F22000984704F1240010F097FF012038BD00BF7B
:10F230003C7A02000827FF1F70B5114C94F8743017
:10F24000012B0D4619D0032B0BBF002228220C23C3
:10F250000F2343F0884343F0401343EA4232042132
:10F2600010F0B9FED4F88830012D0CBFD3F8043269
:10F27000D3F80832BDE87040184700220B23E8E7B6
:10F28000045AFF1F6F2970B50446154600F08182AD
:10F2900000F28980122900F0D1813ED8052900F0C2
:10F2A000718118D8022900F03B8107D8002900F0AD
:10F2B0001A81012900F0268104241AE1032900F0B3
:10F2C00041810429F8D1B94E002840F04481D6F894
:10F2D000BC3213600DE10F2900F082810ED808299D
:10F2E00000F068810E29E7D1002840F06E812021CE
:10F2F000AF4810F07EFE40002860FAE0102900F0D0
:10F300007D811129D8D1002840F08C812921A8487D
:10F3100010F06FFE80102860EBE0182900F0DE810D
:10F320001FD8152900F0B3810DD8132900F094815E
:10F330001429C1D1002840F0A38126219C4810F057
:10F3400058FE2860D5E0162900F0B3811729B3D103
:10F35000002840F0BC812E21954810F04AFE28601C
:10F36000C7E01B2900F0DD810DD8192900F0C48108
:10F370001A29A1D1002840F0CD8133218C4810F00A
:10F3800038FE2860B5E06D2900F0E08100F2EC81E4
:10F390006C2991D1002840F0D2816021844810F07E
:10F3A00028FE2860A5E07D2900F0AB8248D87529A9
:10F3B00000F0508222D8722900F01B820FD87029E9
:10F3C00000F0FD8171297FF477AF06217848002C89
:10F3D00040F0038210F00DFEC0B2286089E073296E
:10F3E00000F01E8274297FF467AF002840F0268267
:10F3F0006E4B5B6AD3F8703113607AE0782900F0C5
:10F400005D820ED8762900F03C8277297FF454AFD4
:10F41000002840F04C825E21654810F0EAFD28602B
:10F4200067E0792900F058827C297FF445AF0028F5
:10F4300040F060825C215E4810F0DBFD286058E0FF
:10F44000882900F0AD8228D8842900F08B8215D855
:10F450007E2900F0648281297FF42EAF002800F01D
:10F4600084801468002C00F072820121504810F052
:10F47000FDFE2860002878D120243AE0852900F09C
:10F480007A8286297FF418AF002840F082825221C8
:10F49000474810F0AEFD28602BE0C82995D010D861
:10F4A000892900F091828A297FF406AF3F48436A98
:10F4B000D3F89021002C40F09D82C2F307422A60CD
:10F4C00017E0D42900F0AA82D62900F0B482D1290D
:10F4D0007FF4F2AE002840F09A825021344810F0B8
:10F4E00088FD286005E030B93721314810F081FDF2
:10F4F0002860204670BD12682D48372110F06BFD42
:10F500000024F6E728B92121294810F072FD28606F
:10F51000EFE712682648212110F05DFD0024E8E79E
:10F5200030B92421224810F064FD00122860E0E781
:10F53000106810F03FFE242102461D4810F04BFDDC
:10F540000024D6E7002840F086822221184810F0D7
:10F5500050FD2860CDE71368C6F8BC32202106F1C3
:10F56000240010F046FD420701D40024C1E7D6F87C
:10F57000BC0210F01FFE24210246701810F02BFD73
:10F580000024B6E730B92821094810F032FD801078
:10F590002860AEE71268940DA405002C40F05D824F
:10F5A00092002821024810F016FDA2E70827FF1F4D
:10F5B0002C27FF1F002840F052820F21A34810F093
:10F5C00018FD00F00100286093E713689F48002BA6
:10F5D0000CBF01220222202110F0FDFC002488E74C
:10F5E00028B92521994810F004FD286081E71268A8
:10F5F0009648252110F0EFFC00247AE730B92A2143
:10F60000924810F0F6FC8010286072E71268940DA2
:10F61000A405002C40F0258292002A218B4810F08E
:10F62000DAFC66E71268940DA405002C40F01B82FA
:10F6300092002921854810F0CEFC5AE728B92721ED
:10F64000824810F0D6FC286053E712687F482721D3
:10F6500010F0C1FC00244CE730B92B217B4810F09E
:10F66000C8FC8010286044E71268940DA405002CA3
:10F6700040F0FB8192002B21744810F0ACFC38E77D
:10F6800012687248262110F0A6FC002431E728B940
:10F690002C216E4810F0ADFC28602AE71268940D0A
:10F6A000A405002C40F0E3812C21684810F093FC65
:10F6B0001FE728B92D21654810F09BFC286018E74A
:10F6C000126862482D2110F086FC002411E71268B0
:10F6D0005E482E2110F07FFC00240AE728B92F2174
:10F6E0005A4810F086FC286003E7126857482F211B
:10F6F00010F071FC0024FCE628B93021534810F0CA
:10F7000078FC2860F5E612685048302110F063FC60
:10F710000024EEE612684D48332110F05CFC002412
:10F72000E7E628B93421494810F063FC2860E0E698
:10F7300012684648342110F04EFC0024D9E61268C5
:10F740004248602110F047FC0024D2E628B961212C
:10F750003E4810F04EFC2860CBE612683B48612121
:10F7600010F039FC0024C4E61C21384824B910F0FC
:10F7700040FC00142860BCE610F03BFC2A68C0F393
:10F78000080040EA02421C21304810F024FC00240A
:10F79000AFE61C212D4824B910F02BFCC0B2286024
:10F7A000A7E610F026FC2B6800F47F02C3F30803E1
:10F7B0001A431C21254810F00EFC002499E628B9B4
:10F7C0005921224810F015FC286092E612681F4863
:10F7D000592110F000FC00248BE610F00AFC2A7876
:10F7E00020F0FF0002430621184810F0F4FB00242B
:10F7F0007FE6062115482CB910F0FBFBC0F307206B
:10F80000286076E610F0F5FB2B681B0220F47F429F
:10F810009BB21A4306210D4810F0DDFB002468E678
:10F8200028B90B4B5B6AD3F86C31136061E6126840
:10F8300006485A2110F0CFFB00245AE6126803480C
:10F840005B2110F0C8FB002453E600BF2C27FF1FEC
:10F850000827FF1F8848436AD3F870311CB9C3F3E7
:10F860000E03136045E6126823F4FF4323F07F0381
:10F87000C2F30E021A435B21243010F0ACFB0024CB
:10F8800037E67D4B5B6AD3F8702118B9C2F30742A3
:10F890002A602EE62B6879481B0403F47F0322F4C8
:10F8A0007F021A435B2110F096FB002421E61268C8
:10F8B00072485E2110F08FFB00241AE628B9182147
:10F8C0006E4810F096FB286013E612686B4818210A
:10F8D00010F081FB00240CE628B91921674810F0CC
:10F8E00088FB286005E612686448192110F073FB54
:10F8F0000024FEE5126861485C2110F06CFB0024D6
:10F90000F7E528B95F215D4810F073FB2860F0E54A
:10F9100012685A485F2110F05EFB0024E9E50621D9
:10F9200056482CB910F065FBC0F307402860E0E5AD
:10F9300010F05FFB2B681B0420F47F0203F47F03AD
:10F940001A4306214D4810F046FB0024D1E507215B
:10F950004A4810F04EFB072120F48002474810F07F
:10F960003AFBC6E5002840F084806521434810F04A
:10F9700040FB2860BDE500287FF4F7AD07213F4834
:10F9800010F037FBC0F38150431E584258412860A5
:10F99000AFE512683948522110F01DFB0024A8E59C
:10F9A0003548436AD3F8902114B9D2B22A60A0E551
:10F9B0002B6822F0FF0203F00F031A436321243067
:10F9C00010F009FB002494E52B4B5B6AD3F89021DF
:10F9D00018B9C2F303222A608BE52B6827481B0263
:10F9E00003F4706322F470621A43632110F0F3FA97
:10F9F00000247EE52B681B0403F47F0322F47F02BE
:10FA00001A436321243010F0E6FA002471E51268ED
:10FA10001A48502110F0DFFA00246AE520B9164B8D
:10FA20005B6ADB69136064E512681448532110F0C7
:10FA3000D2FA00245DE528B91521104810F0D9FA52
:10FA4000286056E513680E4A0C485A43152110F0F9
:10FA5000C2FA00244DE504244BE5102449E50424B2
:10FA600047E5102445E5102443E5102441E5102422
:10FA70003FE504243DE500BF0827FF1F2C27FF1F9B
:10FA8000007102000B4619B901461846FFF7FABB90
:10FA9000082070472DE9F84F424CD4F8C462D4F8DE
:10FAA000C0524FEA062949EA1569C6B24FEA05284D
:10FAB00094F8C802D4F8D452002748EA0602D4F8D1
:10FAC000D06249EA070301302F0E2D0245EA166580
:10FAD00004F5307C3602C0B204F5347EC4F8D0623E
:10FAE000C4F8D452CCE9002384F8C80266467546AF
:10FAF000002954D0042805D91A466D2104F12400A8
:10FB000010F069FAD4F8C02227486C2110F063FA8B
:10FB100001200BF093F9D4F8C02223486C2110F097
:10FB20005AFA94F8C8324FF0000B042BC5E900BB19
:10FB30000CD96F211C4810F05CFAD5E900238146EE
:10FB400043EA090142EA0B00C5E900016E211648AB
:10FB500010F04FFAD5E9002343EAE07994F8C8326F
:10FB6000C3F10803DB0042EA0008A3F1200EC3F151
:10FB7000200C09FA03F208FA0EFE42EA0E0228FAF5
:10FB80000CFC42EA0C02404698406A6000230022C6
:10FB9000C6E900230023C4F8D00284F8C8323846EE
:10FBA000BDE8F88F0827FF1F2C27FF1F08B5024864
:10FBB00010F012FB002008BD2C27FF1F07B5019293
:10FBC00039B9014601AA0120FFF75CFB03B05DF8DB
:10FBD00004FB0820FAE7034BD3F8D8320846DB6869
:10FBE000114618470827FF1FF8B54D4C4D4D4E4B99
:10FBF0006A694E4F04F124063046002110F08DFA58
:10FC00004B49304610F0D2FAFE68736803F1E40203
:10FC1000226203F58272E26103F55172A26103F57B
:10FC20005972626103F56172226103F5697203F52D
:10FC30007970E26003F5717203F204432360336864
:10FC4000A260DB68606098473368A069DB6898470A
:10FC500033686069DB68984733682069DB689847D8
:10FC60003368E068DB6898473368A068DB689847CA
:10FC7000336860685B6998473368A0695B69984737
:10FC8000336860695B699847336820695B699847A6
:10FC90003368E0685B6998473368A0685B69984798
:10FCA0003368206A1B6998473368E0691B69984785
:10FCB000336820681B69984773683A69C4F8D8228A
:10FCC00003F5317353606B69002159701949C3F80A
:10FCD0000412012218491A70C3F80812174B6B66F8
:10FCE000174B2B62174BEB61174BAB61174B6B62DA
:10FCF000174BAB63174B6B63174BAB62174BEB6246
:10FD0000174BAB64174B6B64174B6B65174B2B652D
:10FD1000174BEB65174BAB65174B2A74AB66F8BDF9
:10FD20000827FF1F045AFF1F346E02003C7A0200AE
:10FD300039F2000005F20000D1F1000095FA000050
:10FD4000ADFB0000C1F10000ADF1000099F1000031
:10FD500085FA0000BDFB000081F1000069F10000A0
:10FD600025F1000011F1000005F1000029F000006C
:10FD7000A1EF0000ADEF000019F00000014B0022E0
:10FD80005A607047045AFF1F70B5184E184CF5683A
:10FD900060682B689B6998472B68A0699B689847A7
:10FDA0002B6860699B6898472B6820699B68984717
:10FDB0002B68E0689B6898472B68A0689B68984709
:10FDC0002B68206A9B6898472B68E0699B68984776
:10FDD0002B6820689B6898472B6860689B689847E9
:10FDE0003369BDE870405B6A184700BF3C7A020087
:10FDF000F029FF1F0A460146014810F0A1BB00BFD1
:10FE0000142AFF1F022870B5144649D004D890B1B7
:10FE1000012836D0042432E003284FD0FF28F9D13E
:10FE20002B4CD4F88830D3F8043298476369D3F860
:10FE30000432984703E0126832F0030301D0002433
:10FE40001DE0244B244DDE6868693368D2070AD56B
:10FE50001B69984724683268A86914F0020408D026
:10FE600013699847EBE7DB689847336868699B69D3
:10FE7000EFE7D36898473368A8699B69984720469D
:10FE800070BD144B144DDE681468286933680CB1DA
:10FE90001B69E6E7DB689847336828699B69EDE7EB
:10FEA0000C4B0D4DDE6814683368A868002CEFD148
:10FEB000DB6898473368A8689B69DFE7012107483A
:10FEC00010F078FC20600028B9D12024D7E700BFCB
:10FED000045AFF1F3C7A0200F029FF1F142AFF1F5B
:10FEE0000146014810F01CBD142AFF1F10B503483D
:10FEF000144610F0FCFA206010BD00BF142AFF1F4A
:10FF00006C2938B50C4615460BD06D2902D10A4B29
:10FF1000C3F8BC222A4621460848BDE8384010F004
:10FF2000D8BA054BD3F8BC12054B01F07F01D3F8CA
:10FF3000BC309847EEE700BFF029FF1F142AFF1FCF
:10FF4000045AFF1F08B50448D0F8C022243010F02E
:10FF500021FC002008BD00BFF029FF1F08B50448A0
:10FF6000D0F8C022243010F0F9FB002008BD00BFFB
:10FF7000F029FF1F08B50021024810F0D1FB002036
:10FF800008BD00BF142AFF1F08B54942024810F0FF
:10FF9000C7FB002008BD00BF142AFF1F08B5024898
:10FFA00010F0BEFB002008BD142AFF1F38B50A4B15
:10FFB0000A4CDD6860682B689B69984701200AF04D
:10FFC0003DFF2B6860685B69984704F1240010F0DE
:10FFD0007CFB012038BD00BF3C7A0200F029FF1FE6
:10FFE00038B50A4B0A4CDD6860682B689B699847F6
:10FFF00001200AF023FF2B6860685B69984704F1D1
:020000021000EC
:10000000240010F04DFB012038BD00BF3C7A0200F7
:10001000F029FF1F6F2970B50446154600F0818254
:1000200000F28980122900F0D1813ED8052900F024
:10003000718118D8022900F03B8107D8002900F00F
:100040001A81012900F0268104241AE1032900F015
:1000500041810429F8D1B94E002840F04481D6F8F6
:10006000C03213600DE10F2900F082810ED80829FB
:1000700000F068810E29E7D1002840F06E81202130
:10008000AF4810F034FA40002860FAE0102900F080
:100090007D811129D8D1002840F08C812921A848E0
:1000A00010F025FA80102860EBE0182900F0DE81BE
:1000B0001FD8152900F0B3810DD8132900F09481C1
:1000C0001429C1D1002840F0A38126219C4810F0BA
:1000D0000EFA2860D5E0162900F0B3811729B3D1B4
:1000E000002840F0BC812E21954810F000FA2860CD
:1000F000C7E01B2900F0DD810DD8192900F0C4816B
:100100001A29A1D1002840F0CD8133218C4810F06C
:10011000EEF92860B5E06D2900F0E08100F2EC8195
:100120006C2991D1002840F0D2816021844810F0E0
:10013000DEF92860A5E07D2900F0AB8248D875295A
:1001400000F0508222D8722900F01B820FD870294B
:1001500000F0FD8171297FF477AF06217848002CEB
:1001600040F0038210F0C3F9C0B2286089E073291F
:1001700000F01E8274297FF467AF002840F02682C9
:100180006E4B5B6AD3F8703113607AE0782900F027
:100190005D820ED8762900F03C8277297FF454AF37
:1001A000002840F04C825E21654810F0A0F92860DC
:1001B00067E0792900F058827C297FF445AF002858
:1001C00040F060825C215E4810F091F9286058E0B0
:1001D000882900F0AD8228D8842900F08B8215D8B8
:1001E0007E2900F0648281297FF42EAF002800F080
:1001F00084801468002C00F072820121504810F0B5
:10020000D9FA2860002878D120243AE0852900F026
:100210007A8286297FF418AF002840F0828252212A
:10022000474810F064F928602BE0C82995D010D811
:10023000892900F091828A297FF406AF3F48436AFA
:10024000D3F89021002C40F09D82C2F307422A602F
:1002500017E0D42900F0AA82D62900F0B482D1296F
:100260007FF4F2AE002840F09A825021344810F01A
:100270003EF9286005E030B93721314810F037F9F0
:100280002860204670BD12682D48372110F021F9F2
:100290000024F6E728B92121294810F028F9286020
:1002A000EFE712682648212110F013F90024E8E74F
:1002B00030B92421224810F01AF900122860E0E732
:1002C000106810F01BFA242102461D4810F001F9B5
:1002D0000024D6E7002840F086822221184810F03A
:1002E00006F92860CDE71368C6F8C032202106F170
:1002F000240010F0FCF8420701D40024C1E7D6F82E
:10030000C00210F0FBF924210246701810F0E1F849
:100310000024B6E730B92821094810F0E8F8801029
:100320002860AEE71268940DA405002C40F05D82B1
:1003300092002821024810F0CCF8A2E7F029FF1F14
:10034000142AFF1F002840F052820F21A34810F00A
:10035000CEF800F00100286093E713689F48002B57
:100360000CBF01220222202110F0B3F8002488E7FC
:1003700028B92521994810F0BAF8286081E7126859
:100380009648252110F0A5F800247AE730B92A21F3
:10039000924810F0ACF88010286072E71268940D53
:1003A000A405002C40F0258292002A218B4810F0F1
:1003B00090F866E71268940DA405002C40F01B82AB
:1003C00092002921854810F084F85AE728B927219E
:1003D000824810F08CF8286053E712687F48272184
:1003E00010F077F800244CE730B92B217B4810F04F
:1003F0007EF88010286044E71268940DA405002C54
:1004000040F0FB8192002B21744810F062F838E72D
:1004100012687248262110F05CF8002431E728B9F0
:100420002C216E4810F063F828602AE71268940DBA
:10043000A405002C40F0E3812C21684810F049F815
:100440001FE728B92D21654810F051F8286018E7FA
:10045000126862482D2110F03CF8002411E7126860
:100460005E482E2110F035F800240AE728B92F2124
:100470005A4810F03CF8286003E7126857482F21CB
:1004800010F027F80024FCE628B93021534810F07A
:100490002EF82860F5E612685048302110F019F85F
:1004A0000024EEE612684D48332110F012F80024C3
:1004B000E7E628B93421494810F019F82860E0E649
:1004C00012684648342110F004F80024D9E6126876
:1004D000424860210FF0FDFF0024D2E628B96121D7
:1004E0003E4810F004F82860CBE612683B486121D2
:1004F0000FF0EFFF0024C4E61C21384824B90FF0A8
:10050000F6FF00142860BCE60FF0F1FF2A68C0F384
:10051000080040EA02421C2130480FF0DAFF0024B4
:10052000AFE61C212D4824B90FF0E1FFC0B22860CE
:10053000A7E60FF0DCFF2B6800F47F02C3F308038B
:100540001A431C2125480FF0C4FF002499E628B95E
:10055000592122480FF0CBFF286092E612681F480D
:1005600059210FF0B6FF00248BE60FF0C0FF2A7868
:1005700020F0FF000243062118480FF0AAFF0024D4
:100580007FE6062115482CB90FF0B1FFC0F3072014
:10059000286076E60FF0ABFF2B681B0220F47F4249
:1005A0009BB21A4306210D480FF093FF002468E622
:1005B00028B90B4B5B6AD3F86C31136061E61268A3
:1005C00006485A210FF085FF00245AE612680348B6
:1005D0005B210FF07EFF002453E600BF142AFF1FAB
:1005E000F029FF1F8848436AD3F870311CB9C3F360
:1005F0000E03136045E6126823F4FF4323F07F03E4
:10060000C2F30E021A435B2124300FF062FF002474
:1006100037E67D4B5B6AD3F8702118B9C2F3074205
:100620002A602EE62B6879481B0403F47F0322F42A
:100630007F021A435B210FF04CFF002421E6126871
:1006400072485E210FF045FF00241AE628B91821F0
:100650006E480FF04CFF286013E612686B481821B3
:100660000FF037FF00240CE628B9192167480FF076
:100670003EFF286005E61268644819210FF029FF43
:100680000024FEE5126861485C210FF022FF00247F
:10069000F7E528B95F215D480FF029FF2860F0E5F4
:1006A00012685A485F210FF014FF0024E9E5062183
:1006B00056482CB90FF01BFFC0F307402860E0E557
:1006C0000FF015FF2B681B0420F47F0203F47F0357
:1006D0001A4306214D480FF0FCFE0024D1E5072106
:1006E0004A480FF004FF072120F4800247480FF02A
:1006F000F0FEC6E5002840F08480652143480FF0F5
:10070000F6FE2860BDE500287FF4F7AD07213F48DD
:100710000FF0EDFEC0F38150431E5842584128604F
:10072000AFE51268394852210FF0D3FE0024A8E546
:100730003548436AD3F8902114B9D2B22A60A0E5B3
:100740002B6822F0FF0203F00F031A4363212430C9
:100750000FF0BFFE002494E52B4B5B6AD3F8902189
:1007600018B9C2F303222A608BE52B6827481B02C5
:1007700003F4706322F470621A4363210FF0A9FE40
:1007800000247EE52B681B0403F47F0322F47F0220
:100790001A43632124300FF09CFE002471E5126897
:1007A0001A4850210FF095FE00246AE520B9164B37
:1007B0005B6ADB69136064E51268144853210FF02B
:1007C00088FE00245DE528B9152110480FF08FFE42
:1007D000286056E513680E4A0C485A4315210FF05D
:1007E00078FE00244DE504244BE5102449E504245B
:1007F00047E5102445E5102443E5102441E5102485
:100800003FE504243DE500BFF029FF1F142AFF1F28
:10081000007102000B4619B901461846FFF7FABBF2
:10082000082070472DE9F84F424CD4F8CC62D4F838
:10083000C8524FEA062949EA1569C6B24FEA0528A7
:1008400094F8D002D4F8DC52002748EA0602D4F823
:10085000D86249EA070301302F0E2D0245EA1665DA
:1008600004F5327C3602C0B204F5367EC4F8D86294
:10087000C4F8DC52CCE9002384F8D0026646754601
:10088000002954D0042805D91A466D2104F124000A
:100890000FF01FFED4F8C82227486C210FF019FE74
:1008A00001200AF0CBFAD4F8C82223486C210FF0BB
:1008B00010FE94F8D0324FF0000B042BC5E900BBBA
:1008C0000CD96F211C480FF012FED5E90023814698
:1008D00043EA090142EA0B00C5E900016E2116480E
:1008E0000FF005FED5E9002343EAE07994F8D03211
:1008F000C3F10803DB0042EA0008A3F1200EC3F1B4
:10090000200C09FA03F208FA0EFE42EA0E0228FA57
:100910000CFC42EA0C02404698406A600023002228
:10092000C6E900230023C4F8D80284F8D032384640
:10093000BDE8F88FF029FF1F142AFF1F70B5154C72
:1009400094F87430012B05460E461BD0032B0BBFC9
:10095000002228220C230F2343F0884343F0401346
:1009600043EA4232042128460FF0B3FD012E0CD198
:1009700028460FF06DFED4F88830D3F80432BDE875
:100980007040184700220B23E6E7D4F88830D3F8EC
:100990000832F4E7045AFF1F08B502480FF0C0FE02
:1009A000002008BD142AFF1F07B5019239B901467E
:1009B00001AA0120FFF72EFB03B05DF804FB08201D
:1009C000FAE7034BD3F8E0320846DB6811461847D4
:1009D000F029FF1FF8B54D4C4D4D4E4B6A694E4FF7
:1009E00004F12406304600210FF015FE4B49304635
:1009F0000FF080FEFE68736803F1E402226203F5E3
:100A00008272E26103F55172A26103F5597262616B
:100A100003F56172226103F5697203F57970E26092
:100A200003F5717203F2044323603368A260DB684C
:100A3000606098473368A069DB68984733686069ED
:100A4000DB68984733682069DB6898473368E0685B
:100A5000DB6898473368A068DB689847336860684C
:100A60005B6998473368A0695B6998473368606938
:100A70005B699847336820695B6998473368E06829
:100A80005B6998473368A0685B6998473368206A58
:100A90001B6998473368E0691B6998473368206889
:100AA0001B69984773683A69C4F8E02203F531730B
:100AB00053606B69002159701949C3F8041201226F
:100AC00018491A70C3F80812174B6B66174B2B6244
:100AD000174BEB61174BAB61174B6B62174BAB635B
:100AE000174B6B63174BAB62174BEB62174BAB6447
:100AF000174B6B64174B6B65174B2B65174BEB65EF
:100B0000174BAB65174B2A74AB66F8BDF029FF1F76
:100B1000045AFF1F347002003C7A02003D090100B4
:100B2000E1FF0000ADFF0000250801009909010068
:100B30009DFF000089FF000075FF000015080100FF
:100B4000A90901005DFF000045FF000001FF000052
:100B5000EDFE0000E1FE000005FE00007DFD00004E
:100B600089FD0000F5FD000000207047012070475E
:100B7000014B00225A607047045AFF1F1FB5084BF3
:100B800033F8084C5A7802949C1E019433F8041CE4
:100B900000910146002010F039F904B010BD00BFEB
:100BA0005060FF1F10B5002014460FF0FFFE2060BC
:100BB00010BD00200FF01CBF10B5044618B910F08E
:100BC00017F8204610BD0820FCE710B5044618B9F8
:100BD0000FF0F0FF204610BD0820FCE70021F4E7ED
:100BE0004942F2E7F1E7022804BF0C4B93F8E80012
:100BF00030B90B4BDB681B689B690A4A10681847C1
:100C0000012809D1054B93F8E830012B04D1044B9E
:100C1000DB681B685B69F0E7704700BF045AFF1F81
:100C20003C7A0200E02CFF1F10B50020FFF7DBFF2D
:100C3000044B054ADB6810681B68BDE810409B69DF
:100C4000184700BF3C7A0200E02CFF1F10B5044695
:100C500020B909680FF0D9FF204610BD0820FCE735
:100C600038B50D46044620B90FF0BDFF2860204678
:100C700038BD0820FCE7043938B504461546FA2982
:100C800000F23987DFE811F0FB0037073707370735
:100C90003707370737073707370737073707370764
:100CA0003707370737073707370737073707370754
:100CB0003707370737073707370737073707370744
:100CC0003707370737073707370737073707370734
:100CD0003707370737073707370737073707370724
:100CE0003707370709011901370729013901370784
:100CF0003707370737073707370737073707370704
:100D000037073707370737073707370737073707F3
:100D100037073707370737073707370737073707E3
:100D200037073707370737073707370737073707D3
:100D300037073707370737073707370737073707C3
:100D4000370737073707370749015701650173012F
:100D500081018F019D01AB01B901C701D501E301FB
:100D6000F101FF010D021B02290233023D02370788
:100D7000470251025B0265026F027E028D029C02F5
:100D8000A502370737073707AE02B602BE02C80210
:100D9000D202370737073707DA02E202EA023707DB
:100DA000370737073707370737073707F402FE02D9
:100DB000080312033707370737073707370737079F
:100DC0001C03260330033A0344033707370737076A
:100DD000370737074E0358036803780380038C03F3
:100DE00096039F03A903B003BB03C803D503E20323
:100DF000EF03FC0309041604370723042E043B0405
:100E00004804530460046D047A0487049404A30422
:100E1000B204C104D004DF04EE04FD040D05200576
:100E20003005400550056005700580059005A0055A
:100E3000B005C005CF05370737073707370737072E
:100E4000370737073707370737073707DE05EE0558
:100E5000FE050E061E062E063E064E065E066D06B4
:100E60007C068B069A06A906B806C706D606E406CF
:100E7000F206000737070E07190727072F0728B9BB
:100E800060210FF093FD2860204638BD1268602174
:100E900000200FF0ADFD0024F6E730B9024608212E
:100EA0000FF0C6FD00B22860EEE71388002208218B
:100EB00010460FF0CAFD0024E6E730B902460921CA
:100EC0000FF0B6FD00B22860DEE71388002209218A
:100ED00010460FF0BAFD0024D6E730B901220821F0
:100EE0000FF0A6FD00B22860CEE71388082101228A
:100EF00000200FF0AAFD0024C6E730B90122092125
:100F00000FF096FD00B22860BEE713880921012288
:100F100000200FF09AFD0024B6E7002840F0EE858F
:100F2000012203210FF064FD2246022120460FF02A
:100F30007FFD2860A8E7002840F0E3850122032117
:100F40000FF056FD0122022120460FF071FD2860AE
:100F50009AE7002840F0D885022203210FF048FDCF
:100F60002246022120460FF063FD28608CE700280E
:100F700040F0CD85024603210FF03AFD22460221C2
:100F800020460FF055FD28607EE7002840F0C2851E
:100F9000024603210FF02CFD0122022120460FF012
:100FA00047FD286070E7002840F0B785032211460E
:100FB0000FF01EFD2246022120460FF039FD286069
:100FC00062E7002840F0AC85042203210FF010FDF9
:100FD0002246022120460FF02BFD286054E700280E
:100FE00040F0A185042203210FF002FD012202211D
:100FF00020460FF01DFD286046E7002840F096854A
:10100000052203210FF0F4FC2246022120460FF0B6
:101010000FFD286038E7002840F08B85052203216A
:101020000FF0E6FC0122022120460FF001FD2860AE
:101030002AE7002840F08085062203210FF0D8FC23
:101040002246022120460FF0F3FC28601CE700280E
:1010500040F07585072203210FF0CAFC22460221C9
:1010600020460FF0E5FC28600EE7002840F06A8576
:10107000072203210FF0BCFC0122022120460FF0C1
:10108000D7FC286000E7002840F05F850822032194
:101090000FF0AEFC2246022120460FF0C9FC28606A
:1010A000F2E6002840F05485082203210FF0A0FC4E
:1010B0000122022120460FF0BBFC2860E4E6002854
:1010C00040F04985092203210FF092FC22460221BB
:1010D00020460FF0ADFC2860D6E6002840F03E85A3
:1010E000024612210FF0A4FC00B22860CCE60028D2
:1010F00040F03785012212210FF09AFC00B22860DF
:10110000C2E6002840F03085024613210FF090FC23
:1011100000B22860B8E6002840F029850246152173
:101120000FF086FC00B22860AEE6002840F0228571
:10113000012215210FF07CFC00B22860A4E60028F3
:1011400040F01B85024616210FF072FC00B22860A9
:101150009AE6002840F01485012216210FF068FC61
:1011600000B2286090E6002840F00D850A22032195
:101170000FF03EFC2246022120460FF059FC00B23F
:10118000286081E6002840F001850A2203210FF043
:101190002FFC0122022120460FF04AFC00B22860F9
:1011A00072E6002840F0F5840B2203210FF020FCAA
:1011B0002246022120460FF03BFC00B2286063E685
:1011C000002840F0E984024606210FF031FC286037
:1011D0005AE6002840F0E384012206210FF028FCA3
:1011E000286051E6002840F0DD8441210FF0DEFB4D
:1011F000286049E6002840F0D88442210FF0D6FB51
:10120000286041E6002840F0D384012246210FF0F7
:101210000FFC00B2286037E6002840F0CC8402467C
:1012200046210FF005FC00B228602DE6002840F0B2
:10123000C58447210FF0BAFB286025E6002840F05E
:10124000C08421210FF0B2FB28601DE6002840F089
:10125000BB8422210FF0AAFB286015E6002840F08D
:10126000B684024623210FF0E3FB00B228600BE6B0
:10127000002840F0AF8427210FF098FB20F07F403A
:10128000286001E6002840F0A88428210FF08EFB9A
:1012900020F07F402860F7E5002840F0A18401227B
:1012A0002A210FF0C5FB00B22860EDE5002840F0D0
:1012B0009A8402462A210FF0BBFB00B22860E3E5C6
:1012C000002840F09384024639210FF0B1FB00B2B0
:1012D0002860D9E5002840F08C84012239210FF0E4
:1012E000A7FB00B22860CFE5002840F085840246C5
:1012F0003D210FF09DFB00B22860C5E5002840F0BD
:101300007E8402463F210FF093FB00B22860BBE5CC
:10131000002840F0778402463A210FF089FB00B2A2
:101320002860B1E5002840F07084024653210FF098
:101330007FFB00B22860A7E530B9012264210FF0DD
:1013400077FB00B228609FE513886421012200200A
:101350000FF07BFB002497E530B9024664210FF0C3
:1013600067FB00B228608FE51388002264211046D5
:101370000FF06BFB002487E5002840F049846621CC
:101380000FF014FB28607FE520B968210FF00EFBF9
:10139000286079E5116800200FF02AFC002473E52D
:1013A000002840F03884012269210FF041FB00B28F
:1013B000286069E5002840F03184C24B59890FF05C
:1013C000A9FB286060E5002840F02B8402466921D3
:1013D0000FF02EFB00B2286056E5002840F0248470
:1013E0000FF001FC28604FE518B90FF026FC2860CB
:1013F0004AE5116800200FF01CFC002444E5002899
:1014000040F0158402466D210FF0F2FA6C2120465F
:101410000FF0CCFA286037E5002840F00B84012259
:101420006D210FF0E5FA6C2120460FF0BFFA28601D
:101430002AE5002840F0018402226D210FF0D8FA3D
:101440006C2120460FF0B2FA28601DE5002840F01C
:10145000F78303226D210FF0CBFA6C2120460FF0A9
:10146000A5FA286010E5002840F0ED8304226D21E4
:101470000FF0BEFA6C2120460FF098FA286003E5C1
:10148000002840F0E38305226D210FF0B1FA6C21B2
:1014900020460FF08BFA2860F6E4002840F0D9834C
:1014A00006226D210FF0A4FA6C2120460FF07EFA7F
:1014B0002860E9E4002840F0CF8307226D210FF077
:1014C00097FA6C2120460FF071FA2860DCE418B915
:1014D0000FF0F0FA2860D7E4116800200FF0DCFA72
:1014E0000024D1E4774B598918B90FF009FB286023
:1014F000CAE4126800200FF0F1FA0024C4E40028C6
:1015000040F0AD8301226F210FF072FA6E21204668
:101510000FF04CFA2860B7E418B90FF058FB2860B8
:10152000B2E4116800200FF045FB0024ACE4002871
:1015300040F0988303226F210FF05AFA6E21204663
:101540000FF034FA28609FE4002840F08E830422D4
:101550006F210FF04DFA6E2120460FF027FA286018
:1015600092E4002840F0848305226F210FF040FAB6
:101570006E2120460FF01AFA286085E4002840F01A
:101580007A8306226F210FF033FA6E2120460FF086
:101590000DFA286078E4002840F0708307226F215C
:1015A0000FF026FA6E2120460FF000FA28606BE457
:1015B000002840F0668308226F210FF019FA2246B6
:1015C0006E2120460FF034FA00B228605CE4002857
:1015D00040F05A8308226F210FF00AFA01226E218F
:1015E00020460FF025FA00B228604DE4002840F0B4
:1015F0004E8309226F210FF0FBF922466E2120460F
:101600000FF016FA00B228603EE4002840F0428352
:101610000A226F210FF0ECF922466E2120460FF0CE
:1016200007FA00B228602FE4002840F036830A222F
:101630006F210FF0DDF901226E2120460FF0F8F93D
:1016400000B2286020E4002840F02A830B226F219A
:101650000FF0CEF922466E2120460FF0E9F900B2D4
:10166000286011E4002840F01E830B226F210FF048
:10167000BFF901226E2120460FF0DAF900B228608E
:1016800002E4002840F012830C226F210FF0B0F921
:1016900022466E2120460FF0CBF900B22860FFF7FA
:1016A000F3BB002840F005830C226F210FF0A0F956
:1016B00001226E2120460FF0BBF900B22860FFF72F
:1016C000E3BB00BF4860FF1F002840F0F5820D22F9
:1016D0006F210FF08DF922466E2120460FF0A8F9F8
:1016E00000B22860FFF7D0BB002840F0E8820D224E
:1016F0006F210FF07DF901226E2120460FF098F93D
:1017000000B22860FFF7C0BB002840F0DB820E2249
:101710006F210FF06DF922466E2120460FF088F9F7
:1017200000B22860FFF7B0BB002840F0CE820E2246
:101730006F210FF05DF901226E2120460FF078F93C
:1017400000B22860FFF7A0BB002840F0C1820F2242
:101750006F210FF04DF922466E2120460FF068F9F7
:1017600000B22860FFF790BB002840F0B4820F223F
:101770006F210FF03DF901226E2120460FF058F93C
:1017800000B22860FFF780BB002840F0A78210223B
:101790006F210FF02DF922466E2120460FF048F9F7
:1017A00000B22860FFF770BB002840F09A82112237
:1017B0006F210FF01DF922466E2120460FF038F9F7
:1017C00000B22860FFF760BB002840F08D82112234
:1017D0006F210FF00DF901226E2120460FF028F93C
:1017E00000B22860FFF750BB002840F08082122230
:1017F0006F210FF0FDF822466E2120460FF018F9F8
:1018000000B22860FFF740BB002840F0738213222B
:101810006F210FF0EDF822466E2120460FF008F9F7
:101820002860FFF731BB002840F0678213226F2148
:101830000FF0DEF801226E2120460FF0F9F8286043
:10184000FFF722BB002840F05B82C0226F210FF01F
:10185000CFF822466E2120460FF0EAF800B2286049
:10186000FFF712BB002840F04E82C0226F210FF01C
:10187000BFF801226E2120460FF0DAF800B228608E
:10188000FFF702BB002840F04182C1226F210FF018
:10189000AFF822466E2120460FF0CAF800B2286049
:1018A000FFF7F2BA002840F03482C1226F210FF016
:1018B0009FF801226E2120460FF0BAF800B228608E
:1018C000FFF7E2BA002840F02782C2226F210FF012
:1018D0008FF822466E2120460FF0AAF800B2286049
:1018E000FFF7D2BA002840F01A82C2226F210FF00F
:1018F0007FF801226E2120460FF09AF800B228608E
:10190000FFF7C2BA002840F00D82C3226F210FF00A
:101910006FF822466E2120460FF08AF800B2286048
:10192000FFF7B2BA002840F00082C3226F210FF007
:101930005FF801226E2120460FF07AF800B228608D
:10194000FFF7A2BA002840F0F381C4226F210FF004
:101950004FF822466E2120460FF06AF82860FFF704
:1019600093BA002840F0E781C4226F210FF040F8BD
:1019700001226E2120460FF05BF82860FFF784BA41
:10198000002840F0DB81C5226F210FF031F822469C
:101990006E2120460FF04CF82860FFF775BA00283A
:1019A00040F0CF81C5226F210FF022F801226E2175
:1019B00020460FF03DF82860FFF766BA002840F097
:1019C000C381C6226F210FF013F822466E212046F4
:1019D0000FF02EF82860FFF757BA002840F0B781C3
:1019E000C6226F210FF004F801226E2120460FF06D
:1019F0001FF82860FFF748BA002840F0AB81C722E3
:101A00006F210EF0F5FF22466E2120460FF010F8F0
:101A10002860FFF739BA002840F09F81C7226F2164
:101A20000EF0E6FF01226E2120460FF001F828603B
:101A3000FFF72ABA002840F09381C8226F210EF0E8
:101A4000D7FF6E2120460EF0B1FF2860FFF71CBAC9
:101A5000002840F08881C9226F210EF0C9FF6E2155
:101A600020460EF0A3FF2860FFF70EBA002840F0D2
:101A70007D81CA226F210EF0BBFF6E2120460EF041
:101A800095FF2860FFF700BA002840F07281CB2252
:101A90006F210EF0ADFF6E2120460EF087FF28600B
:101AA000FFF7F2B9B74B18B95B891360FFF7ECB9D0
:101AB00012685A810024FFF7E7B920B9B14B5B7A6D
:101AC0001360FFF7E1B9B04A2878511C0FF0A8F96C
:101AD0000024FFF7D9B9002840F04E81A94B1B7AAA
:101AE0001360FFF7D1B9002840F04981A54BDB888E
:101AF0001360FFF7C9B90424FFF7C6B90424FFF740
:101B0000C3B90424FFF7C0B90424FFF7BDB9042406
:101B1000FFF7BAB90424FFF7B7B90424FFF7B4B943
:101B20000424FFF7B1B90424FFF7AEB90424FFF78A
:101B3000ABB90424FFF7A8B90424FFF7A5B904241E
:101B4000FFF7A2B90424FFF79FB90424FFF79CB95B
:101B50000424FFF799B90424FFF796B90424FFF78A
:101B600093B90424FFF790B90424FFF78DB9042436
:101B7000FFF78AB90424FFF787B90424FFF784B973
:101B80000424FFF781B90424FFF77EB90424FFF78A
:101B90007BB90424FFF778B90424FFF775B904244E
:101BA000FFF772B90424FFF76FB90424FFF76CB98B
:101BB0000424FFF769B90424FFF766B90424FFF78A
:101BC00063B90424FFF760B90424FFF75DB9042466
:101BD000FFF75AB90424FFF757B90424FFF754B9A3
:101BE0000424FFF751B90424FFF74EB90424FFF78A
:101BF0004BB90424FFF748B90424FFF745B904247E
:101C0000FFF742B90424FFF73FB90424FFF73CB9BA
:101C10000424FFF739B90424FFF736B90424FFF789
:101C200033B90424FFF730B90424FFF72DB9042495
:101C3000FFF72AB90424FFF727B90424FFF724B9D2
:101C40000424FFF721B90424FFF71EB90424FFF789
:101C50001BB90424FFF718B90424FFF715B90424AD
:101C6000FFF712B90424FFF70FB90424FFF70CB9EA
:101C70000424FFF709B90424FFF706B90424FFF789
:101C800003B90424FFF700B90424FFF7FDB80424C6
:101C9000FFF7FAB80424FFF7F7B80424FFF7F4B805
:101CA0000424FFF7F1B80424FFF7EEB80424FFF78B
:101CB000EBB80424FFF7E8B80424FFF7E5B80424E0
:101CC000FFF7E2B80424FFF7DFB80424FFF7DCB81D
:101CD0000424FFF7D9B80424FFF7D6B80424FFF78B
:101CE000D3B80424FFF7D0B80424FFF7CDB80424F8
:101CF000FFF7CAB80424FFF7C7B80424FFF7C4B835
:101D00000424FFF7C1B80424FFF7BEB80424FFF78A
:101D1000BBB80424FFF7B8B80424FFF7B5B804240F
:101D2000FFF7B2B80424FFF7AFB80424FFF7ACB84C
:101D30000424FFF7A9B80424FFF7A6B80424FFF78A
:101D4000A3B80424FFF7A0B80424FFF79DB8042427
:101D5000FFF79AB80424FFF797B80424FFF794B864
:101D60000424FFF791B80424FFF78EB80424FFF78A
:101D70008BB80424FFF788B80424FFF785B804243F
:101D8000FFF782B84860FF1F5060FF1F0B4619B96C
:101D900001461846FEF76FBF0820704701207047C4
:101DA00007B5019239B9014601AA0120FEF763FF88
:101DB00003B05DF804FB0820FAE710B40C4630B914
:101DC000044B5B6820469B6810BC114618470020F6
:101DD00010BC7047E02CFF1F70B5284E284DF468EA
:101DE000606823686430DB68286098470120FEF74C
:101DF000FAFE636832696A6003F531735360214B00
:101E000021495A69C2F804122049C2F80812002177
:101E1000117051701E4A1A621E4ADA611E4A9A6196
:101E20001E4A5A621E4ADA641E4A9A631E4A5A635E
:101E30001E4A9A621E4ADA621E4A9A641E4A5A640E
:101E40001E4A5A651E4A1A651E4A1A661E4ADA65F5
:101E500001221A741D4A9A65322040F28A22C3E98F
:101E600002201B4B4FF47A729A8041F270721A6012
:101E700059724FF480725A8170BD00BF3C7A0200E3
:101E8000E02CFF1F045AFF1F6D0B01009D1D010078
:101E9000CB0B0100E50B0100E10B0100DD0B0100A4
:101EA000610C01008D1D0100A11D0100B90B010095
:101EB0004D0C0100B30B0100A50B01007D0B0100CF
:101EC000690B0100E70B0100710B0100290C0100F7
:101ED0004860FF1F00207047014B00225A60704786
:101EE000045AFF1F00200EF0CBBF08B50022104699
:101EF00017210EF0C5FF002210461A210EF0C0FF78
:101F000041F61912192100200EF0BAFF012008BD78
:101F1000EBE710B5002014460EF090FF206010BDD6
:101F2000022804BF0B4B93F8E80030B90A4BDB687A
:101F30001B689B69094A10681847012809D1054B9D
:101F400093F8E830012B04D1034BDB681B685B6915
:101F5000F0E77047045AFF1F3C7A0200F42CFF1F81
:101F600010B50020FFF7DCFF044B054ADB68106862
:101F70001B68BDE810409B69184700BF3C7A02000F
:101F8000F42CFF1FF0B5294B294D5A7885B0074630
:101F900033F8060C0290981E019033F8041C00914F
:101FA000002039460FF0BEF96B68BB4230D105B056
:101FB000F0BD204B1B78032B0FD11F4E20460CF099
:101FC00027FCA26833689A4205D0682100200EF0F1
:101FD00057FFA36833606F60E9E7022B15D1174EF6
:101FE00020460CF0E4FB226933689A42F3D0662164
:101FF00000200EF045FF236933606B2100200EF0B6
:102000001DFF0023A060E361E5E7012BE3D1F4E7C6
:102010000B4C94F82060002ECBD16B2130460EF093
:102020000DFF2661A060E661D5E700BF4E60FF1F8F
:10203000F42CFF1F7C60FF1F8460FF1F8060FF1F68
:102040005860FF1F38B50D46044620B90FF057F809
:102050002860204638BD0820FCE770B50E46E0B980
:102060000F4D95F82040A4B10E4C2278012A02D1E0
:102070000FF045F828610321002021700EF044FF85
:102080006B2100200EF0DAFE3368184468600020EF
:1020900070BD09680FF045F8F9E70820F8E700BFC0
:1020A0005860FF1F7C60FF1F70B50E46A8B90C4D2D
:1020B00095F8204074B10B4C2278012A02D10FF020
:1020C0001EF828610321002021700EF01DFF6E60B4
:1020D000002070BD0FF018F8FAE70820F9E700BFFC
:1020E0005860FF1F7C60FF1F70B50E46A8B90C4DED
:1020F00095F8204074B10B4C2278012A02D10EF0E1
:10210000FEFF28610221002021700EF0FDFEEE602E
:10211000002070BD0EF0E3FFFAE70820F9E700BFEA
:102120005860FF1F7C60FF1F0021DDE74942DBE7AD
:10213000DAE738B515460C4600295DD1AC283BD00E
:1021400018D80C2834D00AD8042829D00B2855D107
:102150005F2120460EF094FE294B5D6126E00D289C
:1021600024D0AB284AD193B20122642120460EF03C
:10217000B4FE1BE0BE2833D008D8B3281FD0BD283A
:102180003CD1114620460EF0CFFE0FE0FB2830D0A8
:10219000FC2833D11B4AE8B2511C0FF0CDF805E002
:1021A000602120460EF06CFE154B1D60204638BDA8
:1021B000134B83F82020F9E793B20A46D5E76B2149
:1021C00020460EF05DFE104B1B78032BEED10C4B1E
:1021D0002A46C3E90155682120460EF051FEE5E785
:1021E0000A4B204619890EF0CCFE074B01221A70CB
:1021F000DCE7064B1A81D9E70824D7E70424D5E7A2
:102200005860FF1F4E60FF1F7C60FF1F4860FF1F6C
:1022100038B515460C46002940F09080B22877D09A
:1022200023D8AB2863D013D80B284DD003D804286B
:1022300041D0042446E00C284ED00D28F9D1404B63
:1022400093F82020002A4CD01B692B60002439E031
:10225000AD2856D053D3AE2858D0B028E9D1394B49
:10226000204619890EF0A9FE47E0C0285ED013D899
:10227000BD2851D005D8B328DBD108460EF069FF40
:102280003BE0BE284CD0BF28D3D101226F2120468D
:102290000EF0F6FD6E2135E0FC2849D004D8FB286D
:1022A000C7D1284B1B891AE0FD2844D0FE28C0D195
:1022B000244B9B8813E0602120460EF0BFFD204B8D
:1022C00028601860204638BD5F2120460EF0B6FD1C
:1022D0001B4B28605861F5E7194B93F820302B60B1
:1022E000F0E7662100200EF0A9FD2860AEE701228C
:1022F000642120460EF0E4FD00B22860E2E70A46C1
:10230000F6E7662120460EF099FDF6E76821F9E729
:1023100008460EF0F4FEF0E708460EF013FEECE778
:10232000084B204619890EF03EFEE6E70222ADE793
:10233000044BDB79D3E7034B9B79D0E70824C1E753
:102340005860FF1F4860FF1F10B40C4630B9054BA2
:102350009B6820469B6810BC11461847002010BCA3
:10236000704700BFF42CFF1F70B5424E424DF46819
:10237000606823686430DB68286098470120FFF7B5
:10238000CFFD63683269AA6003F5317353603B4B3C
:102390003B495A693B4DC2F804123B49C2F8081246
:1023A0000024012111705470384A1A62384ADA61E7
:1023B000384A9A61384A5A62384ADA64384A9A6323
:1023C000384A5A63384A9A62384ADA62384A9A6412
:1023D000384A5A64384A5A65384A1A65384A1A6679
:1023E000384ADA65384A19749A65462140F28A22D9
:1023F000C3E90221354B4FF47A725A8041F2707270
:102400001A804FF480721A81DC712246172120460F
:102410000EF036FD22461A2120460EF031FD41F61F
:102420001912192120460EF02BFD224606212046C6
:102430000EF026FD4FF4FA625F2120460EF020FDDB
:102440004FF47A62602120460EF01AFD28460CF007
:10245000A3F91F4B1C701F4B1C601F4B60212046B3
:102460001C600EF0EBFC5F21286020460EF0E6FCBD
:10247000686170BD3C7A0200F42CFF1F045AFF1FF4
:10248000EB1E01005860FF1F111F0100E920010031
:10249000312101002D2101002921010045200100E9
:1024A0001122010033210100A92001005B2001005D
:1024B000E51E0100131F0100851F0100D51E01004C
:1024C000211F0100D91E0100611F01004860FF1F8C
:1024D0007C60FF1F8460FF1F8060FF1F014B002294
:1024E0005A607047045AFF1F70B5084C261D0546F8
:1024F00023683246014600200EF0FAFF2368324678
:1025000029460120BDE870400EF0F2BF0C2DFF1FE0
:10251000014B18680FF04DB80C2DFF1F01280CD887
:10252000074B1A68202303FA00F040F0020002EB88
:10253000800043680B60002070470820704700BF90
:102540000C2DFF1F012810B5144612D003D302280A
:102550001CD004200AE0114B114ADB6824681B6878
:10256000D2F8A8021CB15B699847002010BD9B6996
:10257000FAE70A4B0A4ADB68D2F8A0021B685B6ADA
:102580009847003018BF01202060EEE7034B044A53
:10259000DB68D2F8A4021B685B6AF1E73C7A0200B0
:1025A0000C2DFF1F022804BF0C4B93F8E80038B92C
:1025B0000B4BDB681B685B690A4AD2F89C02184720
:1025C000012809D1054B93F8E830012B04D1044BC5
:1025D000DB681B689B69EFE7704700BF045AFF1F69
:1025E0003C7A02000C2DFF1F70B50020FFF7DAFFC8
:1025F000134B144CDD68D4F89C022B689B689847F9
:102600002B68D4F8A0029B6898472B68D4F8A402E2
:102610009B6898472B68D4F8B4029B6898472B684E
:10262000D4F8AC029B6898472B68D4F8B0029B683A
:1026300098472B68D4F8A8029B68BDE870401847FB
:102640003C7A02000C2DFF1F2DE9F8431A4C9DF82F
:1026500020609DF824509846D4F8B8320F469B6805
:10266000002147F0800091469847D4F8B832002105
:102670009B6848469847D4F8B83200219B6840468A
:102680009847D4F8B83200219B6830469847D4F870
:10269000B83228469B6801219847236848EA0928F0
:1026A00007F07F0746EA082603EB870745EA062579
:1026B0007D60BDE8F88300BF0C2DFF1F07B5D3B2C6
:1026C0000193C2F307230093C2F30743120EFFF7EF
:1026D000BBFF03B05DF804FB0020FFF7EFBF01284C
:1026E0002DE9F34105460F4628D8DFF8588020260B
:1026F00018F80030864074B263B1114B03EB8003CD
:1027000044F00701D3F8BC22C9B2FFF7D7FF00237A
:1027100008F8053044F00D013A460024C9B22846B5
:10272000FFF7CCFF2846CDE9004423462246F1B20C
:10273000FFF78AFF204602B0BDE8F0810820FAE7E3
:102740000C2DFF1F7800FF1F012873B505460E46AC
:102750001CD82024844044F0070186EAE672A2EBEC
:10276000E672C9B2FFF7AAFF094A0123002E5355AA
:10277000E1B2B8BF02230024CDE900432846234636
:102780002246FFF761FF204602B070BD0820FBE73C
:102790007800FF1F0021D7E74942D5E7D4E738B5D5
:1027A000274D01F07F042B1993F81832DB0704D46E
:1027B0002B6803EB8404606838BDD5F8B83200217B
:1027C0009B6820469847D5F8B83200219B68084698
:1027D0009847D5F8B83200219B6808469847D5F845
:1027E000B83200219B6808469847D5F8B8320121D5
:1027F0009B6800209847D5F8B83200219B68204696
:102800009847D5F8B83200219B6808469847D5F814
:10281000B832002104029B6808469847D5F8B832C0
:10282000002104439B6808469847D5F8B832240233
:1028300004439B6801210020984724022043BBE702
:102840000C2DFF1F10B500201446FFF7A8FF2060D5
:1028500010BD38B50D462021814041F00101C9B2BB
:102860000446FFF79CFF2968014429602046BDE823
:10287000384034E71C2A2DE9F84304460D461E462D
:1028800000F0198300F2A8800C2A00F049824CD88D
:10289000052A00F0E8811AD8022A00F09B8107D8A7
:1028A000002A00F07381012A00F08381042477E17B
:1028B000032A00F0A981042AF8D1CC4B8A001344E2
:1028C000002840F0B481D3F8BC32336068E1082AB4
:1028D00000F0058214D8062A00F0D681072AE5D137
:1028E00020278F4047F01007FFB239462846002CBA
:1028F00040F0E781FFF753FF00F01F0030604FE129
:102900000A2A00F0FB810B2AD0D1002840F0DB8599
:102910002021A94041F01501C9B22846FFF73FFF29
:10292000C04300F0010030603AE1122A00F06282F8
:1029300027D80F2A00F0368211D80D2A00F00E8217
:102940000E2AB3D12021A94041F01401C9B20028B8
:1029500040F022822846FFF722FF306020E1102A53
:1029600000F03182112AA1D12021A94041F00801B3
:10297000C9B2002840F038822846FFF710FF3060C7
:102980000EE1152A00F05E8211D8132A00F043826E
:10299000142A8BD12021A94041F00B01C9B2002893
:1029A00040F04A822846FFF7FAFE3060F8E0172A26
:1029B00000F06A82C0F05782182A7FF477AF202196
:1029C000A94041F01301C9B2002840F06E822846A8
:1029D000FFF7E5FE3060E3E0AC2A00F0288463D81E
:1029E000A52A00F02F8331D8A22A00F0E48218D85B
:1029F0001D2A00F07E828C2A7FF458AF002840F018
:102A00008682090141F06C0101F0FC012846FFF7C4
:102A1000C6FE4FF48073C0F3036043FA00F03060E9
:102A2000BEE0A32A00F0E382A42A7FF43FAF0F01A7
:102A300047F06C07FFB239462846002C40F0F3827D
:102A4000FFF7ADFEC0F300303060A9E0A82A00F027
:102A50008B8314D8A62A00F03B83A72A7FF426AFE5
:102A60000F0147F06C07FFB239462846002C40F0B2
:102A70006D83FFF794FE00F00F00306090E0AA2A0B
:102A80004FEA011700F0A68340F2898347F06D07F3
:102A9000FFB239462846002C40F0BA83FFF77FFE8C
:102AA000C0F3411030607BE0B62A00F04C843ED881
:102AB000B32A00F002841BD8AD2A00F0D383AE2ADB
:102AC0007FF4F4AE0F0147F06D07FFB23946284698
:102AD000002C40F0E383FFF762FE001400F07F0358
:102AE00010F0400018BF6FF07F001843306057E0CF
:102AF000B42A00F0FE83B52A7FF4D8AE20278F4099
:102B00007FB247F014085FFA88F841462846FFF77D
:102B100046FE002C40F0FD83410540F1F88347F06C
:102B20001101C9B22846FFF73AFE306038E0CE2ADC
:102B300000F0478414D8B82A00F01684B92A7FF42C
:102B4000B5AE0F0147F06C07FFB239462846002C9E
:102B500040F02784FFF723FEC0F3035030601FE0EE
:102B6000D22A00F04484D32A00F05484D12A7FF47E
:102B70009DAE2021A94041F01901C9B2002840F0C2
:102B80002F842846FFF70BFE306009E02021A94082
:102B900041F00D01C9B230B92846FFF700FE3060A0
:102BA0002046BDE8F8831A682846FFF787FD002411
:102BB000F6E72021A94041F00101C9B220B9284619
:102BC000FFF7EDFD3060EBE71A682846FFF776FD6A
:102BD0000024E5E72021A94041F00701C9B238B936
:102BE0002846FFF7DCFD3060DAE700BF0C2DFF1F41
:102BF000B74B01225A553268002AB8BF52422846C4
:102C0000FFF75CFD0024CBE7002840F0538420212F
:102C1000A94041F00201C9B22846FFF7C0FD10F4F7
:102C2000000318BF4FF07F4318433060B8E73268A5
:102C30002027002A07FA01F7B8BF5242F9B2284606
:102C4000C3F8BC22FFF7ABFD044608B10024A7E798
:102C5000326847F00701002AB8BF5242C9B228467D
:102C6000FFF72CFD9CE72021A94041F00601C9B2E5
:102C700020B92846FFF793FD306091E71A6828468F
:102C8000FFF71CFD00248BE720278F4047F010073B
:102C9000FFB2394628462CB9FFF781FDC0F3042066
:102CA00030607DE7FFF77BFD33681B0203F4F853C8
:102CB00020F4F8521A4339462846FFF7FFFC002457
:102CC0006EE7FFF76CFD336820F01F0203F01F036F
:102CD0001A4339462846FFF7F1FC002460E7002834
:102CE00040F0EB832021A94041F01501C9B22846EC
:102CF000FFF755FDC0F34020306051E7002840F059
:102D0000DF832021A94041F01501C9B22846FFF711
:102D100046FD10F0020F0CBF0123002333603FE794
:102D200020278F4047F01407FFB2394628462CB9B8
:102D3000FFF735FDC0F34000306031E7FFF72FFDAE
:102D40003368002B20F0020214BF002302231A4331
:102D500039462846FFF7B2FC002421E720278F40A0
:102D600047F01407FFB2394628462CB9FFF717FD84
:102D700000F00100306013E7FFF711FD326820F02A
:102D80000100002A14BF024640F0010239462846DD
:102D9000FFF794FC002403E71A682846FFF78EFC2F
:102DA0000024FDE62021A94041F00401C9B220B968
:102DB0002846FFF7F4FC3060F2E61A682846FFF771
:102DC0007DFC0024ECE62021A94041F00501C9B2B8
:102DD00020B92846FFF7E3FC3060E1E61A68284690
:102DE000FFF76CFC0024DBE61A682846FFF766FC58
:102DF0000024D5E62021A94041F00A01C9B220B93A
:102E00002846FFF7CCFC3060CAE61A682846FFF770
:102E100055FC0024C4E62021A94041F00301C9B2B9
:102E200020B92846FFF7BBFC3060B9E61A6828468F
:102E3000FFF744FC0024B3E61A682846FFF73EFC7F
:102E40000024ADE62021A94041F00C01C9B220B90F
:102E50002846FFF7A4FC3060A2E61A682846FFF770
:102E60002DFC00249CE62021A94041F01101C9B2AB
:102E700020B92846FFF793FC306091E61A6828468F
:102E8000FFF71CFC00248BE62021A94041F0120131
:102E9000C9B220B92846FFF782FC306080E61A6884
:102EA0002846FFF70BFC00247AE61A682846FFF74D
:102EB00005FC002474E60F0147F06C07FFB23946A9
:102EC00028463CB9FFF76BFCC0F38040306067E6F2
:102ED0007800FF1FFFF763FC33689B0403F4802333
:102EE00020F480221A4339462846FFF7E7FB0024E6
:102EF00056E6002840F0EA82C44B20201B68884038
:102F000040F0020003EB80004368336048E61B6832
:102F1000102B4AD00DDC022B43D004DC012B16D041
:102F20004FF0FF3314E0042B3DD0082BF8D10523DC
:102F30000EE0402B3BD003DC202BF1D1032307E034
:102F4000802B36D0B3F5807FEAD1002300E0082340
:102F50003360336801333FF479AE2C0144F06C04E4
:102F6000E4B221462846FFF71AFC33681B0603F03B
:102F7000706320F070621A4321462846FFF79EFBDB
:102F800021462846FFF70BFC33681B0603F07063ED
:102F900020F0706221461A432846FFF78FFB002479
:102FA000FEE50723D4E70623D2E70423D0E7022374
:102FB000CEE70123CCE70F0147F06C07FFB239469B
:102FC00028462CB9FFF7EBFBC0F3C1303060E7E5D2
:102FD000FFF7E5FB3368DB0303F4C03320F4C032B2
:102FE0001A4339462846FFF769FB0024D8E50F014C
:102FF00047F06C07FFB2394628462CB9FFF7CFFBE4
:10300000C0F380303060CBE5FFF7C9FB33689B032A
:1030100003F4804320F480421A4339462846FFF7E0
:103020004DFB0024BCE5FFF7BAFB33681B0303F438
:10303000805320F480521A4339462846FFF73EFB5E
:103040000024ADE50F0147F06C07FFB23946284672
:10305000FFF7A5FB3946814600F480482846B4B9FD
:10306000B8F1000F05D0FFF79AFBC0F3C310306032
:1030700096E5FFF794FB19F4006FC0F3021001D13D
:103080003060E3E540F008003060444688E5B8F180
:10309000000F0ED0FFF783FB3368DB0103F4F0630E
:1030A00020F4F0621A4339462846FFF707FB002454
:1030B00076E5FFF774FB33681B0103F0700320F023
:1030C00070021A4339462846FFF7F8FA444667E586
:1030D0000F0147F06C07FFB239462846FFF75FFB48
:1030E000394600F4804828467CB9B8F1000F05D075
:1030F000FFF755FBC0F30210306051E5FFF74FFBBF
:10310000C0F3C310306044464AE5B8F1000F0ED05A
:10311000FFF745FB33681B0103F0700320F07002DA
:103120001A4339462846FFF7C9FA002438E5FFF765
:1031300036FB3368DB0103F4F06320F4F0621A43DA
:1031400039462846FFF7BAFA444629E5FFF727FB38
:10315000336820F00F0203F00F031A433946284664
:10316000FFF7ACFA00241BE50F0147F06D07FFB233
:10317000394628462CB9FFF712FBC0F3C030306047
:103180000EE5FFF70CFB3368DB039BB220F4004233
:103190001A4339462846FFF791FA002400E547F024
:1031A0006D07FFB2394628462CB9FFF7F8FAC0F38D
:1031B00041303060F4E4FFF7F2FA33685B0303F464
:1031C000C04320F4C0421A4339462846FFF776FA36
:1031D0000024E5E447F06D07FFB2394628462CB9D4
:1031E000FFF7DDFAC0F303203060D9E4FFF7D7FA28
:1031F00033681B0203F4706320F470621A4339468B
:103200002846FFF75BFA0024CAE400BF0C2DFF1F1D
:10321000FFF7C5FA33685B0103F0600320F060023A
:103220001A4339462846FFF749FA0024B8E40F014B
:1032300047F06D07FFB2394628462CB9FFF7AFFAC1
:1032400000F00F003060ABE4FFF7A9FA336820F01C
:103250000F0203F00F031A4339462846FFF72EFAF0
:1032600000249DE40F0147F06D07FFB23946284660
:103270002CB9FFF794FAC0F30060306090E4FFF7D8
:103280008EFA33681B0603F0807320F080721A43B5
:1032900039462846FFF712FA002481E4FFF77FFA47
:1032A00033681B0403F4FE0320F4FE021A4339467C
:1032B0002846FFF703FA002472E40F0147F06C0779
:1032C000FFB2394628462CB9FFF769FAC0F34040EF
:1032D000306065E4FFF763FA33685B0403F400339E
:1032E00020F400321A4339462846FFF7E7F9002454
:1032F00056E4002840F0ED80090141F06F01C9B2A9
:103300002846FFF74CFAC0F30440306048E43460CC
:1033100046E447F011013268C9B22846FFF7CEF9FA
:1033200041462846FFF73BFA3368002B20F48062C1
:103330000CBF00234FF480631A4341462846FFF731
:10334000BDF900242CE42021A94041F01101C9B2AB
:1033500020B92846FFF723FA306021E41A6828468E
:10336000FFF7ACF900241BE40F0147F06C07FFB234
:10337000394628462CB9FFF712FAC0F340303060C6
:103380000EE4FFF70CFA33685B0303F4005320F4F8
:1033900000521A4339462846FFF790F90024FFF7F8
:1033A000FFBBFFF7FCF933681B0503F4700320F43F
:1033B00070021A4339462846FFF780F90024FFF7C8
:1033C000EFBB002840F08880090141F06F01C9B2CD
:1033D0002846FFF7E4F9C0F309003060FFF7E0BBCF
:1033E0001A682846FFF76AF90024FFF7D9BB2021A5
:1033F000A94041F01A01C9B228B92846FFF7CFF910
:103400003060FFF7CDBB1A682846FFF757F9002454
:10341000FFF7C6BBE8B979B101297FF4C1AB01461A
:103420002846FFF7BCF900F06000A0F120035842E5
:1034300058413060FFF7B4BB0846FFF7B0F900F021
:103440001800A0F110025042504130602C46FFF7A6
:10345000A7BB21B1012917D00024FFF7A1BB084663
:10346000FFF79DF9336853B120F0080242F01002D3
:1034700000210846FFF722F90024FFF791BB20F056
:10348000100242F00802F3E700212846FFF787F90F
:10349000336853B120F0400242F0200200210120A5
:1034A000FFF70CF90024FFF77BBB20F0200242F06D
:1034B0004002F3E70424FFF773BB0424FFF770BB5B
:1034C0000424FFF76DBB0424FFF76ABB0424FFF755
:1034D00067BB0424FFF764BB0424FFF761BB012929
:1034E000134603D802460020FFF7C4B908207047EE
:1034F00007B50129019207D8024601AB0120FFF769
:10350000B9F903B05DF804FB0820FAE708B52221F9
:103510000020FFF744F950B942210120FFF73FF99D
:1035200028B9044B1868BDE808400EF03BB80020ED
:1035300008BD00BF0C2DFF1F70B5434C434E201D2E
:103540000DF098FFF5686B6803F58272C4F8A0224D
:1035500003F59272C4F8A42203F57172C4F8A8228C
:1035600003F5797203F16400C4F8AC2203F204425B
:1035700003F22443C4F8B4322B68C4F8B022DB68E9
:10358000C4F89C0298472B68D4F8A802DB689847D7
:103590002B68D4F8A8029B6998472B68D4F8A0023E
:1035A0001B6998472B68D4F8A4021B6998472B68BD
:1035B000D4F8B4021B6998472B68D4F8AC021B6995
:1035C00098472B68D4F8B0021B6998476B6832693A
:1035D000C4F8B82203F5317353601D4B1D495A6975
:1035E0002260C2F804121C49C2F80812012000210E
:1035F00051701070194A1A62194ADA61194A9A61AF
:10360000194A5A62194A9A63194A5A63194A9A62BC
:10361000194ADA62194A9A64194A5A64194A5A6567
:10362000194A1A65194ADA64194A1A66194ADA6592
:1036300002221A743221B622C3E90221164A9A657F
:10364000BDE87040FEF7AEBF0C2DFF1F3C7A0200B4
:10365000045AFF1F0D350100112501004927010003
:103660009D2701009927010095270100DF34010003
:10367000F1340100DF26010053280100D9260100A2
:1036800045280100E9240100452501001D25010010
:10369000A5250100DD240100E925010001289FBFC7
:1036A000034B53F820300B60002088BF0820704780
:1036B000DC2FFF1F014B00225A607047045AFF1F86
:1036C00070B5094C0546D4F89832224601460020D0
:1036D0000DF0B6FFD4F89832224629460120BDE805
:1036E00070400DF0ADBF00BFDC2FFF1F024BD3F8C1
:1036F00098020DF0F0BF00BFDC2FFF1F012810B5AE
:10370000144603D002280FD004200CE00A4B0B4AC9
:10371000DB68D2F8A0021B685B6A9847003018BFCC
:1037200001202060002010BD034B044ADB68D2F862
:10373000A4021B685B6AF0E73C7A0200DC2FFF1FE3
:10374000022804BF0C4B93F8E80038B90B4BDB6838
:103750001B685B690A4AD2F89C021847012809D104
:10376000054B93F8E830012B04D1044BDB681B6850
:103770009B69EFE7704700BF045AFF1F3C7A0200C5
:10378000DC2FFF1F70B50020FFF7DAFF094B0A4C52
:10379000DD68D4F89C022B689B6898472B68D4F8A6
:1037A000A0029B6898472B68D4F8A4029B68BDE8E8
:1037B000704018473C7A0200DC2FFF1F2DE9F843C8
:1037C0001A4C9DF820609DF824509846D4F8A832F1
:1037D0000F469B68002147F0800091469847D4F837
:1037E000A83200219B6848469847D4F8A8320021A7
:1037F0009B6840469847D4F8A83200219B68304621
:103800009847D4F8A83228469B6801219847D4F8F5
:10381000983248EA092807F07F0746EA082603EBB2
:10382000870745EA06257D60BDE8F883DC2FFF1F8A
:1038300007B5D3B20193C2F307230093C2F3074342
:10384000120EFFF7BBFF03B05DF804FB0020FFF78B
:10385000EFBF01282DE9F34105460F462BD8174B42
:1038600003EB0008202698F89422864074B272B1C7
:10387000D3F8983246F0070203EB820344F00701C5
:103880005A68C9B2FFF7D4FF002388F8943244F095
:103890000D013A460024C9B22846FFF7C9FF284661
:1038A000CDE9004423462246F1B2FFF787FF2046C8
:1038B00002B0BDE8F0810820FAE700BFDC2FFF1F4F
:1038C000012873B505460C4621D82026864084EA97
:1038D000E47246F00701A2EBE472C9B2FFF7A8FF59
:1038E0000C4B2B44002C4FF0010283F894224FF034
:1038F0000004ACBF134602230193284600942346DC
:103900002246F1B2FFF75AFF204602B070BD0820F0
:10391000FBE700BFDC2FFF1F0021D1E74942CFE7C3
:10392000CEE738B5284D01F07F042B1993F81432F7
:10393000DB0705D4D5F8983203EB8404606838BD02
:10394000D5F8A83200219B6820469847D5F8A832C0
:1039500000219B6808469847D5F8A83200219B684B
:1039600008469847D5F8A83200219B680846984732
:10397000D5F8A83201219B6800209847D5F8A832D5
:1039800000219B6820469847D5F8A83200219B6803
:1039900008469847D5F8A832002104029B680846DB
:1039A0009847D5F8A832002104439B6808469847F9
:1039B000D5F8A832240204439B68012100209847CF
:1039C00024022043BBE700BFDC2FFF1F10B50020FF
:1039D0001446FFF7A6FF206010BD38B50D46202124
:1039E000814041F00101C9B20446FFF79AFF2968FE
:1039F000014429602046BDE838402AE71C2A2DE909
:103A0000F04104460D461E4600F02F8300F2AF80C1
:103A10000C2A00F03D8253D8052A00F0DC8121D821
:103A2000022A00F0948109D8002A00F06E81012A50
:103A300000F07C8104242046BDE8F081032A00F0D8
:103A4000A181042AF6D1C74B2021A940D3F898328E
:103A500041F00707BA001344002840F0A6815B68D4
:103A60003360E8E7082A00F0F28114D8062A00F053
:103A7000C381072ADED120278F4047F01007FFB20D
:103A800039462846002C40F0D481FFF74AFF00F069
:103A90001F003060CFE70A2A00F0E8810B2AC9D165
:103AA000002840F0B8852021A94041F01501C9B295
:103AB0002846FFF736FFC04300F001003060BAE748
:103AC000122A00F06F8227D80F2A00F0438211D803
:103AD0000D2A00F00B820E2AACD12021A94041F022
:103AE0001401C9B2002840F02F822846FFF719FFC1
:103AF0003060A0E7102A00F03E82112A9AD12021DE
:103B0000A94041F00801C9B2002840F0458228468A
:103B1000FFF707FF30608EE7152A00F06B8211D89F
:103B2000132A00F05082142A84D12021A94041F0A8
:103B30000B01C9B2002840F057822846FFF7F1FE7A
:103B4000306078E7172A00F07982C0F06482182A82
:103B50007FF470AF2021A94041F01301C9B20028C1
:103B600040F07D822846FFF7DCFE306063E7AB2A39
:103B700000F0228461D8A52A00F0278331D8A22A38
:103B800000F0DC8218D81D2A00F08B828C2A7FF48A
:103B900051AF002840F08D82090141F06C0101F025
:103BA000FC012846FFF7BDFE4FF48073C0F30360AD
:103BB00043FA00F030603EE7A32A00F0DB82A42A3B
:103BC0007FF438AF0F0147F06C07FFB23946284643
:103BD000002C40F0EB82FFF7A4FEC0F30030306011
:103BE00029E7A82A00F09D8312D8A62A00F0438373
:103BF000A72A7FF41FAF0F0147F06C07FFB23946C9
:103C00002846002C40F08283FFF78BFE346012E7D9
:103C1000A92A00F0A383AA2A7FF40CAF0F0147F072
:103C20006D07FFB239462846002C40F0B583FFF7F8
:103C300078FEC0F303203060FDE6B52A00F04C8426
:103C40002CD8AE2A00F0058414D8AC2A00F0D48316
:103C5000AD2A7FF4EFAE0F0147F06D07FFB2394692
:103C60002846002C40F0E583FFF75BFEC0F30060C0
:103C70003060E0E6B32A00F01184B42A7FF4DAAEB3
:103C8000002840F0CE84090141F06F01C9B22846F6
:103C9000FFF747FEC0F304403060CCE6CE2A00F0C8
:103CA000668414D8B62A00F03F84B82A7FF4C2AEE6
:103CB0000F0147F06C07FFB239462846002C40F050
:103CC0004684FFF72EFEC0F340303060B3E6D12AC1
:103CD000FFF4B0AED22A40F29284D32A7FF4AAAE87
:103CE000002840F05F84002900F04F8401297FF410
:103CF000A2AE01462846FFF714FE00F06000A0F1D6
:103D0000200358425841306095E62021A94041F0F7
:103D10000D01C9B220B92846FFF703FE30608AE6DC
:103D20001A682846FFF784FD002484E62021A94074
:103D300041F00101C9B220B92846FFF7F2FD306019
:103D400079E61A682846FFF773FD002473E6202100
:103D5000A94041F00701C9B230B92846FFF7E1FD9B
:103D6000306068E6DC2FFF1FB34B2B44012283F841
:103D700094223268002AB8BF52422846FFF758FD05
:103D8000002458E6002840F03D842021A94041F05D
:103D90000201C9B22846FFF7C4FD10F4000318BFA2
:103DA0004FF07F431843306045E63268002AB8BFC1
:103DB00052425A60C9B22846FFF7B3FD044608B123
:103DC000002438E63268002AB8BF5242F9B22846C9
:103DD000FFF72EFD2FE62021A94041F00601C9B2D0
:103DE00020B92846FFF79DFD306024E61A68284672
:103DF000FFF71EFD00241EE620278F4047F0100726
:103E0000FFB2394628462CB9FFF78BFDC0F30420DA
:103E1000306010E6FFF785FD33681B0203F4F853AA
:103E200020F4F8521A4339462846FFF701FD0024D2
:103E300001E6FFF776FD336820F01F0203F01F0351
:103E40001A4339462846FFF7F3FC0024F3E500281F
:103E500040F0DB832021A94041F01501C9B228467A
:103E6000FFF75FFDC0F340203060E4E5002840F03C
:103E7000CF832021A94041F01501C9B22846FFF7A0
:103E800050FD10F0020F0CBF012300233360D2E578
:103E900020278F4047F01407FFB2394628462CB937
:103EA000FFF73FFDC0F340003060C4E5FFF739FD88
:103EB0003368002B0CBF0023022320F002021A43B8
:103EC00039462846FFF7B4FC39462846FFF729FD56
:103ED0003368022B20F0080214BF002308231A4382
:103EE00039462846FFF7A4FC0024A4E520278F408C
:103EF00047F01407FFB2394628462CB9FFF711FDE9
:103F000000F00100306096E5FFF70BFD326820F00D
:103F10000100002A0CBF024640F001023946284643
:103F2000FFF786FC39462846FFF7FBFC3368022B77
:103F300020F0040214BF002304231A433946284604
:103F4000FFF776FC002476E51A682846FFF770FC38
:103F5000002470E52021A94041F00401C9B220B934
:103F60002846FFF7DEFC306065E51A682846FFF753
:103F70005FFC00245FE52021A94041F00501C9B2A2
:103F800020B92846FFF7CDFC306054E51A68284672
:103F9000FFF74EFC00244EE51A682846FFF748FC60
:103FA000002448E52021A94041F00A01C9B220B906
:103FB0002846FFF7B6FC30603DE51A682846FFF753
:103FC00037FC002437E52021A94041F00301C9B2A4
:103FD00020B92846FFF7A5FC30602CE51A68284672
:103FE000FFF726FC002426E51A682846FFF720FC88
:103FF000002420E52021A94041F00C01C9B220B9DC
:104000002846FFF78EFC306015E51A682846FFF752
:104010000FFC00240FE52021A94041F01101C9B295
:1040200020B92846FFF77DFC306004E51A68284671
:10403000FFF7FEFB0024FEE4DC2FFF1F2021A94038
:1040400041F01201C9B220B92846FFF76AFC30607E
:10405000F1E41A682846FFF7EBFB0024EBE41A684A
:104060002846FFF7E5FB0024E5E40F0147F06C0765
:10407000FFB2394628462CB9FFF753FCC0F3804005
:104080003060D8E4FFF74DFC33689B0403F48023D1
:1040900020F480221A4339462846FFF7C9FB002442
:1040A000C9E4002840F0BA82CA4B53F8213033608B
:1040B000C1E41B68102B3BD00DDC022B34D004DC98
:1040C000012B16D04FF0FF3314E0042B2ED0082B19
:1040D000F8D105230EE0402B2CD003DC202BF1D1AE
:1040E000032307E0802B27D0B3F5807FEAD100239C
:1040F00000E008233360336801333FF461AE2C01E4
:1041000044F06C04E4B221462846FFF70AFC336809
:104110001B0603F0706320F0706221461A432846A4
:10412000FFF786FB002486E40723E3E70623E1E7A5
:104130000423DFE70223DDE70123DBE70F0147F07C
:104140006C07FFB2394628462CB9FFF7EAFBC0F3EB
:10415000C13030606FE4FFF7E4FB3368DB0303F446
:10416000C03320F4C0321A4339462846FFF760FBBB
:10417000002460E40F0147F06C07FFB2394628467F
:104180002CB9FFF7CEFBC0F38030306053E4FFF76B
:10419000C8FB33689B0303F4804320F480421A4336
:1041A00039462846FFF744FB002444E4FFF7B9FBF7
:1041B00033681B0303F4805320F480521A433946BA
:1041C0002846FFF735FB002435E40F0147F06C0764
:1041D000FFB239462846FFF7A4FB00F48048B4B983
:1041E000B8F1000F07D039462846FFF79AFBC0F315
:1041F000C31030601FE40311010503F0700301D404
:104200003360DDE543F008033360444613E4394688
:104210002846B8F1000F0FD0FFF783FB3368DB01AE
:1042200003F4F06320F4F0621A4339462846FFF79E
:10423000FFFA0024FFF7FFBBFFF773FB326812029F
:1042400020F4006002F40062024339462846FFF77A
:10425000EFFA39462846FFF764FB33681B0103F089
:10426000700320F070021A4339462846FFF7E0FA3F
:104270004446FFF7E0BB0F0147F06C07FFB2394639
:104280002846FFF74EFB394680462846C4B918F445
:10429000804407D0FFF745FBC0F3021030600024D4
:1042A000FFF7C9BBFFF73DFB18F4006FC0F3C31065
:1042B00001D1306084E540F008003060FFF7BBBBFF
:1042C000FFF72FFB10F48044394628460FD0FFF744
:1042D00028FB33681B0103F0700320F070021A43BF
:1042E00039462846FFF7A4FA0024FFF7A4BBFFF7DE
:1042F00018FB3368DB0103F4F06320F4F0621A4327
:1043000039462846FFF794FAFFF795BBFFF709FBFC
:10431000394620F00F022846FFF78AFA0024FFF7FB
:104320008ABB0F0147F06D07FFB23946284634B902
:10433000FFF7F7FAC0F3C0303060FFF77CBBFFF740
:10434000F0FA3368DB039BB220F400421A4339468B
:104350002846FFF76DFA0024FFF76DBB0F0147F009
:104360006D07FFB23946284634B9FFF7DAFAC0F3D1
:1043700041303060FFF75FBBFFF7D3FA33685B0370
:1043800003F4C04320F4C0421A4339462846FFF7DD
:104390004FFA0024FFF74FBBFFF7C3FA33681B0245
:1043A00003F4706320F470621A4339462846FFF71D
:1043B0003FFA0024FFF73FBB0F0147F06D07FFB244
:1043C0003946284644B9FFF7ACFAC0F341103060D3
:1043D000FFF731BBDC2FFF1FFFF7A3FA33685B0148
:1043E00003F0600320F060021A4339462846FFF7C5
:1043F0001FFA0024FFF71FBB0F0147F06D07FFB244
:104400003946284634B9FFF78CFA00F00F003060C7
:10441000FFF711BBFFF785FA336820F00F0203F0B6
:104420000F031A4339462846FFF702FA0024FFF724
:1044300002BBFFF776FA33681B0603F0807320F0A7
:1044400080721A4339462846FFF7F2F90024FFF735
:10445000F2BA0F0147F06D07FFB2394628466CB932
:10446000FFF75FFA001400F07F0310F0400018BF60
:104470006FF07F0018433060FFF7DDBAFFF751FAA5
:1044800033681B0403F4FE0320F4FE021A4339468A
:104490002846FFF7CDF90024FFF7CDBA0F0147F00A
:1044A0006C07FFB23946284634B9FFF73AFAC0F331
:1044B00040403060FFF7BFBAFFF733FA33685B0460
:1044C00003F4003320F400321A4339462846FFF73C
:1044D000AFF90024FFF7AFBA20278F407FB247F033
:1044E0001101C9B228B92846FFF71BFA3060FFF75F
:1044F000A2BA47F014041A68E4B22846FFF798F904
:1045000021462846FFF70DFA3368002B20F480621D
:104510000CBF00234FF4806321461A432846FFF75F
:1045200087F90024FFF787BA2021A94041F0110143
:10453000C9B228B92846FFF7F4F93060FFF77BBA13
:104540001A682846FFF774F90024FFF774BAFFF7DA
:10455000E8F933685B0303F4005320F400521A4374
:1045600039462846FFF764F90024FFF764BA0028AB
:104570005AD1090141F06F01C9B22846FFF7D1F9BC
:10458000C0F309003060FFF756BA0846FFF7C9F9D3
:1045900000F01800A0F110025042504130602C464B
:1045A000FFF749BA21B1012915D00024FFF743BA1A
:1045B0000846FFF7B6F9336820F0180243B142F01D
:1045C000100200210846FFF733F90024FFF733BA41
:1045D00042F00802F5E700212846FFF7A2F9336808
:1045E00020F0600243B142F0200200210120FFF7D9
:1045F0001FF90024FFF71FBA42F04002F5E700243C
:10460000FFF719BA0424FFF716BA0424FFF713BA08
:104610000424FFF710BA0424FFF70DBA0424FFF7AF
:104620000ABA0424FFF707BA0424FFF704BA07B54F
:104630000129019207D8024601AB0120FFF7DEF9FC
:1046400003B05DF804FB0820FAE70129134603D8FC
:1046500002460020FFF7D2B90820704708B5222192
:104660000020FFF75EF958B942210120FFF759F900
:1046700030B9044BD3F89802BDE808400DF022B8D9
:10468000002008BDDC2FFF1F70B5304C304E204697
:104690000CF098FFF5686B6803F5827203F1640013
:1046A00003F59273C4F8A4322B68C4F8A022DB6827
:1046B000C4F89C0298472B68D4F8A0021B6998475D
:1046C0002B68D4F8A4021B6998476B683269C4F858
:1046D000A82203F5317353601E4B1F495A69C4F871
:1046E0009822C2F804121D49C2F808120121117063
:1046F000002151701A4A1A621A4ADA611A4A9A61FA
:104700001A4A5A621A4A9A631A4A5A631A4A9A62A7
:104710001A4ADA621A4A9A641A4A5A641A4A5A6552
:104720001A4A1A651A4ADA641A4A1A661A4ADA657D
:1047300002204FF48C723221C3E902211874174A07
:104740009A65BDE87040FEF7FBBF00BFDC2FFF1F7E
:104750003C7A0200045AFF1F5D460100ED3601005D
:10476000C1380100213901001D390100193901004A
:104770004B4601002F46010053380100DB39010090
:104780004D380100CD390100C1360100FD36010070
:104790009D36010041370100B53601008537010023
:1047A00001289FBF044B03EB8000C3690B6094BFDB
:1047B00000200820704700BF9432FF1F014B0022E9
:1047C0005A607047045AFF1F014601480DF019B99D
:1047D0009432FF1F0A46014601480CF0B1BF00BFEA
:1047E0009432FF1F10B500201446FFF7F3FF20603E
:1047F00010BD38B514460A46014603481D460CF064
:104800009FFF2040E84038BD9432FF1F13460A4600
:10481000014601480CF090BF9432FF1F0020F5E7DD
:104820002DE9F0470C4D089C06460F4690460A4677
:104830000146284699460CF083FF04FA09F24240EB
:1048400002EA080282EA000331463A462846BDE8F9
:10485000F0470CF071BF00BF9432FF1F01480DF00C
:1048600030B800BF9432FF1F08B522210020FFF7A7
:10487000B1FF48B942210120FFF7ACFF20B903483E
:10488000BDE808400DF005B8002008BD9432FF1FB8
:10489000012810B5144612D003D302281CD00420DE
:1048A0000AE0114B114ADB6824681B68D2F8B00299
:1048B0001CB15B699847002010BD9B69FAE70A4B61
:1048C0000A4ADB68D2F8A8021B685B6A9847003086
:1048D00018BF01202060EEE7034B044ADB68D2F8E2
:1048E000AC021B685B6AF1E73C7A02009432FF1F5E
:1048F000022804BF0C4B93F8E80038B90B4BDB6877
:104900001B685B690A4AD2F8A4021847012809D13A
:10491000054B93F8E830012B04D1044BDB681B688E
:104920009B69EFE7704700BF045AFF1F3C7A020003
:104930009432FF1F70B50020FFF7DAFF134B144CC1
:10494000DD68D4F8A4022B689B6898472B68D4F8DC
:10495000A8029B6898472B68D4F8AC029B689847DC
:104960002B68D4F8BC029B6898472B68D4F8B40233
:104970009B6898472B68D4F8B8029B6898472B68C7
:10498000D4F8B0029B68BDE8704018473C7A02003A
:104990009432FF1F01282DE9F041044688461FD8B4
:1049A000104F07EB80072025D7F8C02285406EB254
:1049B0003AB146F00701C9B2FFF728FF0023C7F854
:1049C000C03246F00D014246C9B22046FFF71EFF35
:1049D00020460022E9B2FFF719FF0020BDE8F08170
:1049E0000820FBE79432FF1F38B50D462021814097
:1049F00041F00101C9B20446FFF7ECFE2968014409
:104A000029602046BDE83840C4E701282DE9F0417F
:104A10000446884623D8134F07EB8007202585409E
:104A2000D7F8C03245F00706F6B223B93146FFF792
:104A3000D1FEC7F8C00288EAE872A2EBE8723146FC
:104A40002046FFF7E3FEB8F1000F2046B4BF022274
:104A50000122E9B2FFF7DAFE0020BDE8F08108206C
:104A6000FBE700BF9432FF1F0021CEE74942CCE7AD
:104A7000CBE71C2A2DE9F34104460D461E4600F003
:104A8000FB8200F2AE800C2A00F03B8252D8052A4D
:104A900000F0E3811FD8022A00F0A28107D8002A83
:104AA00000F07781012A00F0888104247BE1032A49
:104AB00000F0AA81042AF8D1C84B2021A940D3F8DC
:104AC000C83241F00707BA001344002840F0AF8114
:104AD0005B68336067E1082A00F0F18113D8062A89
:104AE00000F0CC81072AE0D12021A94041F010013B
:104AF000C9B2002840F0DA8103461F222846FFF79A
:104B000078FE30604FE10A2A00F0E9810B2ACCD10F
:104B1000002840F04C852021A94041F015010346B2
:104B20000122C9B22846FFF764FEB0FA80F04009BE
:104B3000306038E1122A00F03E8227D80F2A00F0B8
:104B4000128211D80D2A00F0F2810E2AADD1202157
:104B5000A94041F01401C9B2002840F0FE81284666
:104B6000FFF738FE30601EE1102A00F00D82112A96
:104B70009BD12021A94041F00801C9B2002840F092
:104B800014822846FFF726FE30600CE1152A00F05B
:104B90003A8211D8132A00F01F82142A85D12021CD
:104BA000A94041F00B01C9B2002840F026822846F6
:104BB000FFF710FE3060F6E0172A00F04682C0F0E2
:104BC0003382182A7FF471AF2021A94041F01301EC
:104BD000C9B2002840F04A822846FFF7FBFD30604A
:104BE000E1E0AC2A00F0C98362D8A52A00F0DA829D
:104BF00032D8A22A00F09E8219D81D2A00F05382D2
:104C00008C2A7FF452AF002840F05682090141F00F
:104C10006C0118234FF0706201F0FC012846FFF789
:104C2000E8FD4FF4807343FA00F03060BBE0A32A44
:104C300000F09782A42A7FF438AF090141F06C019B
:104C4000C9B2002840F0A4820C234FF480522846B9
:104C5000FFF7CFFD3060A6E0A82A00F0428313D80A
:104C6000A62A00F0F282A72A7FF41FAF090141F0C3
:104C70006C01C9B2002840F02B8303460F2228465E
:104C8000FFF7B7FD30608EE0AA2A4FEA011100F06D
:104C9000558340F23D8341F06D01C9B2002840F0D8
:104CA0006383052360222846FFF7A3FD30607AE086
:104CB000B62A00F0D6833DD8B32A00F097831AD8DD
:104CC000AD2A00F07283AE2A7FF4EFAE090141F005
:104CD0006D01C9B2002840F07F8310234FF4FE021B
:104CE0002846FFF786FD10F0400318BF6FF07F03E2
:104CF0001843306057E0B42A00F08F83B52A7FF460
:104D0000D4AE20278F407FB247F014085FFA88F8AE
:104D1000002840F0918341462846FFF75BFD41059E
:104D200040F1908047F01101C9B22846FFF752FDCB
:104D3000306038E0CE2A00F0C68314D8B82A00F0DC
:104D4000A183B92A7FF4B1AE090141F06C01C9B267
:104D5000002840F0AE8314234FF470022846FFF77A
:104D600048FD30601FE0D22A00F0C183D32A00F052
:104D7000CF83D12A7FF499AE2021A94041F01901B7
:104D8000C9B2002840F0AD832846FFF723FD30600C
:104D900009E02021A94041F00D01C9B238B92846E7
:104DA000FFF718FD3060204602B0BDE8F0811A68B8
:104DB0002846FFF72BFD0024F5E72021A94041F00C
:104DC0000101C9B220B92846FFF704FD3060EAE7C7
:104DD0001A682846FFF71AFD0024E4E79432FF1F03
:104DE0002021A94041F00701C9B220B92846FFF7A8
:104DF000F1FC3060D7E71A68002AB8BF5242284653
:104E0000FFF704FD0024CEE7002840F0C8832021EE
:104E1000A94041F00201C9B22846FFF7DBFC10F4BB
:104E2000000318BF4FF07F4318433060BBE7326880
:104E3000002AB8BF52425A60C9B22846FFF7CAFCDE
:104E4000044608B10024AEE73268002AB8BF5242D7
:104E5000F9B22846FFF7DAFCA5E72021A94041F086
:104E60000601C9B220B92846FFF7B4FC30609AE7C2
:104E70001A682846FFF7CAFC002494E72021A940BD
:104E800041F01001C9B238B908234FF4F85228464E
:104E9000FFF7AFFC306086E71B6800934FF4F852D1
:104EA00008232846FFF7BCFC00247CE71B6800931E
:104EB0001F2200232846FFF7B3FC002473E70028D5
:104EC00040F06F832021A94041F0150109234FF4E0
:104ED0000072C9B22846FFF78CFC306063E70028F7
:104EE00040F062832021A94041F0150101230222F4
:104EF000C9B22846FFF77DFCB0FA80F04009306067
:104F000051E72021A94041F01401C9B230B9012371
:104F100002222846FFF76DFC306044E71B680093CF
:104F2000022201232846FFF77BFC00243BE72021D7
:104F3000A94041F01401C9B230B90023012228462A
:104F4000FFF757FC30602EE71B6800930122002317
:104F50002846FFF765FC002425E71A682846FFF776
:104F600055FC00241FE72021A94041F00401C9B2EB
:104F700020B92846FFF72EFC306014E71A6828464F
:104F8000FFF744FC00240EE72021A94041F0050171
:104F9000C9B220B92846FFF71DFC306003E71A6844
:104FA0002846FFF733FC0024FDE61A682846FFF781
:104FB0002DFC0024F7E62021A94041F00A01C9B2E6
:104FC00020B92846FFF706FC3060ECE61A68284650
:104FD000FFF71CFC0024E6E62021A94041F0030174
:104FE000C9B220B92846FFF7F5FB3060DBE61A6846
:104FF0002846FFF70BFC0024D5E61A682846FFF781
:1050000005FC0024CFE62021A94041F00C01C9B2E3
:1050100020B92846FFF7DEFB3060C4E61A68284650
:10502000FFF7F4FB0024BEE62021A94041F0110166
:10503000C9B220B92846FFF7CDFB3060B3E61A6845
:105040002846FFF7E3FB0024ADE62021A94041F00C
:105050001201C9B220B92846FFF7BCFB3060A2E6B6
:105060001A682846FFF7D2FB00249CE61A682846F7
:10507000FFF7CCFB002496E6090141F06C01C9B2B0
:1050800038B912234FF480222846FFF7B2FB306074
:1050900089E61B6800934FF4802212232846FFF70D
:1050A000BFFB00247FE6002840F08482B94800EB73
:1050B0008100C369336076E61B68102B34D00DDCA9
:1050C000022B2DD004DC012B16D04FF0FF3314E05F
:1050D000042B27D0082BF8D105230EE0402B25D038
:1050E00003DC202BF1D1032307E0802B20D0B3F584
:1050F000807FEAD1002300E0082333603368581C26
:105100003FF4A0AE290141F06C0100934FF07062B2
:10511000182301F0FC012846FFF782FB002442E639
:105120000723EAE70623E8E70423E6E70223E4E7A8
:105130000123E2E7090141F06C01C9B238B90F233C
:105140004FF4C0322846FFF754FB30602BE61B6853
:1051500000934FF4C0320F232846FFF761FB002471
:1051600021E6090141F06C01C9B238B90E234FF4B0
:1051700080422846FFF73DFB306014E61B68009331
:105180004FF480420E232846FFF74AFB00240AE62C
:105190001B6800934FF480520C232846FFF740FB16
:1051A000002400E60F0147F06C07FFB240BB0E235E
:1051B0004FF4804239462846FFF71BFB804640B13A
:1051C00007234FF4F06239462846FFF712FB3060A0
:1051D000E9E50423702239462846FFF70AFB0B2332
:1051E00030604FF4006239462846FFF702FB002882
:1051F0003FF428AE336843F0080333604446D2E5F9
:1052000039462846FFF7E6FA10F48044336809D09F
:1052100000934FF4F062072339462846FFF700FB5E
:105220000024C0E5C3F3C0030093394628460B238E
:105230004FF40062FFF7F4FA3368009370220423FE
:1052400039462846FFF7ECFAADE50F0147F06C0749
:10525000FFB23946284624BBFFF7BCFA10F480445D
:1052600008D00423702239462846FFF7C2FA0024EA
:10527000306098E507234FF4F06239462846FFF77F
:10528000B8FA0B2330604FF4006239462846FFF726
:10529000B0FA00283FF4D6AD336843F0080333601A
:1052A00081E5FFF797FA3368009310F4804407D044
:1052B0000423702239462846FFF7B2FA002472E52B
:1052C00007234FF4F06239462846FFF7A9FA6AE54A
:1052D0001B6800930F2200232846FFF7A1FA002441
:1052E00061E5090141F06D01C9B238B90F234FF4EE
:1052F00000422846FFF77DFA306054E51B680093B2
:105300004FF400420F232846FFF78AFA00244AE5AB
:1053100041F06D01C9B238B90D234FF4C04228469F
:10532000FFF767FA30603EE51B6800934FF4C04218
:105330000D232846FFF774FA002434E541F06D018F
:10534000C9B238B908234FF470622846FFF751FA02
:10535000306028E51B6800934FF4706208232846EC
:10536000FFF75EFA00241EE51B6800936022052308
:105370002846FFF755FA002415E5090141F06D01B3
:10538000C9B248B903460F222846FFF732FA306007
:1053900009E500BF9432FF1F1B6800930F22002312
:1053A0002846FFF73DFA0024FDE4090141F06D01B4
:1053B000C9B238B918234FF080722846FFF719FA9E
:1053C0003060F0E41B6800934FF080721823284689
:1053D000FFF726FA0024E6E41B6800934FF4FE0270
:1053E00010232846FFF71CFA0024DCE4090141F0F1
:1053F0006C01C9B238B911234FF400322846FFF7C7
:10540000F8F93060CFE41B6800934FF400321123A9
:105410002846FFF705FA0024C5E4002840F0CD80B7
:10542000090141F06F0110234FF4F812C9B2284668
:10543000FFF7DFF93060B6E447F011011A68C9B22E
:105440002846FFF7E3F93368003318BF01230093C0
:105450004FF480620A2341462846FFF7E1F9002411
:10546000A1E42021A94041F01101C9B220B9284688
:10547000FFF7B0F9306096E41A682846FFF7C6F9DE
:10548000002490E4090141F06C01C9B238B90D2340
:105490004FF400522846FFF7ACF9306083E41B68F4
:1054A00000934FF400520D232846FFF7B9F900246A
:1054B00079E41B6800934FF4700214232846FFF729
:1054C000AFF900246FE400287AD1090141F06F019F
:1054D000034640F2FF32C9B22846FFF78AF930602E
:1054E00061E41A682846FFF791F900245BE4202163
:1054F000A94041F01A01C9B220B92846FFF76AF95C
:10550000306050E41A682846FFF780F900244AE426
:10551000D8B971B101297FF446AC01462846FFF79E
:1055200059F900F06000A0F1200358425841306062
:1055300039E40846FFF74EF900F01800A0F1100218
:105540005042504130602C462DE419B1012913D04E
:10555000002428E40846FFF73DF9336820F01802DC
:105560003BB142F0100200210846FFF74FF900243A
:1055700019E442F00802F6E700212846FFF72AF96D
:10558000336820F060023BB142F02002002101208C
:10559000FFF73CF9002406E442F04002F6E7042459
:1055A00001E40424FFF7FFBB0424FFF7FCBB042441
:1055B000FFF7F9BB0424FFF7F6BB0424FFF7F3BBA6
:1055C0000424FFF7F0BB07B50129019207D8024672
:1055D00001AB0120FFF74DFA03B05DF804FB082092
:1055E000FAE7012938B505460C460FD1084B1022C1
:1055F00000210CF0A1F82846054B214618220CF09A
:105600009BF80448BDE838400CF00EB938BD00BF27
:10561000C80405009432FF1F0129134603D802462F
:105620000020FFF726BA08207047012810B40C4666
:1056300007D8054BD3F8CC3220469B6810BC1146E6
:105640001847002010BC70479432FF1F2DE9F0412D
:10565000604C614D614B6169C5F8C8128CB001277F
:10566000CDE900735E4ADFF8E081002328460CF0A4
:10567000B3F85C4928460CF008F9D8F80C60736858
:1056800003F58272C5F8A82203F59272C5F8AC2220
:1056900003F57172C5F8B02203F5797203F1640065
:1056A000C5F8B42203F2044203F22443C5F8BC3225
:1056B0003368C5F8B822DB68C5F8A4029847336898
:1056C000D5F8B002DB6898473368D5F8B0029B691B
:1056D00098473368D5F8A8021B6998473368D5F80E
:1056E000AC021B6998473368D5F8BC021B69984720
:1056F0003368D5F8B4021B6998473368D5F8B80207
:105700001B6998477368D8F81020C5F8CC2203F5B8
:1057100031735360344B029303F19F2303F56A0303
:1057200056330393314A324B3248CDE90423324B8E
:105730006FF08061CDE90613A3F1D943A3F591136E
:10574000A3F2272308932D4B02AACDE909030021D8
:105750004FF477432846ADF82C300CF0ECF902AA50
:10576000394628460CF0E7F96369254AC3F8042254
:10577000244AC3F8082200221F705A70224B236269
:10578000224BE361224BA361224B6362224BA36352
:10579000224B6363224BA362224BE362224BA3643E
:1057A000224B6364224B6365224B2365224BE364E7
:1057B000224B2366224BE365022323743225DE232A
:1057C000C4E9023538461F4BA365FFF791F80CB0CA
:1057D000BDE8F081045AFF1F9432FF1F0024F4003B
:1057E00034720200E355010054B5AAAA29294924BC
:1057F00022421010224240007D77BBB580FFFF5649
:10580000694801005D4801000B4A0100714A01002E
:105810006D4A0100694A010019560100C75501008F
:1058200095490100E94901001D480100E5470100D3
:10583000C947010091480100A1470100F14801005A
:10584000BD470100354901003C7A020001289FBF95
:10585000044B03EB8000C3680B6094BF002008205A
:10586000704700BF7035FF1F014B00225A60704720
:10587000045AFF1F38B5064C0546014620460CF079
:10588000F1FA29462046BDE838400CF0EBBA00BFDB
:105890007035FF1F10B5034814460CF076FA2060EF
:1058A00010BD00BF7035FF1F01480CF060BA00BF8B
:1058B0007035FF1F10B50446054800EB84020B4607
:1058C000D2F8982221460CF0BCFB002010BD00BF8E
:1058D0007035FF1F10B50446054800EB84030A46E7
:1058E000D3F8983221460CF08EFB002010BD00BF8B
:1058F0007035FF1F08B5014602480CF081FB0020FF
:1059000008BD00BF7035FF1F08B50A4601460248B2
:105910000CF073FB002008BD7035FF1F08B50A4668
:10592000014602480CF067FB002008BD7035FF1FE0
:1059300008B50A46014602480CF03FFB002008BDAE
:105940007035FF1F01480CF01FBB00BF7035FF1FF3
:1059500008B5222107480CF018FA48B94221054839
:105960000CF013FA20B90348BDE808400CF0F4BA73
:10597000002008BD7035FF1F012810B5144612D055
:1059800003D302281CD004200AE0114B114ADB6823
:1059900024681B68D2F8AC021CB15B6998470020F0
:1059A00010BD9B69FAE70A4B0A4ADB68D2F8A402E9
:1059B0001B685B6A9847003018BF01202060EEE743
:1059C000034B044ADB68D2F8A8021B685B6AF1E764
:1059D0003C7A02007035FF1F022804BF0C4B93F87D
:1059E000E80038B90B4BDB681B685B690A4AD2F8E0
:1059F000A0021847012809D1054B93F8E830012B84
:105A000004D1044BDB681B689B69EFE7704700BF5C
:105A1000045AFF1F3C7A02007035FF1F70B500204A
:105A2000FFF7DAFF134B144CDD68D4F8A0022B68A3
:105A30009B6898472B68D4F8A4029B6898472B680A
:105A4000D4F8A8029B6898472B68D4F8B8029B68E2
:105A500098472B68D4F8B0029B6898472B68D4F815
:105A6000B4029B6898472B68D4F8AC029B68BDE8E9
:105A7000704018473C7A02007035FF1F1C2A2DE940
:105A8000F04106460C461F4600F0298300F2A9802B
:105A90000C2A00F034824DD8052A00F0D5811BD89D
:105AA000022A00F08C8107D8002A00F06481012AC4
:105AB00000F07481042668E1032A00F09781042A2B
:105AC000F8D1DFF824838D004544002840F0A181FF
:105AD000D5F898323B6058E1082A00F0F28115D8D9
:105AE000062A00F0C281072AE4D1202101FA04F439
:105AF00044F01004E4B22146BB48002E40F0D381AC
:105B00000CF043F900F01F0038603EE10A2A00F073
:105B1000E7810B2ACED1002840F0F2852021A14058
:105B200041F01501C9B2B0480CF02FF900F00100A6
:105B300038602AE1122A00F06E8227D80F2A00F07E
:105B4000428211D80D2A00F009820E2AB2D12021FA
:105B5000A14041F01401C9B2002840F02E82A248B1
:105B60000CF013F9386010E1102A00F03D82112A80
:105B7000A0D12021A14041F00801C9B2002840F085
:105B8000448299480CF001F93860FEE0152A00F0D3
:105B90006A8211D8132A00F04F82142A8AD1202158
:105BA000A14041F00B01C9B2002840F056828E4856
:105BB0000CF0EBF83860E8E0172A00F07982C0F0CA
:105BC0006382182A7FF476AF2021A14041F01301AF
:105BD000C9B2002840F07D8283480CF0D6F83860C6
:105BE000D3E0AB2A00F00F8463D8A52A00F0288305
:105BF00031D8A22A00F0DD8218D81D2A00F08B824D
:105C00008C2A7FF457AF002840F08E82090141F0C2
:105C10006C0101F0FC0174480CF0B7F84FF480738C
:105C200000F00F0043FA00F03860AEE0A32A00F065
:105C3000DC82A42A7FF43EAF0C0144F06C04E4B291
:105C400021466948002E40F0EC820CF09EF8C0F32B
:105C50000030386099E0A82A00F08D8314D8A62A75
:105C600000F03783A72A7FF425AF0C0144F06C04C1
:105C7000E4B221465C48002E40F06F830CF085F8BA
:105C800000F00F00386080E0A92A00F09183AA2A72
:105C90007FF410AF0C0144F06D04E4B22146524889
:105CA000002E40F0A1830CF070F8C0F303203860A0
:105CB0006BE0B52A00F02C842CD8AE2A00F0E983E2
:105CC00014D8AC2A00F0BB83AD2A7FF4F3AE0C01EC
:105CD00044F06D04E4B221464348002E40F0CA83EC
:105CE0000CF053F8C0F3006038604EE0B32A00F0C7
:105CF000F383B42A7FF4DEAE002840F00785090163
:105D000041F06F01C9B238480CF03FF8C0F30440CD
:105D100038603AE0CE2A00F0528414D8B62A00F057
:105D20002B84B82A7FF4C6AE0C0144F06C04E4B2B4
:105D300021462D48002E40F032840CF026F8C0F3A6
:105D40004030386021E0D22A00F05284D32A00F09B
:105D50006284D12A7FF4AEAE202101FA04F444F02B
:105D60001904E4B221462048002E40F037840CF09C
:105D70000CF8386009E02021A14041F00D01C9B2C2
:105D800030B919480CF001F838603046BDE8F081B0
:105D90001A6815480BF0EBFF0026F6E72021A1401A
:105DA00041F00101C9B220B90F480BF0EEFF386095
:105DB000EBE71A680C480BF0DAFF0026E5E7202134
:105DC000A14041F00701C9B220B907480BF0DDFF3F
:105DD0003860DAE71A680448002AB8BF52420BF06C
:105DE000C6FF0026D1E700BF7035FF1F002840F036
:105DF0007E842021A14041F00201C9B2AB480BF0E2
:105E0000C4FF10F4000318BF4FF07F4318433860FD
:105E1000BBE71B682026002B06FA01F6B8BF5B42E1
:105E2000F1B24046C5F898320BF0AFFF044608B116
:105E30000026AAE746F00701D5F89822C9B24046E5
:105E40000BF095FF2646A0E72021A14041F0060176
:105E5000C9B220B995480BF098FF386095E71A68E9
:105E600092480BF084FF00268FE7202101FA04F40A
:105E700044F01004E4B221468C482EB90BF085FFA3
:105E8000C0F30420386080E70BF07FFF3B681B0203
:105E900003F4F85320F4F8521A43214683480BF0D8
:105EA00066FF002671E70BF070FF3B6820F01F02D1
:105EB00003F01F031A4321467C480BF058FF0026CD
:105EC00063E7002840F016842021A14041F015012D
:105ED000C9B276480BF059FFC0F34020386054E750
:105EE000002840F00A842021A14041F01501C9B2E8
:105EF0006E480BF04AFFC0F34000386045E72021B0
:105F000001FA04F444F01404E4B2214667482EB9BF
:105F10000BF03BFFC0F34000386036E70BF035FF75
:105F20003B68002BD4BF0023022320F002021A4357
:105F300021465E480BF01BFF21465C480BF025FF15
:105F40003B68022B20F0080214BF002308231A43E9
:105F5000214656480BF00BFF002616E7202101FAD8
:105F600004F444F01404E4B2214650482EB90BF076
:105F70000CFF00F00100386007E70BF006FF3A68FD
:105F800020F00100002AD4BF024640F00102214661
:105F900046480BF0ECFE214644480BF0F6FE3B6809
:105FA000022B20F0040214BF002304231A432146CD
:105FB0003E480BF0DCFE0026E7E61A683B480BF093
:105FC000D6FE0026E1E62021A14041F00401C9B23D
:105FD00020B936480BF0D9FE3860D6E61A68334847
:105FE0000BF0C5FE0026D0E62021A14041F00501BE
:105FF000C9B220B92D480BF0C8FE3860C5E61A6852
:106000002A480BF0B4FE0026BFE61A6827480BF0BA
:10601000AEFE0026B9E62021A14041F00A01C9B236
:1060200020B922480BF0B1FE3860AEE61A681F486E
:106030000BF09DFE0026A8E62021A14041F00301BF
:10604000C9B220B919480BF0A0FE38609DE61A6865
:1060500016480BF08CFE002697E61A6813480BF0E2
:1060600086FE002691E62021A14041F00C01C9B234
:1060700020B90E480BF089FE386086E61A680B4896
:106080000BF075FE002680E62021A14041F01101B1
:10609000C9B220B905480BF078FE386075E61A6879
:1060A00002480BF064FE00266FE600BF7035FF1F4C
:1060B0002021A14041F01201C9B220B9B4480BF02F
:1060C00064FE386061E61A68B1480BF050FE0026A5
:1060D0005BE61A68AE480BF04AFE002655E60C0156
:1060E00044F06C04E4B22146A9482EB90BF04DFEF1
:1060F000C0F38040386048E60BF047FE3B689B04E5
:1061000003F4802320F480221A432146A0480BF098
:106110002EFE002639E6002840F0F5829C4901EB6E
:106120008404E3683B6030E61B68102B3BD00DDC39
:10613000022B34D004DC012B16D04FF0FF3314E0D7
:10614000042B2ED0082BF8D105230EE0402B2CD0A9
:1061500003DC202BF1D1032307E0802B27D0B3F5FC
:10616000807FEAD1002300E008233B603B680133D5
:106170003FF45EAE240144F06C04E4B2214684484E
:106180000BF003FE3B681B0603F0706320F07062A7
:106190001A4321467E480BF0EAFD0026F5E5072369
:1061A000E3E70623E1E70423DFE70223DDE701233A
:1061B000DBE70C0144F06C04E4B2214674482EB9CC
:1061C0000BF0E3FDC0F3C1303860DEE50BF0DDFD20
:1061D0003B68DB0303F4C03320F4C0321A4321468A
:1061E0006B480BF0C4FD0026CFE50C0144F06C04B5
:1061F000E4B2214666482EB90BF0C7FDC0F340302B
:106200003860C2E50BF0C1FD3B685B0303F400534B
:1062100020F400521A4321465D480BF0A8FD0026E9
:10622000B3E50BF0B2FD3B681B0303F4805320F48D
:1062300080521A43214656480BF099FD0026A4E5EA
:106240000D0145F06C05EDB2294651480BF09DFD5E
:106250002946C0F380344E486EB92CB10BF095FD41
:10626000C0F3C310386090E50BF08FFDC0F302104F
:106270003860264689E574B10BF087FD3B68DB0189
:1062800003F4F06320F4F0621A43294640480BF00F
:106290006EFD002679E50BF078FD3A68120220F4D5
:1062A000006002F400620243294639480BF05FFDAA
:1062B000294637480BF069FD3B681B0103F070036A
:1062C00020F070021A43294631480BF050FD264653
:1062D0005BE50D0145F06C05EDB229462C480BF04D
:1062E00054FD2946C0F380342948BEB92CB10BF0C7
:1062F0004CFDC0F30210386047E50BF046FDC0F3DB
:10630000C3103860294622480BF03FFD3B68000A65
:1063100000F0080003433B60264636E574B10BF0FD
:1063200034FD3B681B0103F0700320F070021A4338
:10633000294617480BF01BFD002626E50BF025FD2E
:106340003B68DB0103F4F06320F4F0621A43294652
:106350000F480BF00CFD264617E50BF016FD3B68C9
:1063600020F00F0203F00F031A43214608480BF0F8
:10637000FEFC002609E50C0144F06D04E4B2214660
:1063800003483EB90BF001FDC0F3C0303860FCE4B7
:106390007035FF1F0BF0F9FC3B68DB039BB220F468
:1063A00000421A432146AE480BF0E1FC0026ECE423
:1063B0000C0144F06D04E4B22146A9482EB90BF05B
:1063C000E4FCC0F341303860DFE40BF0DEFC3B68F6
:1063D0005B0303F4C04320F4C0421A432146A048A3
:1063E0000BF0C5FC0026D0E40BF0CFFC3B681B0291
:1063F00003F4706320F470621A43214698480BF04E
:10640000B6FC0026C1E40C0144F06D04E4B2214660
:1064100093482EB90BF0B9FCC0F341103860B4E4D6
:106420000BF0B3FC3B685B0103F0600320F06002FB
:106430001A4321468A480BF09AFC0026A5E40C0179
:1064400044F06D04E4B2214685482EB90BF09DFC62
:1064500000F00F00386098E40BF097FC3B6820F0E8
:106460000F0203F00F031A4321467D480BF07FFC17
:1064700000268AE40BF089FC3B681B0603F080735E
:1064800020F080721A43214675480BF070FC0026FC
:106490007BE40C0144F06D04E4B22146704866B917
:1064A0000BF073FC001400F07F0310F0400018BFE5
:1064B0006FF07F001843386067E40BF066FC3B68C0
:1064C0001B0403F4FE0320F4FE021A432146644831
:1064D0000BF04DFC002658E40C0144F06C04E4B2CF
:1064E00021465F482EB90BF050FCC0F340403860A5
:1064F0004BE40BF04AFC3B685B0403F4003320F4EC
:1065000000321A43214656480BF031FC00263CE489
:10651000202505FA01F14DB245F01404E4B288B922
:1065200021464F480BF031FC10F4806007D045F055
:106530001101C9B24A480BF028FC386025E43860E4
:10654000064622E445F011011A684548C9B20BF02D
:106550000EFC214642480BF018FC3B68002B20F44F
:1065600080620CBF00234FF480631A4321463C48ED
:106570000BF0FDFB002608E42021A14041F01101B1
:10658000C9B228B936480BF000FC3860FFF7FDBBF4
:106590001A6833480BF0EBFB0026FFF7F6BB0BF055
:1065A000F4FB3B685B0303F4005320F400521A43EE
:1065B00021462B480BF0DBFB0026FFF7E6BB00284B
:1065C00040F0A780090141F06F01C9B224480BF0E7
:1065D000DCFBC0F309003860FFF7D7BB0BF0D5FB3D
:1065E0003A681F4821460BF0C2FB0026FFF7CDBBDF
:1065F0002021A14041F01A01C9B228B918480BF076
:10660000C4FB3860FFF7C1BB1A6815480BF0AFFB3D
:106610000026FFF7BABBE8B979B101297FF4B5AB21
:1066200001460F480BF0B1FB00F06000A0F1200321
:10663000584258413860FFF7A8BB09480BF0A5FB4A
:1066400000F01800A0F11002504250413860264678
:10665000FFF79BBB31B1012926D00026FFF795BB80
:106660007035FF1F2C480BF090FB3B68002B14BFCC
:106670000023082320F008021A43214626480BF085
:1066800076FB214624480BF080FB3B68002B20F072
:1066900010020CBF002310231A4321461E480BF0A2
:1066A00066FB2646FFF771BB00211B480BF06DFB14
:1066B0003B68002B0CBF0023202320F020021A434C
:1066C000002115480BF053FB002113480BF05DFB34
:1066D0003B68002B20F0400214BF002340231A43E4
:1066E00000210D480BF043FB0026FFF74EBB0426AC
:1066F000FFF74BBB0426FFF748BB0426FFF745BB5B
:106700000426FFF742BB0426FFF73FBB0426FFF732
:106710003CBB0426FFF739BB7035FF1F07B50129C5
:10672000019207D8024601AB0120FFF7A7F903B099
:106730005DF804FB0820FAE7012910B504460DD1E5
:10674000074A10210BF013FB2046054A18210BF0D5
:106750000EFB0448BDE810400BF05EBB10BD00BF4F
:10676000C80405007035FF1F0129134603D80246EF
:106770000020FFF783B908207047034BD3F8BC32E1
:106780000846DB68114618477035FF1FF8B54B4CBB
:106790004B4D62694B4B4C4F284600210BF01DFBC3
:1067A0004A4928460BF005FCFE68736803F58272BF
:1067B000C5F8A42203F59272C5F8A82203F57172F8
:1067C000C5F8AC2203F5797203F16400C5F8B02274
:1067D00003F2044203F22443C5F8B8323368C5F823
:1067E000B422DB68C5F8A00298473368D5F8AC023C
:1067F000DB6898473368D5F8AC029B6998473368E3
:10680000D5F8A4021B6998473368D5F8A8021B691C
:1068100098473368D5F8B8021B6998473368D5F8AC
:10682000B0021B6998473368D5F8B4021B699847D2
:1068300073683A69C5F8BC2203F531735360636924
:10684000234AC3F80422234AC3F8082201221A70FB
:1068500000225A70204B2362204BE361204BA3613E
:10686000204B6362204BA363204B6363204BA362E6
:10687000204BE362204BA364204B6364204B636591
:10688000204B2365204BE364204B2366204BE365BC
:1068900032224FF48C73C4E902321E4BA3652B687D
:1068A0000220D3F8A020D3F820312074C5F8982214
:1068B000C5F89C32BDE8F840FFF78EB8045AFF1FB8
:1068C0007035FF1F347402003C7A02003967010002
:1068D0005159010045590100315901001D5901006C
:1068E00009590100F5580100696701001D670100A1
:1068F000D5580100B5580100A9580100955801006C
:1069000075580100795901004D580100D95901000D
:10691000695801001D5A010018B9034B5B680B60F0
:1069200070470820704700BF3C38FF1F014B002212
:106930005A607047045AFF1F0428F8B514467FD0E8
:1069400008D801284BD020D3022867D0032834D0A0
:10695000042433E0062800F0A080C0F092800728CD
:1069600000F0A380FC28F3D1584B594DDE68146821
:106970003368D5F8A002002C00F0A380DB689847AC
:106980003368D5F8A0029B6916E0126832F0030361
:1069900040F099804D4B4E4DDE68D5F89402336837
:1069A000D2070DD51B69984724683268D5F8900244
:1069B00014F002040BD01369984700242046F8BD58
:1069C000DB6898473368D5F894029B69EBE7D36896
:1069D00098473368D5F890029B699847EEE71268AC
:1069E00044F620639A426EDC394BD3F8B402374B3D
:1069F000DB6842F210711B688A42CCBF5B699B69FD
:106A00009847226842F2117392FBF3F103FB1121C4
:106A1000304B89B29B6800209847CEE72B4B146817
:106A2000DD68D5E9003000F5F2703CB1DB689847CD
:106A3000D5E900309B6900F5F270BDE79B68CCE7B3
:106A4000224B234EDF6815683B68D6F8A0024DB193
:106A5000012D11D01B6998473B68D6F8A0025B6AEC
:106A6000984707E0DB6898473B689B69D6F8A00227
:106A7000984728462060A0E7DB6898473B685B6939
:106A8000F4E7124B124ADB68D2F8AC021B685B6A6F
:106A90009847003018BF0120ECE70C4B0C4ADB682C
:106AA000D2F8B0021B685B6AF2E7094B1268D3F8B0
:106AB000A802064BDB681B68012A0CBF5B699B6957
:106AC0007AE71B6989E7102478E700BF3C7A020067
:106AD0003C38FF1FDC09FF1F224B70B5DD68224CDC
:106AE0002B68D4F898029B6998472B68D4F8B802B1
:106AF0009B6898472B68D4F8B4029B6898472B682A
:106B0000D4F89C029B6898472B68D4F8A0029B6835
:106B100098472B68D4F8A4029B6898472B68D4F850
:106B200090029B6898472B68D4F894029B6898471A
:106B30002B68D4F8AC029B6898472B68D4F8B00255
:106B40009B6898472B68D4F8A8029B6898472B68E5
:106B5000D4F898029B689847044BBDE870405B6886
:106B6000184700BF3C7A02003C38FF1FDC09FF1FBA
:106B700001480BF0B0BA00BF3C38FF1F0146014886
:106B80000BF053BB3C38FF1F10B5034814460BF005
:106B9000B0FA206010BD00BF3C38FF1F08B50348A5
:106BA000D0F8BC220BF0D0FB002008BD3C38FF1F02
:106BB00008B50348D0F8BC220BF0B2FB002008BD9A
:106BC0003C38FF1F08B502480BF0A7FB002008BDAA
:106BD0003C38FF1F08B502480BF09CFB002008BDA5
:106BE0003C38FF1F08B502480BF092FB002008BD9F
:106BF0003C38FF1F08B502480BF076FB002008BDAB
:106C00003C38FF1F01480BF0F7BA00BF3C38FF1FAC
:106C100038B522210D480D4C0BF06BFA10B9204607
:106C20000BF0D2FA0A4BD4F8B402DD682B689B69EA
:106C300098472B68D4F890021B6998472B68D4F8C2
:106C400094021B699847012038BD00BF3C38FF1FE4
:106C50003C7A0200022804BF0C4B93F8E80038B9D4
:106C60000B4BDB681B685B690A4AD2F8980218472D
:106C7000012809D1054B93F8E830012B04D1044BCE
:106C8000DB681B689B69EFE7704700BF045AFF1F72
:106C90003C7A02003C38FF1F012908B508D1054A9B
:106CA00070210BF018FA0448BDE808400BF066BAF2
:106CB00008BD00BFC80405003C38FF1F8C2970B513
:106CC0000446154600F01A8300F298800E2900F061
:106CD0002F8241D8062900F0B38119D8022900F08B
:106CE0006C8107D8002900F04B81012900F0578101
:106CF00004244BE1042900F07D8140F26C810028DE
:106D000040F097812621BE480BF0F3F928603DE161
:106D10000A2900F0C4810FD8072900F0A9810829A9
:106D2000E6D1002840F00C863521B5480BF0E1F99A
:106D3000C0F34020286029E10C2900F0CA8140F20C
:106D4000BC813421AE48002C40F0DF810BF0D1F93A
:106D500000F00100286019E1152900F03D821FD8DC
:106D6000112900F008820DD80F2900F0EF811029B9
:106D7000BED1002840F0F8812521A1480BF0B9F9D7
:106D8000286003E1132900F0128240F202820028F9
:106D900040F01B822B219A480BF0ABF92860F5E0FC
:106DA0001C2900F05F821AD8182900F035821B29AF
:106DB00000F0408217299BD1924E002840F01A82A1
:106DC00015218F480BF095F930B14FF08073B3FB6C
:106DD000F0F0864228BF06462E600024D6E0212926
:106DE00000F05882222900F06F821D2980D10028EE
:106DF00040F0AF85824B5B681360C7E0B32900F0B9
:106E0000308457D8A82900F0958324D8A42900F00D
:106E1000EB8210D8A22900F0C082A3297FF468AFCA
:106E20006C217748002C40F0D0820BF062F9C0F35F
:106E300080302860AAE0A62900F02C8340F2EC8282
:106E40006C216F48002C40F067830BF052F900F082
:106E50000F0028609AE0AB2900F0AD8310D8A92973
:106E600000F07F83AA297FF443AF6D216448002C92
:106E700040F092830BF03DF9C0F30320286085E0D9
:106E8000AD2900F0C783C0F0AE83AE297FF430AFE8
:106E90006D215B48002C40F0D5830BF02AF90014DB
:106EA00000F07F0310F0400018BF6FF07F00184320
:106EB00028606BE0BB2900F0898436D8B62900F041
:106EC00017841FD8B42900F0E483B5297FF410AFEC
:106ED00034214B48002C40F0E9830BF00AF94305BC
:106EE00040F1E283142146480BF003F9454B30B1E1
:106EF0004FF08072B2FBF0F0834228BF03462B6054
:106F0000002443E0B92900F0248400F23A84B8292F
:106F10007FF4EEAE6C213A48002C40F00B840BF06D
:106F2000E8F8C0F34030286030E0CC2900F0C88495
:106F300012D8BF2900F08084C02900F09D84BC29AC
:106F40007FF4D6AE70212E48002C40F068840BF000
:106F5000D0F8C0B2286019E0D12900F0CB84D22942
:106F600000F0D884CE297FF4C3AE002840F0F78427
:106F70006F2123480BF0BDF8C0F30900286005E03D
:106F800030B92D211E480BF0B4F82860204670BDA2
:106F900012681B482D210BF09EF80024F6E728B953
:106FA000212117480BF0A5F82860EFE71268144874
:106FB00021210BF090F80024E8E728B92721104898
:106FC0000BF097F82860E1E712680D4827210BF0D5
:106FD00082F80024DAE7002840F0AC842221084837
:106FE0000BF087F810F4000318BF4FF07F431843ED
:106FF0002860CBE7024E38B9D6F8BC321360C5E73B
:107000003C38FF1FFFFF0F001368A748002BB8BFD5
:107010005B422021C6F8BC320BF06BF80446002816
:1070200040F08B84D6F8BC229F4827210BF053F800
:10703000ACE712689C4826210BF04DF80024A5E728
:10704000102199482CB90BF054F8C0F304202860A3
:107050009CE70BF04EF82B681B0203F4F85320F466
:10706000F8521A43102190480BF035F800248DE7B0
:1070700010218D482CB90BF03CF800F01F0028605F
:1070800084E70BF036F82B6820F01F0203F01F0393
:107090001A43102184480BF01EF8002476E70028DC
:1070A00040F05184352180480BF023F810F0020F96
:1070B0000CBF012300232B6068E7002840F04684C2
:1070C000352179480BF015F8C04300F00100286025
:1070D0005CE7342174482CB90BF00BF8C0F3400086
:1070E000286053E70BF005F82C6834B940F0020231
:1070F00034216D480AF0EFFF48E720F00202342106
:1071000069480AF0E8FF002440E70AF0F2FF2C6823
:1071100034B940F00102342163480AF0DCFF35E75E
:1071200020F00102342160480AF0D5FF00242DE749
:1071300028B934215C480AF0DCFF286026E7126891
:10714000594834210AF0C7FF00241FE728B9242139
:1071500055480AF0CEFF286018E7126852482421EB
:107160000AF0B9FF002411E712684F4825210AF000
:10717000B2FF00240AE728B928214B480AF0B9FFDA
:10718000286003E71268484828210AF0A4FF002479
:10719000FCE628B92A2144480AF0ABFF2860F5E64E
:1071A000126841482A210AF096FF0024EEE628B929
:1071B00023213D480AF09DFF2860E7E612683A481F
:1071C00023210AF088FF0024E0E6126836482B21CC
:1071D0000AF081FF0024D9E628B92C2132480AF0B0
:1071E00088FF2860D2E612682F482C210AF073FF2E
:1071F0000024CBE613686BB14FF0807292FBF3F280
:10720000B242A8BF32462A60152127480AF063FF20
:107210000024BBE63246F6E728B9332122480AF0BB
:1072200068FF2860B2E612681F4833210AF053FF56
:107230000024ABE66C211C482CB90AF05AFFC0F3BD
:10724000C0402860A2E60AF054FF2B68DB0403F478
:10725000002320F400221A436C2113480AF03BFF5C
:10726000002493E66C2110482CB90AF042FFC0F3C9
:10727000804028608AE60AF03CFF2B689B0403F4F8
:10728000802320F480221A436C2107480AF023FF50
:1072900000247BE60021044844B90AF02AFF00F0EC
:1072A0000100286072E600BF3C38FF1F0AF021FF92
:1072B0002B6820F0010203F001031A430021B548B6
:1072C0000AF009FF002461E638B90146B1480AF026
:1072D00010FFC0F34000286058E60021AD480AF0D6
:1072E00008FF2B685B0003F0020320F002021A4340
:1072F0000021A8480AF0EFFE002447E658B96C21A7
:10730000A4480AF0F6FE4FF48073C0F3036043FA1A
:1073100000F028603AE61368102B27D00DDC022B12
:1073200020D004DC012B16D04FF0FF3314E0042BE7
:107330001AD0082BF8D105230EE0402B18D003DC1F
:10734000202BF1D1032307E0802B13D0B3F5807FEE
:10735000EAD1002300E008232B602B6801330BD116
:10736000102413E60723F7E70623F5E70423F3E7E2
:107370000223F1E70123EFE76C2186480AF0B9FE0A
:107380002B681B0603F0706320F070621A436C21B7
:1073900080480AF0A0FE0024F8E56C217D482CB955
:1073A0000AF0A7FEC0F3C1302860EFE50AF0A1FEA5
:1073B0002B68DB0303F4C03320F4C0321A436C2182
:1073C00074480AF088FE0024E0E50AF092FE2B687B
:1073D0009B0303F4804320F480421A436C216D48E0
:1073E0000AF079FE0024D1E56C216A482CB90AF034
:1073F00080FEC0F300302860C8E50AF07AFE2B68F2
:107400001B0303F4805320F480521A436C2161481B
:107410000AF061FE0024B9E56C215E480AF069FEBD
:1074200000F4804394B93BB16C215A480AF061FEE4
:10743000C0F3C3102860A9E5C0F3021300F4006094
:1074400003430CBF002308232B609FE583B16C210D
:1074500050480AF04EFE2B68DB0103F4F06320F481
:10746000F0621A436C214B480AF035FE00248DE58A
:107470002A6811074CBF40F4006020F4006012013C
:1074800020F07000D2B202436C2142480AF023FE81
:1074900000247BE56C213F480AF02BFEACB910F4C8
:1074A000804307D06C213B480AF023FEC0F3021052
:1074B00028606BE5C0F3C31200F4006002430CBF08
:1074C000002208222A601C4660E56C2131480AF03F
:1074D00010FE10F480444FF06C012E480ED00AF0DC
:1074E00008FE2B681B0103F0700320F070021A43A2
:1074F0006C2128480AF0EFFD002447E50AF0F9FD69
:107500002B68DB0103F4F06320F4F0621A436C2172
:1075100020480AF0E0FD39E50AF0EBFD2B6820F089
:107520000F0203F00F031A436C211A480AF0D3FD2F
:1075300000242BE56D2117482CB90AF0DAFDC0F3C1
:10754000C030286022E50AF0D4FD2B68DB039BB233
:1075500020F400421A436D210E480AF0BCFD0024BD
:1075600014E56D210B482CB90AF0C3FDC0F341307E
:1075700028600BE50AF0BDFD2B685B0303F4C043F4
:1075800020F4C0421A436D2102480AF0A4FD0024F1
:10759000FCE400BF3C38FF1F0AF0ABFD2B681B0268
:1075A00003F4706320F470621A436D21B7480AF047
:1075B00092FD0024EAE46D21B4482CB90AF099FD4B
:1075C000C0F341102860E1E40AF093FD2B685B01F1
:1075D00003F0600320F060021A436D21AB480AF00B
:1075E0007AFD0024D2E46D21A8482CB90AF081FD6F
:1075F00000F00F002860C9E40AF07BFD2B6820F042
:107600000F0203F00F031A436D21A0480AF063FD37
:107610000024BBE46D219D482CB90AF06AFDC0F33B
:1076200000602860B2E40AF064FD2B681B0603F0DA
:10763000807320F080721A436D2194480AF04BFD4C
:107640000024A3E40AF055FD2B681B0403F4FE0399
:1076500020F4FE021A436D218C480AF03CFD002400
:1076600094E46C2189482CB90AF043FDC0F34040F2
:1076700028608BE40AF03DFD2B685B0403F40033C3
:1076800020F400321A436C2180480AF024FD0024C3
:107690007CE4002840F060816F217C480AF029FDDD
:1076A000C0F30440286071E42C606FE40AF021FD0F
:1076B0002B68002B0CBF00234FF4806320F4806202
:1076C0001A43342171480AF006FD2968704B69B1EC
:1076D0004FF0807292FBF1F29A42A8BF1A462A60DC
:1076E00014216A480AF0F7FC00244FE41A46F6E732
:1076F000674E70B9142165480AF0FBFC30B14FF0B9
:107700008072B2FBF0F2964228BF16462E6000242B
:107710003CE4136863B14FF0807292FBF3F2B24223
:10772000A8BF3246142159480AF0D5FC00242DE4A4
:107730003246F7E70AF0DDFC2B685B0303F40053E5
:1077400020F400521A436C2150480AF0C4FC002473
:107750001CE46C214D482CB90AF0CBFCC0F303505B
:10776000286013E40AF0C5FC2B681B0503F47003C2
:1077700020F470021A436C2144480AF0ACFC002447
:1077800004E4434E78B9132140480AF0B2FC30B10A
:107790004FF08073B3FBF0F0864228BF06462E60A0
:1077A0000024FFF7F3BB136873B14FF0807292FBB4
:1077B000F3F2B242A8BF32462A60132133480AF0DE
:1077C0008AFC0024FFF7E2BB3246F5E770212F4820
:1077D00034B90AF08EFCC0F307202860FFF7D6BB4F
:1077E0000AF087FC2A68120220F47F4092B202431A
:1077F000702126480AF06FFC002124480AF079FC29
:107800002B68002B20F004020CBF002304231A4332
:1078100000211E480AF05FFC0024FFF7B7BB0AF006
:1078200068FC2A7820F0FF000243702117480AF014
:1078300052FC0024FFF7AABB40B9702113480AF09C
:1078400058FCC0F301402860FFF7A0BB1368032B6E
:107850003FF686AD70210D480AF04BFC2B681B04E7
:1078600003F4403320F440321A43702107480AF0F1
:1078700032FC0024FFF78ABB60B9702103480AF08C
:1078800038FCC0F380402860FFF780BB3C38FF1F06
:10789000FFFF0F001368012B3FF662AD70213148E6
:1078A0000AF027FC2B689B0403F4802320F4802239
:1078B0001A4370212B480AF00EFC0024FFF766BB28
:1078C0007021284834B90AF014FCC0F30150286034
:1078D000FFF75CBB0AF00DFC2B681B0503F440139B
:1078E00020F440121A4370211E480AF0F4FB0024D1
:1078F000FFF74CBB30B939211A480AF0FAFB28606F
:10790000FFF744BB1268174839210AF0E4FB002452
:10791000FFF73CBB30B93A2112480AF0EAFB286075
:10792000FFF734BB12680F483A210AF0D4FB002459
:10793000FFF72CBB0424FFF729BB0024FFF726BB6D
:107940000424FFF723BB0424FFF720BB0424FFF724
:107950001DBB0424FFF71ABB0424FFF717BB042444
:10796000FFF714BB3C38FF1F07B5019239B9014638
:1079700001AA0120FFF7A2F903B05DF804FB08207B
:10798000FAE70B4619B901461846FFF797B90820E0
:107990007047034BD3F8C0320846DB6811461847DE
:1079A0003C38FF1F70B5644E644CF5686B6803F19A
:1079B0006402C4F8982203F1A402C4F89C2203F1E3
:1079C000C402C4F8A02203F59272C4F8902203F511
:1079D000A272C4F8942203F5D272C4F8B42203F55B
:1079E000E272C4F8B82203F5617203F18400C4F8AE
:1079F000A82203F5697203F57173C4F8AC322B68E1
:107A0000C4F8B0221B69C4F8A40298472B68D4F8C4
:107A1000A0021B6998472B68D4F89C021B69984701
:107A20002B68D4F8AC021B6998472B68D4F8B002D5
:107A30001B6998472B68D4F8A802DB6898472B6825
:107A4000D4F890021B6998472B68D4F894021B69FC
:107A500098472B68D4F89802DB6898472B68D4F8CD
:107A6000B402DB6898472B68D4F8B802DB68984703
:107A70002B68D4F8A8029B6998476B683269C4F8F0
:107A8000C02203F5317353602D4B2E495A692E489D
:107A9000C2F804122D49C2F8081200260121117003
:107AA000567018622A48D8612A4898612A48586254
:107AB0002A4898632A4858632A4898622A48D86214
:107AC0002A4898642A4858642A4858652A481865FC
:107AD0002A48D8642A4818662A48D865197432207A
:107AE0004FF4F071C3E90210274999652046274BEE
:107AF00031460AF026FB264920460AF092FB23680D
:107B00000220D3F8A030C4F8BC32FFF7A3F82B68EA
:107B1000D4F8B802DB689847D4F8B8021D4C0423A7
:107B200043752B681B68984723689847A3683146BC
:107B30003046BDE8704018473C7A02003C38FF1FD1
:107B4000045AFF1F116C0100F56B0100056C010068
:107B5000E56B0100D56B0100C56B01008379010065
:107B600069790100B16B01009D6B0100716B01002F
:107B7000896B01007D6B0100396901001969010001
:107B8000556C01002D690100D96A010034760200AC
:107B9000996C0100DC09FF1F18B9034B1B680B60CF
:107BA00070470820704700BF0C3BFF1F014B0022AD
:107BB0005A607047045AFF1F234B70B5DD68234C91
:107BC0002B68D4F898029B6998472B68D4F8A802D0
:107BD0009B6998472B68D4F8AC029B6998472B683F
:107BE000D4F89C029B6898472B68D4F8A0029B6845
:107BF00098472B68D4F8A4029B6898472B68D4F860
:107C000090029B6898472B68D4F894029B68984729
:107C10002B68D4F8B0029B6898472B68D4F8B4025C
:107C20009B6898472B68D4F898029B6898472B6804
:107C3000D4F8A8029B6898472B68D4F8AC029B68DC
:107C4000BDE87040184700BF3C7A02000C3BFF1FA4
:107C5000034A0146D2F8B83200200AF0BCBB00BF8C
:107C60000C3BFF1F024BD3F8B8020AF0EEBB00BF7B
:107C70000C3BFF1F38B5284D00F07F042B1993F8FB
:107C80000C32DB0705D4D5F8B83203EB8404606806
:107C900038BDD5F8BC3200219B6820469847D5F8FE
:107CA000BC3200219B6808469847D5F8BC320021B9
:107CB0009B6808469847D5F8BC3200219B68084667
:107CC0009847D5F8BC3201219B6800209847D5F829
:107CD000BC3200219B6820469847D5F8BC32002171
:107CE0009B6808469847D5F8BC32002104029B687F
:107CF00008469847D5F8BC32002104439B680846E3
:107D00009847D5F8BC32240204439B680121002027
:107D1000984724022043BBE70C3BFF1F022804BF07
:107D20000C4B93F8E80038B90B4BDB681B685B69B8
:107D30000A4AD2F898021847012809D1054B93F84E
:107D4000E830012B04D1044BDB681B689B69EFE72B
:107D5000704700BF045AFF1F3C7A02000C3BFF1F14
:107D6000012870B506460F4D0F4C07D1EB6AC4F8D9
:107D7000C0325B68984784F8C46270BD94F8C4321E
:107D8000012B03D1D4F8C0329B689847EB682A696D
:107D90005B68C4F8BC2203F531735360002384F898
:107DA000C432EAE73C7A02000C3BFF1F0528F8B515
:107DB0000C46154600F0A6801FD802286BD003D8C9
:107DC00000283ED0042455E0032876D00428F9D1B9
:107DD000614B624EDF6814683B68D6F8A002002C45
:107DE00000F08180012C00F088801B6998473B6877
:107DF000D6F8A0025B6A98477DE0082800F08E80E4
:107E000009D80628DED1544B544ADB68D2F8B402B4
:107E10001B685B6A7DE0092800F08980FC28D1D1CD
:107E20004D4B4E4EDF6814683B68D6F8A002002C1C
:107E300000F08D80DB6898473B68D6F8A0029B690C
:107E400016E0126832F0030340F08380424B434E49
:107E5000DF68D6F894023B68D2070DD51B699847B6
:107E60002C683B68D6F8900214F002040BD01B6912
:107E7000984700242046F8BDDB6898473B68D6F851
:107E800094029B69EBE7DB6898473B68D6F8900261
:107E90009B699847EEE7304B1468DE68D6E90030FE
:107EA00000F5F2703CB1DB689847D6E900309B6979
:107EB00000F5F270DCE79B68EBE7284BD3F8A802EB
:107EC000254BDB681B6839B1146814F0010401D03C
:107ED0005B69CDE79B69DCE75B6A9847003018BFB8
:107EE00001202860C6E7DB6898473B689B69D6F8A5
:107EF000A002984720462860BBE7DB6898473B68AC
:107F00005B69F4E7144B154ADB68D2F8B0021B68D2
:107F10005B6A9847003018BF0120ECE710680F4BF0
:107F200000F0010083F8C502FFF71AFFA1E70A4B32
:107F30001268DC68D4E90030012A00F5F27004D13F
:107F4000DB689847D4E90030B1E79B6890E71B698C
:107F50009FE710248EE700BF3C7A02000C3BFF1F16
:107F60007FB52C4B00F07F041A191D4692F80C22A5
:107F700012F0010F06D1D3F8B83203EB8404606825
:107F800004B070BD01220523032101A8ADF804301F
:107F90008DF8064006F0B4FBD5F8C0328DF8070026
:107FA000DB699847D5F8C03204215B690DEB01000D
:107FB000984702F03DFF0646D5F8C0321B6A984745
:107FC00007281FD9D5F8C03208219B690DEB0100A5
:107FD00098470122072102A89DF80F5006F090FB58
:107FE000854214D19DF80830052B10D19DF8093039
:107FF000FF2B0CD19DF80A30A34208D1DDF80B000D
:1080000000BABDE7304602F023FF3228D4D94FF042
:10801000FF30B5E70C3BFF1F024B93F8C53203B1AD
:108020009EE727E60C3BFF1F38B52220FFF7F4FF41
:10803000094C18B9D4F8B8020AF0FEF9074BD4F885
:108040009002DD682B681B6998472B68D4F894026E
:108050001B699847012038BD0C3BFF1F3C7A02008A
:1080600010B508461446FFF7D7FF206010BD2DE974
:10807000F74F354D9DF8304095F8C5629DF8347046
:1080800001F07F0990469A4649F08000AB469EB3C6
:1080900005238DF802008DF8032007210122684690
:1080A000ADF800308DF804A08DF805408DF806700D
:1080B00006F026FBD5F8C0328DF80700DB6998473B
:1080C0000025DBF8C0321DF80500DB680135984754
:1080D000082DF6D1022002F0B1FE47EA0424DBF8B5
:1080E000B83244EA0A4403EB890944EA0864C9F84F
:1080F000044003B0BDE8F08FD5F8BC3231469B6830
:108100009847D5F8BC3231469B6840469847D5F829
:10811000BC3231469B6850469847D5F8BC32314650
:108120009B6820469847D5F8BC3201219B683846A9
:1081300098474AEA082344EA0324D5F8B83247EAC4
:10814000042403EB8909D2E70C3BFF1F07B5D3B228
:108150000193C2F307230093C2F30743120EFFF704
:1081600086FF03B05DF804FB0020FFF7EFBF73B597
:108170000D460646E8B9104C94F8C63243B1D4F81F
:10818000B8322721D3F8A020FFF7E0FF84F8C662B9
:1081900000242A462D210020FFF7D8FF2046CDE9F4
:1081A0000044234622462021FFF761FF204602B00B
:1081B00070BD0820FBE700BF0C3BFF1F38B50C4625
:1081C00005462120FFF728FF2368C11821602846B3
:1081D000BDE83840CBE737B50D460446C8B90E4B6D
:1081E000012283F8C62281EAE172A2EBE172272123
:1081F000FFF7ACFF002DACBF01230223CDE9004304
:108200002046234622462021FFF731FF204603B0B7
:1082100030BD0820FBE700BF0C3BFF1F0021DAE761
:108220004942D8E7D7E7222970B50446154600F041
:10823000D88200F286800E2900F003823ED80629FB
:1082400000F0958118D8022900F04B8107D8002949
:1082500000F02C81012900F0378104242BE104294E
:1082600000F0618140F25181002840F079812620A0
:10827000FFF7D2FE28601EE10A2900F0A5810ED882
:10828000072900F08B810829E7D1002840F0B1854B
:108290003520FFF7C1FEC0F3402028600BE10C2918
:1082A00000F0AA8140F29D813420002C40F0BB8177
:1082B000FFF7B2FE00F001002860FCE0152900F095
:1082C0000F821DD8112900F0DD810CD80F2900F094
:1082D000C5811029C1D1002840F0CD812520FFF7AC
:1082E0009BFE2860E7E0132900F0E68140F2D78189
:1082F000002840F0EE812B20FFF78EFE2860DAE0A8
:108300001B2900F02A820CD8172900F0FB811829BC
:10831000A3D1002840F01A823320FFF77DFE2860A9
:10832000C9E01D2900F04782C0F02E82212994D196
:10833000002840F04782FFF76FFE00F00100286040
:10834000B9E0AE2900F0F7834FD8A72900F0658384
:1083500028D8A32900F0B8820FD88C2900F05882C1
:10836000A2297FF47AAF6C20002C40F09E82FFF7A8
:1083700053FEC0F3C13028609DE0A52900F0D282F1
:1083800040F2B9826C20FFF747FE00F48046002CD3
:1083900040F01F83002E00F01183000900F07000F0
:1083A000286088E0AA2900F073830FD8A82900F07C
:1083B0004A83A9297FF451AF6D20002C40F05983E6
:1083C000FFF72AFEC0F34130286074E0AC2900F0CA
:1083D0008D8340F274836D20002C40F09D83FFF765
:1083E0001BFEC0F30060286065E0BB2900F05984E3
:1083F00033D8B62900F0EB831DD8B42900F0B98337
:10840000B5297FF42AAF3420002C40F0BE83FFF75B
:1084100003FE430540F1B7831420FFF7FDFDB74B82
:1084200030B14FF08072B2FBF0F0834228BF0346B8
:108430002B6000243FE0B92900F0FA8300F20F849A
:10844000B8297FF40AAF6C20002C40F0E283FFF7DC
:10845000E3FDC0F3403028602DE0CC2900F08F848C
:1084600011D8BF2900F04F84C02900F06A84BC29CC
:108470007FF4F3AE7020002C40F03884FFF7CCFD81
:10848000C0B2286017E0D12900F09284D22900F010
:108490009E84CE297FF4E1AE002840F0B9846F209D
:1084A000FFF7BAFDC0F30900286004E028B92D20C9
:1084B000FFF7B2FD2860204670BD12682D21002014
:1084C000FFF744FE0024F6E720B92120FFF7A4FDC2
:1084D0002860F0E7126821210020FFF737FE002412
:1084E000E9E720B92720FFF797FD2860E3E7126846
:1084F000002AB8BF524227210020FFF727FE804BF9
:10850000012283F8C6220024D5E7002840F06E84BB
:108510002220FFF781FD10F4000318BF4FF07F43C6
:1085200018432860C7E7764BD3F8B82218B9D2F8B9
:10853000A0302B60BFE72B68002BB8BF5B42C2F8AE
:10854000A0302020FFF768FD044608B10024B2E700
:108550002A68002AB8BF52422721FFF7F7FDAAE791
:10856000126826210020FFF7F1FD0024A3E7102068
:108570002CB9FFF751FDC0F3042028609BE7FFF7FB
:108580004BFD2B681B0203F4F85320F4F8521A43F6
:1085900010210020FFF7DAFD00248CE710202CB911
:1085A000FFF73AFD00F01F00286084E7FFF734FD75
:1085B0002B6820F01F0203F01F031A431021002034
:1085C000FFF7C4FD002476E7002840F0158435202D
:1085D000FFF722FD10F0020F0CBF012300232B60D8
:1085E00069E7002840F00B843520FFF715FDC043F4
:1085F00000F0010028605EE734202CB9FFF70CFD85
:10860000C0F34000286056E7FFF706FD2B685B00CB
:1086100003F0020320F002021A4334210020FFF786
:1086200095FD002447E7FFF7F7FC2B6820F00102D7
:1086300003F001031A4334210020FFF787FD0024D3
:1086400039E720B93420FFF7E7FC286033E71268E8
:1086500034210020FFF77AFD00242CE720B92420E4
:10866000FFF7DAFC286026E7126824210020FFF7D4
:108670006DFD00241FE7126825210020FFF766FD2D
:10868000002418E720B92820FFF7C6FC286012E76D
:10869000126828210020FFF759FD00240BE720B9BC
:1086A0002A20FFF7B9FC286005E712682A2100207C
:1086B000FFF74CFD0024FEE620B92320FFF7ACFCB9
:1086C0002860F8E6126823210020FFF73FFD002410
:1086D000F1E612682B210020FFF738FD0024EAE6BE
:1086E00020B92C20FFF798FC2860E4E612682C21C2
:1086F0000020FFF72BFD0024DDE600BFFFFF0F0089
:108700000C3BFF1FBB4E78B91520FFF785FC48B125
:108710004FF08073B3FBF0F0B04288BF3046286062
:108720000024C8E6B348FAE713686BB14FF08072D3
:1087300092FBF3F2B242A8BF32462A601521002014
:10874000FFF704FD0024B6E6AA4AF6E712683321D3
:108750000020FFF7FBFC0024ADE66C202CB9FFF7EE
:108760005BFCC0F3C0402860A5E6FFF755FC2B6812
:10877000DB0403F4002320F400221A436C210020C0
:10878000FFF7E4FC002496E66C202CB9FFF744FCCC
:10879000C0F3804028608EE6FFF73EFC2B689B0408
:1087A00003F4802320F480221A436C210020FFF779
:1087B000CDFC00247FE6002840F024838E4B1B680C
:1087C000136078E60020FFF727FC2B6820F00102F9
:1087D00003F0010300211A430846FFF7B7FC002409
:1087E00069E628B9FFF718FCC0F34000286062E68C
:1087F0000020FFF711FC2B685B0003F0020320F060
:10880000020200211A430846FFF7A0FC002452E6AA
:1088100050B96C20FFF700FC4FF48073C0F3036085
:1088200043FA00F0286046E61368102B27D00DDCD1
:10883000022B20D004DC012B16D04FF0FF3314E0C4
:10884000042B1AD0082BF8D105230EE0402B18D0AA
:1088500003DC202BF1D1032307E0802B13D0B3F5E9
:10886000807FEAD1002300E008232B602B680133CE
:108870000BD110241FE60723F7E70623F5E70423AF
:10888000F3E70223F1E70123EFE76C20FFF7C4FBD6
:108890002B681B0603F0706320F070621A436C2192
:1088A0000020FFF753FC002405E6FFF7B5FB2B681B
:1088B000DB0303F4C03320F4C0321A436C210020E0
:1088C000FFF744FC0024F6E56C202CB9FFF7A4FB6D
:1088D000C0F380302860EEE5FFF79EFB2B689B031A
:1088E00003F4804320F480421A436C210020FFF7F8
:1088F0002DFC0024DFE56C202CB9FFF78DFBC0F3C5
:1089000000302860D7E5FFF787FB2B681B0303F4D3
:10891000805320F480521A436C210020FFF716FC8C
:108920000024C8E56C20FFF777FB0646C4B910F4B5
:10893000804405D0C60906F4F0662E600024BAE52E
:108940006C20FFF769FB16F00B0F4FEA201000F0C8
:10895000700001D12860F9E540F008002860AAE520
:108960006C20FFF759FB10F480444FF06C000ED0E0
:10897000FFF752FB2B68DB0103F4F06320F4F06295
:108980001A436C210020FFF7E1FB002493E5FFF779
:1089900043FB6C2120F400622046FFF7D7FB6C20DC
:1089A000FFF73AFB2B681B0103F0700320F0700205
:1089B0001A436C212046FFF7C9FB7CE5C309020579
:1089C00003F4F06301D42B60C0E543F008032B608F
:1089D00071E56C2096B1FFF71FFB2B681B0103F0BC
:1089E000700320F070021A436C210020FFF7AEFBE9
:1089F000002460E5FFFF0F000C3BFF1FFFF70CFB9F
:108A00002B68DB0103F4F06320F4F0621A436C215D
:108A10003046FFF79BFB34464DE56C202CB9FFF741
:108A2000FBFA00F00F00286045E5FFF7F5FA2B6828
:108A300020F00F0203F00F031A436C210020FFF710
:108A400085FB002437E56D202CB9FFF7E5FAC0F36C
:108A5000C03028602FE5FFF7DFFA2B68DB039BB2FD
:108A600020F400421A436D210020FFF76FFB002421
:108A700021E5FFF7D1FA2B685B0303F4C04320F430
:108A8000C0421A436D210020FFF760FB002412E56D
:108A90006D202CB9FFF7C0FAC0F3032028600AE567
:108AA000FFF7BAFA2B681B0203F4706320F47062BC
:108AB0001A436D210020FFF749FB0024FBE46D20E1
:108AC0002CB9FFF7A9FAC0F341102860F3E4FFF7CF
:108AD000A3FA2B685B0103F0600320F060021A43E5
:108AE0006D210020FFF732FB0024E4E46D202CB957
:108AF000FFF792FA00F00F002860DCE4FFF78CFA31
:108B00002B6820F00F0203F00F031A436D210020A1
:108B1000FFF71CFB0024CEE4FFF77EFA2B681B0650
:108B200003F0807320F080721A436D210020FFF75C
:108B30000DFB0024BFE46D2064B9FFF76DFA00144B
:108B400000F07F0310F0400018BF6FF07F00184363
:108B50002860B0E4FFF760FA2B681B0403F4FE03FF
:108B600020F4FE021A436D210020FFF7EFFA0024E3
:108B7000A1E4002840F049816F20FFF74DFAC0F3CF
:108B80000440286097E42C6095E4FFF745FA2B68D1
:108B9000002B0CBF00234FF4806320F480621A4343
:108BA00034210020FFF7D2FA29689B4B69B14FF0BE
:108BB000807292FBF1F29A42A8BF1A462A601421F1
:108BC0000020FFF7C3FA002475E41A46F6E7924E38
:108BD00068B91420FFF720FA30B14FF08073B3FB6F
:108BE000F0F0864228BF06462E60002463E4136836
:108BF0006BB14FF0807292FBF3F2B242A8BF3246E3
:108C00002A6014210020FFF7A1FA002453E4324621
:108C1000F6E7FFF701FA2B685B0303F4005320F437
:108C200000521A436C210020FFF790FA002442E41E
:108C30006C202CB9FFF7F0F9C0F3035028603AE438
:108C4000FFF7EAF92B681B0520F4700203F47003A8
:108C50001A436C210020FFF779FA00242BE46E4EB2
:108C600068B91320FFF7D8F930B14FF08073B3FB28
:108C7000F0F0864228BF06462E6000241BE41368ED
:108C80006BB14FF0807292FBF3F2B242A8BF324652
:108C90002A6013210020FFF759FA00240BE4324622
:108CA000F6E770202CB9FFF7B7F9C0F3072028606A
:108CB00001E4FFF7B1F92A68120220F47F4092B272
:108CC000024370210020FFF741FA0020FFF7A4F9CA
:108CD0002B689B0003F0040320F0040200211A43D8
:108CE0000846FFF733FA0024FFF7E5BBFFF794F9D6
:108CF0002A7820F0FF00024370210020FFF726FAB7
:108D00000024FFF7D8BB38B97020FFF785F9C0F30E
:108D100001402860FFF7CFBB1368032B3FF6A9ADD6
:108D20007020FFF779F92B681B0403F4403320F41B
:108D300040321A4370210020FFF708FA0024FFF7A1
:108D4000BABB38B97020FFF767F9C0F380402860DC
:108D5000FFF7B1BB1368012B3FF68BAD7020FFF717
:108D60005BF92B689B0403F4802320F480221A43D0
:108D700070210020FFF7EAF90024FFF79CBB702068
:108D800034B9FFF749F9C0F301502860FFF793BBEE
:108D9000FFF742F92B681B0503F4401320F440123F
:108DA0001A4370210020FFF7D1F90024FFF783BB9D
:108DB00028B93920FFF730F92860FFF77CBB12682B
:108DC00039210020FFF7C2F90024FFF774BB28B94E
:108DD0003A20FFF721F92860FFF76DBB12683A21AE
:108DE0000020FFF7B3F90024FFF765BB0424FFF769
:108DF00062BB0424FFF75FBB0424FFF75CBB0424C1
:108E0000FFF759BB0424FFF756BB0424FFF753BBFD
:108E10000424FFF750BB00BFFFFF0F0007B501920E
:108E200039B9014601AA0120FFF7FDF903B05DF849
:108E300004FB0820FAE70B4619B901461846FFF76C
:108E4000F2B908207047044B93F8C53208460BB1BD
:108E5000FFF786B8FEF70EBF0C3BFF1F38B5554C29
:108E6000204609F081FA544BDD686B6803F18402F7
:108E7000C4F8A42203F1A402C4F89C2203F1C402A2
:108E8000C4F8A02203F59272C4F8902203F5A272EE
:108E9000C4F8942203F5C272C4F8A82203F5E27262
:108EA00003F16400C4F8AC2203F5697203F5717331
:108EB000C4F8B0322B68C4F8B422DB68C4F8980256
:108EC00098472B68D4F8A802DB6898472B68D4F839
:108ED000AC02DB6898472B68D4F898025B69984726
:108EE0002B68D4F8A8029B6998472B68D4F8AC0289
:108EF0005B6998472B68D4F8A4021B6998472B68D4
:108F0000D4F8A0021B6998472B68D4F89C021B690F
:108F100098472B68D4F8B0021B6998472B68D4F89F
:108F2000B4021B6998472B68D4F890021B699847D4
:108F30002B68D4F894021B69984794F8C502FEF791
:108F40000FFF1E4B1E495A69C4F8B822C2F804121A
:108F50001C49C2F8081200200121507011701A4AF1
:108F60001A621A4ADA611A4A9A611A4A5A621A4A03
:108F70009A631A4A5A631A4A9A621A4ADA621A4A6F
:108F80009A641A4A5A641A4A5A651A4A1A651A4A57
:108F9000DA641A4A1A661A4ADA6519744FF42572A5
:108FA0003221C3E90221174A9A650220BDE8384000
:108FB000FEF7B4BE0C3BFF1F3C7A0200045AFF1FB1
:108FC00029800100657C0100D78101002582010014
:108FD000218201001D820100378E01001D8E0100DB
:108FE0006F810100BD810100698101006180010084
:108FF000517C0100AD7D0100997B01001D7D0100C8
:10900000AD7B0100B97B010018B9034B5B680B60B5
:1090100070470820704700BFE03DFF1F014B002252
:109020005A607047045AFF1F0428F8B50C461546CD
:1090300070D005D8022845D056D8C8B1042430E0F5
:10904000062800F09480C0F08680FC28F6D14E4BB4
:109050004E4EDF6814683B68D6F8A002002C00F082
:109060008E80DB6898473B68D6F8A0029B6916E0C3
:10907000126832F0030340F08480434B434EDF68B4
:10908000D6F894023B68D2070DD51B6998472C6827
:109090003B68D6F8900214F002040BD01B69984785
:1090A00000242046F8BDDB6898473B68D6F8940258
:1090B0009B69EBE7DB6898473B68D6F890029B69B1
:1090C0009847EEE7304B1468DE68D6E9003000F5CB
:1090D000F2703CB1DB689847D6E900309B6900F537
:1090E000F270DCE79B68EBE7284BD3F8A802264B2D
:1090F000DB681B6839B1146814F0010401D05B69A6
:10910000CDE79B69DCE75B6A9847003018BF012018
:109110002860C6E71C4B1D4EDF6814683B68D6F814
:10912000A0024CB1012C11D01B6998473B68D6F8BE
:10913000A0025B6A984707E0DB6898473B689B6939
:10914000D6F8A002984720462860A9E7DB68984730
:109150003B685B69F4E70C4B0C4ADB68D2F8B00261
:109160001B685B6A9847003018BF0120ECE7064B8C
:10917000064ADB68D2F8B4021B685B6AF2E71B6937
:109180009EE710248DE700BF3C7A0200E03DFF1F00
:10919000234B70B5DD68234C2B68D4F898029B698B
:1091A00098472B68D4F8A8029B6998472B68D4F895
:1091B000AC029B6998472B68D4F89C029B6898473F
:1091C0002B68D4F8A0029B6898472B68D4F8A402B7
:1091D0009B6898472B68D4F890029B6898472B6847
:1091E000D4F894029B6898472B68D4F8B0029B6827
:1091F00098472B68D4F8B4029B6898472B68D4F83A
:1092000098029B6898472B68D4F8A8029B689847F7
:109210002B68D4F8AC029B68BDE87040184700BFCB
:109220003C7A0200E03DFF1F0146014809F09AB96F
:10923000E03DFF1F10B50348144609F050F92060C7
:1092400010BD00BFE03DFF1F014809F03AB900BF63
:10925000E03DFF1F08B50348D0F8B82209F040FAF6
:10926000002008BDE03DFF1F08B50348D0F8B82234
:1092700009F022FA002008BDE03DFF1F08B50248B2
:1092800009F017FA002008BDE03DFF1F08B50248AD
:1092900009F00CFA002008BDE03DFF1F08B50248A8
:1092A00009F002FA002008BDE03DFF1F08B50248A2
:1092B00009F0E6F9002008BDE03DFF1F014809F074
:1092C000C6B900BFE03DFF1F38B522210A480A4C4D
:1092D00009F005F910B9204609F0A4F9074BD4F8B4
:1092E0009002DD682B681B6998472B68D4F89402BC
:1092F0001B699847012038BDE03DFF1F3C7A020002
:10930000022804BF0C4B93F8E80038B90B4BDB681C
:109310001B685B690A4AD2F898021847012809D1EC
:10932000054B93F8E830012B04D1044BDB681B6834
:109330009B69EFE7704700BF045AFF1F3C7A0200A9
:10934000E03DFF1F222970B50446154600F0FC825F
:1093500000F28E800E2900F01C8241D8062900F010
:10936000A98119D8022900F05E8107D8002900F0F0
:109370003D81012900F0498104243DE1042900F0E8
:10938000728140F26181002840F08D812621B94828
:1093900009F0A5F828602FE10A2900F0BA810FD85A
:1093A000072900F09F810829E6D1002840F0F985BF
:1093B0003521B04809F093F8C0F3402028601BE144
:1093C0000C2900F0C08140F2B2813421A948002C60
:1093D00040F0D18109F083F800F0010028600BE132
:1093E000152900F02A821FD8112900F0F5810DD827
:1093F0000F2900F0DC811029BED1002840F0E58162
:1094000025219C4809F06BF82860F5E0132900F04D
:10941000FF8140F2EF81002840F008822B2195481F
:1094200009F05DF82860E7E01B2900F041820DD8C3
:10943000172900F0108218299ED1002840F03182AF
:1094400033218C4809F04BF82860D5E01D2900F045
:109450005F82C0F0458221298ED1002840F06482CD
:109460000146844809F03BF800F001002860C3E0A1
:10947000AE2900F0238453D8A72900F08A832AD884
:10948000A32900F0D98210D88C2900F07782A22974
:109490007FF472AF6C217748002C40F0BE8209F057
:1094A0001EF8C0F3C1302860A6E0A52900F0F482C0
:1094B00040F2DA826C216F4809F011F800F480461E
:1094C000002C40F04583002E00F03783000900F0A7
:1094D0007000286090E0AA2900F09A8310D8A8298B
:1094E00000F06E83A9297FF447AF6D216148002CFD
:1094F00040F07D8308F0F3FFC0F3413028607BE04B
:10950000AC2900F0B58340F29B836D215948002CB3
:1095100040F0C58308F0E3FFC0F3006028606BE013
:10952000BB2900F0888436D8B62900F015841FD8EE
:10953000B42900F0E283B5297FF41EAF34214D48F1
:10954000002C40F0E78308F0CAFF430540F1E083B8
:109550001421484808F0C3FF474B30B14FF08072E8
:10956000B2FBF0F0834228BF03462B60002443E0A7
:10957000B92900F0238400F23984B8297FF4FCAEC5
:109580006C213C48002C40F00A8408F0A8FFC0F38E
:109590004030286030E0CC2900F0C68412D8BF29C2
:1095A00000F07E84C02900F09B84BC297FF4E4AEE7
:1095B00070213048002C40F0668408F090FFC0B263
:1095C000286019E0D12900F0C984D22900F0D6849E
:1095D000CE297FF4D1AE002840F0F2846F212548D7
:1095E00008F07DFFC0F30900286005E030B92D21A7
:1095F000204808F074FF2860204670BD12681D489E
:109600002D2108F05EFF0024F6E728B92121194832
:1096100008F065FF2860EFE712681648212108F07E
:1096200050FF0024E8E728B92721124808F057FF27
:109630002860E1E712680F48002AB8BF524227218C
:1096400008F03FFF0024D7E7002840F0A78422213C
:10965000084808F044FF10F4000318BF4FF07F43A0
:1096600018432860C8E7034E40B9D6F8B8321360F3
:10967000C2E700BFE03DFF1FFFFF0F001368A848CF
:10968000002BB8BF5B422021C6F8B83208F027FF94
:10969000044608B10024AFE7D6F8B822A048272135
:1096A00008F00FFFA8E712689D48262108F009FF7F
:1096B0000024A1E710219A482CB908F010FFC0F34C
:1096C0000420286098E708F00AFF2B681B0203F4C7
:1096D000F85320F4F8521A431021914808F0F1FE93
:1096E000002489E710218E482CB908F0F8FE00F01C
:1096F0001F00286080E708F0F2FE2B6820F01F02B0
:1097000003F01F031A431021854808F0DAFE0024F5
:1097100072E7002840F048843521814808F0DFFED8
:1097200010F0020F0CBF012300232B6064E7002818
:1097300040F03D8435217A4808F0D1FEC04300F066
:109740000100286058E7342175482CB908F0C7FE9D
:10975000C0F3400028604FE708F0C1FE2B685B00B3
:1097600003F0020320F002021A4334216C4808F08F
:10977000A8FE002440E708F0B2FE2B6820F00102AA
:1097800003F001031A433421654808F09AFE0024CF
:1097900032E728B93421624808F0A1FE28602BE79F
:1097A00012685F48342108F08CFE002424E728B9B1
:1097B00024215B4808F093FE28601DE71268584892
:1097C000242108F07EFE002416E712685448252163
:1097D00008F077FE00240FE728B92821504808F048
:1097E0007EFE286008E712684D48282108F069FECF
:1097F000002401E728B92A21494808F070FE2860B2
:10980000FAE6126846482A2108F05BFE0024F3E6D7
:1098100028B92321424808F062FE2860ECE612686D
:109820003F48232108F04DFE0024E5E612683C483D
:109830002B2108F046FE0024DEE628B92C2138480A
:1098400008F04DFE2860D7E6126835482C2108F054
:1098500038FE0024D0E688B91521314808F03FFED3
:1098600050B14FF08073B3FBF0F02E4B984228BFFD
:10987000184628600024BFE62A48FAE7136873B147
:109880004FF0807292FBF3F2264B9A42A8BF1A4621
:109890002A601521224808F014FE0024ACE6214A73
:1098A000F6E712681E48332108F00BFE0024A3E6F9
:1098B0006C211B482CB908F012FEC0F3C040286090
:1098C0009AE608F00CFE2B68DB0403F4002320F476
:1098D00000221A436C21124808F0F3FD00248BE6A5
:1098E0006C210F482CB908F0FAFDC0F380402860C5
:1098F00082E608F0F4FD2B689B0403F4802320F437
:1099000080221A436C21064808F0DBFD002473E630
:10991000002840F04F83024B5B6813606CE600BF89
:10992000E03DFF1FFFFF0F000021B84808F0D7FD02
:109930002B6820F0010203F001031A430021B34811
:1099400008F0BFFD002457E638B90146AF4808F0DB
:10995000C6FDC0F3400028604EE60021AB4808F089
:10996000BEFD2B685B0003F0020320F002021A43E5
:109970000021A64808F0A5FD00243DE658B96C2159
:10998000A24808F0ACFD4FF48073C0F3036043FAC3
:1099900000F0286030E61368102B27D00DDC022B76
:1099A00020D004DC012B16D04FF0FF3314E0042B41
:1099B0001AD0082BF8D105230EE0402B18D003DC79
:1099C000202BF1D1032307E0802B13D0B3F5807F48
:1099D000EAD1002300E008232B602B6801330BD170
:1099E000102409E60723F7E70623F5E70423F3E746
:1099F0000223F1E70123EFE76C21844808F06FFDB3
:109A00002B681B0603F0706320F070621A436C2110
:109A10007E4808F056FD0024EEE508F060FD2B6856
:109A2000DB0303F4C03320F4C0321A436C217748BF
:109A300008F047FD0024DFE56C2174482CB908F0DC
:109A40004EFDC0F380302860D6E508F048FD2B6855
:109A50009B0303F4804320F480421A436C216B483B
:109A600008F02FFD0024C7E56C2168482CB908F0E8
:109A700036FDC0F300302860BEE508F030FD2B68ED
:109A80001B0303F4805320F480521A436C215F4877
:109A900008F017FD0024AFE56C215C4808F01FFDBD
:109AA0000646CCB910F4804405D0C60906F4F06629
:109AB0002E600024A0E56C21544808F010FD16F03B
:109AC0000B0F4FEA201000F0700001D12860E1E593
:109AD00040F0080028608FE56C214C4808F0FFFC3E
:109AE00010F480444FF06C0148480ED008F0F7FCA9
:109AF0002B68DB0103F4F06320F4F0621A436C215D
:109B0000424808F0DEFC002476E508F0E8FC6C2111
:109B100020F400623D4808F0D4FC6C213B4808F07A
:109B2000DEFC2B681B0103F0700320F070021A4367
:109B30006C21364808F0C5FC5EE5C309020503F454
:109B4000F06301D42B60A5E543F008032B6053E5D7
:109B50006C212E4876B108F0C2FC2B681B0103F083
:109B6000700320F070021A436C21284808F0A9FC09
:109B7000002441E508F0B3FC2B68DB0103F4F0633B
:109B800020F4F0621A436C21204808F09AFC344615
:109B900032E56C211D482CB908F0A1FC00F00F0043
:109BA000286029E508F09BFC2B6820F00F0203F0E9
:109BB0000F031A436C21154808F083FC00241BE5B1
:109BC0006D2112482CB908F08AFCC0F3C03028601F
:109BD00012E508F084FC2B68DB039BB220F4004202
:109BE0001A436D21094808F06CFC002404E508F0D4
:109BF00076FC2B685B0303F4C04320F4C0421A4395
:109C00006D21024808F05DFC0024F5E4E03DFF1FF3
:109C10006D21B8482CB908F062FCC0F3032028601D
:109C2000EAE408F05CFC2B681B0203F4706320F488
:109C300070621A436D21AF4808F043FC0024DBE456
:109C40006D21AC482CB908F04AFCC0F341102860E3
:109C5000D2E408F044FC2B685B0103F0600320F0C1
:109C600060021A436D21A34808F02BFC0024C3E4D2
:109C70006D21A0482CB908F032FC00F00F002860DC
:109C8000BAE408F02CFC2B6820F00F0203F00F035D
:109C90001A436D21974808F014FC0024ACE408F046
:109CA0001EFC2B681B0603F0807320F080721A43A1
:109CB0006D21904808F005FC00249DE46D218D483D
:109CC00064B908F00CFC001400F07F0310F04000B1
:109CD00018BF6FF07F00184328608DE408F0FFFB89
:109CE0002B681B0403F4FE0320F4FE021A436D21CB
:109CF000804808F0E6FB00247EE4002840F05D8107
:109D00006F217C4808F0EBFBC0F30440286073E44B
:109D10002C6071E408F0E3FB2B68002B0CBF0023E0
:109D20004FF4806320F480621A433421714808F0B4
:109D3000C8FB2968704B69B14FF0807292FBF1F259
:109D40009A42A8BF1A462A6014216A4808F0B9FB53
:109D5000002451E41A46F6E7674E70B914216548AD
:109D600008F0BDFB30B14FF08073B3FBF0F08642DA
:109D700028BF06462E6000243EE413686BB14FF006
:109D8000807292FBF3F2B242A8BF32462A601421DD
:109D9000584808F096FB00242EE43246F6E708F017
:109DA0009EFB2B685B0303F4005320F400521A431C
:109DB0006C21504808F085FB00241DE46C214D48BF
:109DC0002CB908F08CFBC0F30350286014E408F0B1
:109DD00086FB2B681B0520F4700203F470031A4302
:109DE0006C21444808F06DFB002405E4424E78B92C
:109DF0001321404808F073FB30B14FF08073B3FB80
:109E0000F0F0864228BF06462E600024FFF7F4BB20
:109E1000136873B14FF0807292FBF3F2B242A8BFA5
:109E200032462A601321334808F04BFB0024FFF729
:109E3000E3BB3246F5E770212E4834B908F04FFBFA
:109E4000C0F307202860FFF7D7BB08F048FB2A685B
:109E5000120220F47F4092B202437021254808F09C
